:020000040800F2
:100000000000022015970008FD960008FD960008E4
:10001000FD960008FD960008FD960008000000000F
:10002000000000000000000000000000FD96000835
:10003000FD96000800000000FD96000805970008E6
:10004000FD960008FD960008FD960008FD96000844
:10005000FD960008FD960008FD960008FD96000834
:10006000FD960008FD960008FD960008F5180008AA
:10007000FD960008FD960008FD960008FD96000814
:10008000FD960008FD960008E5070008FD960008AB
:10009000FD960008FD960008FD960008FD960008F4
:1000A000FD960008FD960008FD960008FD960008E4
:1000B000410A0008610A0008FD9600088D0E00083C
:1000C000A5160008FD960008FD960008FD9600089C
:1000D00091090008650D0008FD960008FD960008CE
:1000E000FD960008FD960008FD960008FD960008A4
:1000F000FD960008FD960008FD9600080519000809
:10010000FD960008FD960008FD960008FD96000883
:10011000FD960008FD960008FD960008FD96000873
:10012000FD960008FD960008FD960008FD96000863
:10013000FD9600080000000000000000FD96000889
:10014000FD960008FD960008FD960008FD96000843
:10015000FD960008FD960008FD960008FD96000833
:10016000FD960008FD960008FD960008FD96000823
:10017000FD960008FD960008FD96000800000000AE
:1001800000000000FD9600080000000000000000D4
:10019000FD9600080000000000000000FD96000829
:1001A000000000000000000000000000FD960008B4
:1001B000FD960008FD960008FD960008FD960008D3
:0401C000FD960008A0
:10020000BFF34F8F0549064BCA6802F4E060034311
:10021000CB60BFF34F8F00BFFDE700BF00ED00E0F4
:100220000400FA0510B5174BDC68C4F30223C3F1D0
:10023000070CBCF1040F28BF4FF0040C1C1D062C4A
:10024000E6464FF0FF348CBFA3F1030C4FF0000CD7
:1002500004FA0EF321EA030104FA0CF422EA040280
:1002600001FA0CF313431901421CCCB206D000F181
:10027000604000F5614C8CF8004310BD014B83F8E1
:10028000234010BD00ED00E0F0B583B06F4A876DEC
:10029000166800230193C36D3D68082202FA03F13A
:1002A0002942044604D001680868400700F1A18093
:1002B00067489840284204D021684A69110600F135
:1002C0009180644A9A402A4204D0216808688007D5
:1002D00000F1818010209840284203D021680A68EC
:1002E000110766D44FF0200C0CFA03F0284215D009
:1002F00025682A68D50611D5B86094F83510052907
:1003000035D027683B68580340F187803B68190364
:1003100040F19280E56B0DB12046A847606D002842
:1003200045D0626DD2071BD527684B4D052184F857
:1003300035103B68A5FB061623F00100B20A3860B1
:1003400003E021680B68DB0704D5019F0137974262
:100350000197F6D90025012084F8345084F835003F
:10036000E36C23B3204603B0BDE8F040184726688D
:10037000326822F0160131602568686920F0800338
:100380006B61266C002E5CD021680D6825F008009A
:100390000860E66D3F23B340BB60236D00274FF03C
:1003A000010C84F8347084F835C0002BDAD103B026
:1003B000F0BDB86023681868400327D41968CA05DF
:1003C00003D41A6822F008001860216C09B1204695
:1003D0008847E36D86E7BA60636D43F004026265A7
:1003E000E36D77E7B860636D43F002006065E36D2D
:1003F00067E70B6823F004000860E16D8A40BA608B
:10040000626D42F001036365E36D51E71B681903F8
:10041000DBD5A16C0029DAD1DBE7386810F48075F0
:100420007FF478AF3A6822F010013960012784F830
:10043000345084F835706DE7656C002D7FF46CAF37
:100440006CE7A26C002A9FD1A3E700BF0000002048
:100450000100800004008000B5814E1B2DE9F04FA3
:100460000023734D734C83B04FF0010E4FF003091E
:1004700003E00133102B00F0BF800F680EFA03F287
:1004800002EA070A32EA0707F3D14F6827F010069D
:10049000022E14D1DF0800EB870803F007064FEAAD
:1004A000860CD8F820B00F690F2606FA0CF607FA6A
:1004B0000CF72BEA06063743C8F820704F68D0F8CF
:1004C00000B007F003064FEA430806FA08F709FAF6
:1004D00008F62BEA060C47EA0C0707604F6827F07E
:1004E000100B0BF1FF37012F6FEA060612D8876851
:1004F00006EA070CCF6807FA08FB4BEA0C0787608F
:100500004F68D0F804C0C7F300179F402CEA0202DE
:1005100017434760C7688A683E4002FA08F73E43BF
:10052000C6604A68D600A4D5002701976E6C46F4D1
:1005300080426A646F6C23F0030807F480460196DA
:1005400008F1804B019A0BF59C3203F003074FEA48
:10055000870C0F26976806FA0CF627EA0607364E30
:10056000B0421DD006F58068404548D0334EB042B9
:100570004AD0DFF8CCB058454BD0DFF8C8804045B2
:100580004CD0DFF8C4B058454DD0DFF8C0804045AE
:100590000CBF4FF006084FF0080808FA0CF6374376
:1005A00097604A6826686FEA0A0CD20354BF0CEAC7
:1005B00006064AEA060626604A686768960354BF3C
:1005C0000CEA07074AEA070767604E68A768F20265
:1005D00054BF0CEA07074AEA0707A7604E68E268BB
:1005E000B60203F1010354BF0CEA02024AEA020216
:1005F000102BE2607FF441AF03B0BDE8F08F01261D
:1006000006FA0CF63743CBE7022606FA0CF6374318
:10061000C6E7032606FA0CF63743C1E7042606FAB6
:100620000CF63743BCE7052606FA0CF63743B7E766
:1006300000380240003C0140000002400008024037
:10064000000C02400010024000140240001802405A
:10065000836B93F83D1093F83E202129C8B2D2B2A3
:1006600028D0222824D01968086820F480620A6003
:100670001968086840F400720A601968486820F434
:1006800080524A60196848684FF0000C20F40062FC
:100690004A60A3F82AC0186C48B94FF0200C83F8C0
:1006A0003DC093F83E1083F83E0040290FD07047BC
:1006B000202AD8D119684A6822F400624A60196871
:1006C000002058854B6843F440704860704770477D
:1006D000836B1868026800214FF0200C22F48062BE
:1006E0000260598583F83DC083F83E10196C41F0D3
:1006F00010001864704700BF836B1868016821F40C
:1007000080610160586B00225A850265996B4FF039
:10071000200C0A6593F83D0083F83DC083F83E2025
:10072000704700BF2D4A0368904210B43CD0B0F12E
:10073000804F27D0A2F57C44A04223D004F5806CE2
:1007400060451FD00CF58062904241D002F578449C
:10075000A04229D0224A904218D002F5806C604510
:1007600014D00CF58064A04210D0A4F598329042C9
:100770000CD002F5806C604508D00CF58064A04276
:1007800008D103E04A6823F070031343CA6823F4D6
:100790004073134303608C68C4620968816201235B
:1007A0005DF8044B436170474C68CA6823F07003DE
:1007B000234323F44073134303608A68C2620C68C6
:1007C00084620969016301235DF8044B436170474A
:1007D0004C68CA6823F070032343D8E70000014047
:1007E00000400140694A536819685868890701D573
:1007F00080064DD419685868490701D5000618D4F9
:1008000019685868C90701D5410606D4196858689F
:10081000890601D541017FD470471968C807F5D50D
:10082000516C6FF0010041F48031516418605368DD
:10083000ECE7516CC90603D4506C40F4005151648C
:10084000986810F4401F1ED1996B11F4401F02D01C
:100850009868400517D45968490514D49968D06937
:1008600001F0405101430ED1586820F080015960D9
:10087000506C20F480515164506CC00503D4516C0D
:1008800041F0010050646FF00C0119605368B7E744
:10089000516CC90603D4506C40F4007151649968DE
:1008A000D06901F04051014340D0D96C44F27C70D2
:1008B00089B200FB01F1C1F30F3C42F61F308445C1
:1008C000A2F84CC059D942F62D418C4558D942F670
:1008D000E550844557D943F2C7218C458CBF4FF072
:1008E000040C4FF0030C92F8400082F84EC001282F
:1008F0000DD0012182F84010986820F00101996024
:100900009868C00726D54FF0000C82F840C06FF001
:100910001201196053686DE7916C6FF0200041F08F
:10092000020191641860526810607047D86A10F430
:10093000700F1ED1586820F020015960506C20F4CF
:1009400080715164506CC104AFD4516C41F001000E
:100950005064AAE7596821F0806020F020015960B6
:10096000506C20F4885C2CF0010141F001005064CF
:10097000C9E79968480598D4DCE74FF0000CB2E766
:100980004FF0010CAFE74FF0020CACE74000012044
:1009900010B40A4B0A4A186DD3F88810C4680C804A
:1009A000196D4B684FF400744FF4806023F04003DE
:1009B0004B60946190615DF8044B704740000120EA
:1009C0000004024010B41B4A02F1A8031168116D23
:1009D000146883B0C2F88000C2F8883003E013685E
:1009E0001B1B642B17D88B689B07F8D50288CA603D
:1009F00000200190CC6801948B680193019B4A68A8
:100A000042F0400048600C6844F040030B6003B0C3
:100A10005DF8044B7047084B08249C614FF400625A
:100A2000402080214FF480549A61986199619C61C3
:100A3000FEE700BF4000012000000240704700BFF9
:100A400010B54FF080442369DB0706D503484168A1
:100A50008847226922F00103236110BD00000020B5
:100A60004A4B1869C10700D47047494B93F8AA2034
:100A70004AB193F8AB2062B946494FF4805088617F
:100A8000013283F8AB20414A136923F0010111615F
:100A9000704793F84E10481CB2EB400F6DDB0429F1
:100AA0006BD0122AECD910B493F8404083B00022E6
:100AB000012C019255D05968012083F840008C68C0
:100AC000E20714D4344A354C12688868A4FB024209
:100AD000940C04EB440240F0010088600192019CF8
:100AE0002CB10198421E0192019C002CF9D188681A
:100AF000C40736D55A6C22F4E06424F0010040F4B7
:100B000080725A644C68600505D5586C20F4405CCE
:100B10004CF480525A645C6C14F4805018BF986C8A
:100B20004FF0000418BF20F006006FF02202986416
:100B300083F840400A60596819484C6844F0806C5A
:100B40004CF020024A604068C20602D0154CA14217
:100B500007D18A6812F0405F03D1886840F0804472
:100B60008C600A4A002183F8AB10136923F001005E
:100B7000106103B05DF8044B70470648416981F489
:100B8000805C4CF0805181618BE700BF0004004025
:100B900040000120000002400000002083DE1B43D3
:100BA00000230140002001406B4B93F8E520202AF0
:100BB00001D00020704710B5684A212483F8E54031
:100BC00005294FF04004946140F29180002800F024
:100BD0008E804FF4047CA3F8ECC000EB010C0139CB
:100BE00011F003014FF0020236D010F8014B102C27
:100BF00004D183F8EE4010F8014C032203EB020EFF
:100C000001298EF8EC4002F1010225D0022911D011
:100C100010F8011B102906D19C18013284F8EC1041
:100C200010F8011C92B2541C1A4482F8EC10A2B2C3
:100C3000FC2A5CD810F8011B102906D19C1801323F
:100C400084F8EC1010F8011C92B2541C1A4482F87B
:100C5000EC10A2B2FC2A4AD810F8011B102906D1C8
:100C60009C18013284F8EC1010F8011C92B203EBCE
:100C7000020E541C84458EF8EC10A1B247D0FC291A
:100C800035D8024612F801EBBEF1100F06D15C1800
:100C9000013184F8ECE012F801EC89B24A1C92B2FE
:100CA0001944FC2A81F8ECE021D890F801E0BEF16B
:100CB000100F06D19C18013284F8ECE090F801E0A6
:100CC00092B2511C8CB21A44FC2C82F8ECE00ED883
:100CD00090F802E0BEF1100F00F1030033D021467E
:100CE0004C1CA2B21944FC2A81F8ECE0B4D91B4A8E
:100CF0001B48C3F8CC004FF0000C20214FF48004B7
:100D000083F8E510A3F8D2C09461002010BD901CB8
:100D100013FA80FC19441248C3F8CC000332A3F83C
:100D2000D220D3F8AC400D4A1020032381F8EC0008
:100D30008CF8EC30E3684FF4800143F08003E3600B
:100D40009161012010BD1A19013482F8ECE010F80D
:100D500001ECA1B2C4E700BF40000120000802403E
:100D60002C01012070B5474CD4F8AC301A68D96812
:100D7000950601D5880629D4160601D50D0604D49A
:100D8000500601D54A0619D470BDD4F8CC20511CA8
:100D9000C4F8CC1010785860B4F8D2C00CF1FF350C
:100DA000AEB2A4F8D260002EEED1DC6824F080024E
:100DB000DA60D96841F04000D86070BDD86820255D
:100DC00020F04006DE6084F8E55070BD2E4DD4F86A
:100DD000F021A8685B68111ADBB2882984F8EC312D
:100DE0000DD90021102BC4F8F00184F8F41184F817
:100DF000F511C9D14FF0010C84F8F5C170BD94F81C
:100E0000F5619EB3022B94F8F4610ED0032B1FD032
:100E1000102B13D1002EB7D04FF0000C501C84F8CB
:100E2000F5C1C4F8F001137070BD4EB9012284F809
:100E3000F56184F8F421C4F8F00170BD002EA3D050
:100E40000025C4F8F00184F8F45184F8F55170BD20
:100E5000002E99D00529F3D942798B1F9A42EFD100
:100E6000D4F8F81101B18847A860E9E7102BC1D088
:100E700094F8F461002E87D0501CC4F8F001137070
:100E800070BD00BF4000012000000020F0B5B04B55
:100E9000D3F8FC2195695169546893F83A021028F7
:100EA0008BB04BD0C6B2402E48D0AA48084000288C
:100EB00000F0C880A00500F15B81A74F2F40A74D2F
:100EC0000D40002F00F0F280A54F0F40002F00F0E2
:100ED0006D81660540F16A81002D40F06A8193F8CA
:100EE0003952B3F826C21FFA8CF1EEB221B3D3F80F
:100EF0002002441CC3F8204207781761B3F8265239
:100F000005F1FF3C1FFA8CF1A3F82612B3F8260274
:100F100084B28CB9292E0FD1566826F48067282018
:100F2000576093F8395293F83A2205F003010A43C7
:100F3000C3F82C2283F839020BB0F0BD11F0011F69
:100F400030D0A00500F1EA80834A84482A40084056
:100F5000002A4AD0824A0A40002A42D0670540D57A
:100F6000002800F08081A605E6D5D3F8285293F832
:100F700039022128E0D1B3F82642D3F8FC61A7B2A8
:100F8000002F00F05282D3F820727A1CC3F820227E
:100F900039783161B3F826C20CF1FF36B5B2A3F847
:100FA0002652C9E76F480840002840F0AF80694EDC
:100FB0000E40002EC8D0A605C6D593F83A72FEB2F0
:100FC000D3F82872D3F82CE293F839C2BCF1220F7F
:100FD00000F0888101905069019092690192019A14
:100FE000B2E70028BFD10BB0F0BD5F4D0D402DB36F
:100FF000650523D5002800F0F480A4059CD5D3F81E
:101000002842B3F82662D3F8FC11B7B2032F00F0E0
:10101000B581B3F8260282B2022A00F0C681D3F865
:1010200020520C696E1CC3F820622C70B3F826C2E3
:101030000CF1FF37B9B2A3F826127DE70028DCD106
:101040000BB0F0BD494F0F40002F3FF436AFA7055E
:101050007FF533AF93F839C2546824F4E0665660E4
:10106000099057690997146844F001061660D3F88F
:10107000FC71099A3A68ACF1280122F480640229D3
:101080005FFA8CF53C6040F25081D3F82C022228A4
:1010900002D0222D7FF450AF00254FF0200CC3F872
:1010A0002C5283F839C283F83A5245E72E4808405B
:1010B000002860D060055ED5002D5FD193F83942DD
:1010C000B3F826128FB2E6B2002F3FF435AFD3F853
:1010D00020521269681CC3F820022A70B3F826C295
:1010E0000CF1FF34A1B2A3F82612B3F82672BDB2F8
:1010F000002D7FF421AF2A2E7FF41EAFD3F8FC61C0
:10110000726822F48064282074600AE7A7057FF5DE
:101110001BAFD3F84072F8B2106115E793F83A624A
:10112000402E00F00D81D3F80C72B7F5804F00F01F
:10113000CC80D3F84C02002840F00B81D3F8400259
:10114000C61106F0060747F0F0001061FCE600BF8C
:101150004000012002000100040010000400010012
:1011600080000100080001004000010010000100A3
:1011700093699369E0E6002D3FF4DEAEA1057FF5AB
:10118000DBAEB3F82642A1B200293FF4D5AED3F8C6
:1011900020621269771CC3F820723270B3F826C23D
:1011A0000CF1FF35A8B2A3F82602C5E6002D3FF4E6
:1011B000C3AEA4057FF5C0AEB3F826C21FFA8CF10A
:1011C00000293FF4B9AED3F820526E1CC3F8206258
:1011D00028781061B3F82622541EA7B2A3F826720D
:1011E000AAE693F8390222287FF4A6AEB3F826C205
:1011F000D3F8FC111FFA8CF2032A3FF610AF951EAC
:10120000012DD3F8284240F260810E68022C14BFF1
:1012100026F4806646F480660E60D3F8FC71796827
:1012200021F4E0607860D3F820523A696C1CC3F86E
:1012300020422A70B3F826C20CF1FF36B7B2A3F8E9
:10124000267293F8391293F83A0201F00302104320
:101250002025C3F82C0283F83952002593F83A224E
:1012600083F83A5268E693F83942B3F8240293F8C7
:101270003A72D3F82862E2B2F9B2002840F08C80CA
:10128000212A00F0368140297FF456AE222A7FF4CD
:1012900053AEB3F82652ACB2002C00F0238193F881
:1012A0003A02402800F0B481D3F82042D3F8FC7110
:1012B000601CC3F8200222783A61B3F826C20CF110
:1012C000FF36B1B2A3F8261236E693F83962D3F8A6
:1012D0004072212E16BF47F0010707F0FE07FFB24C
:1012E000176131E6D3F84C0210B9402E00F01E8190
:1012F000D3F84C622EB9D3F80C02B0F5404F00F091
:101300002F81B3F82662B0B2002840F0A880069082
:1013100056690696976906970698106840F4007615
:1013200016600022C3F84C220EE6AC49C3F828121E
:101330002026C3F82C0283F8396283F83A02FBE5D1
:10134000D3F84C0298B9D3F8406206F0FE07176153
:10135000FAE5D3F84C62012E7FF4F6ADD3F8407273
:10136000F81100F0060646F0F1071761ECE5D3F836
:10137000406246F00107F8B21061E5E5042C0FD099
:10138000082C0DD014F5803F0AD0D3F82052D3F8A2
:10139000FC116E1C0C6946E6212A7FF474AF78E7D5
:1013A0000E6826F480670F60EFE7042C71D0082CDC
:1013B0006FD014F5803F6CD00F68022C14BF27F457
:1013C000806747F480670F6093F839C293F83A0258
:1013D0000CF003010843C3F82C02D3F82022D3F801
:1013E000FC51541C2E69C3F820421670B3F82672C3
:1013F000D3F82012D3F8FC0107F1FF3C1FFA8CF25E
:10140000A3F8262205694C1CC3F820420D70B3F8DE
:101410002662D3F8FC71711E88B2A3F826027A689E
:1014200022F4407420257C6015E7042D39D0082D66
:1014300037D015F5803F34D0726822F4E0617160D6
:1014400093F8396293F83A5206F0030005432024DA
:10145000C3F82C5283F83A7283F839426CE5B3F83A
:101460002662B0B2012800F08B80B3F82672BEB2BB
:10147000022E00F0B580106840F480671760D3F842
:10148000FC610022029270690290B7690297029A89
:1014900047E71225C3F82C520C6844F400760E601E
:1014A0009BE7726822F4E0657560306800214FF0B8
:1014B000200C40F400743460C3F82C1283F839C255
:1014C00093F83A2283F83A1236E5022C0C6800F0C1
:1014D000B38024F480670F60D3F8FC11086840F4EF
:1014E00000620A60D3F8FC516B6823F48061696084
:1014F00022E5042ED3F8FC711FD0082E1DD016F55E
:10150000803F1AD07C6824F4E0627A6093F83972E4
:1015100093F83A6207F003052E434FF0200CC3F80E
:101520002C6283F83A0283F839C205E508905069C5
:10153000089096690896089A06E57C6824F4E062AB
:101540007A603E680020202546F400713960C3F8B7
:101550002C0283F8395293F83A2283F83A02EBE4EA
:10156000079657690797906907900798166846F499
:1015700080771760D3F84C220132C3F84C22E3E4A1
:10158000042F18D0082F16D0BEF1120F13D0D3F8A5
:1015900028721068022F14BF20F4806040F480602D
:1015A0001060D3F8FC610022059277690597B06955
:1015B0000590059AB5E6166826F480601060D3F8A9
:1015C000FC71002204927E690496B8690490049824
:1015D0003A6842F400763E60A3E600BF0000FFFFD9
:1015E000D3F828621068022E2AD020F48066166094
:1015F000D3F8FC01026842F400670760D3F8FC21CD
:10160000002603965069039097690397039A88E62A
:10161000D3F84C72C7B9D3F84852D3F8FC11D3F8B9
:101620004442012D23D0C4F307270F61D3F84C02A5
:101630000130C3F84C027FE444F480660E6051E749
:1016400040F480671760D9E7D3F84C22012A16D0FE
:10165000D3F84C62022E7FF46FAC93F83912222932
:1016600019D093F83952212D7FF466AC1CE6E2B212
:101670000A61D3F84C620236C3F84C625CE4D3F8DA
:101680004472D3F8FC01FAB20261D3F84C6201361D
:10169000C3F84C6250E4D3F8FC512B6843F48074D7
:1016A0002C6049E470B58F4C8F48D4F8FC315A69EE
:1016B000596802423ED0CE0502F481354ED5D4F8A9
:1016C0003C6246F001006FF48076C4F83C025E6133
:1016D000002D00F09A80D4F83C526FF4007645F06B
:1016E000020012F4823FC4F83C025E6128D094F8F4
:1016F0003A52B4F826C294F83902D4F82C62202D5C
:101700001FFA8CF1C0B200F08580D4F83C1241F091
:101710000406C4F83C621D6845F400711960D4F8F1
:10172000FC316FF48060586112F4843F16D0D4F815
:10173000FC310AE012F4813F58D112F4823F59D1B2
:1017400012F4843F0AD0C90508D5D4F83C226FF4BE
:10175000006642F00805C4F83C525E61D4F83C02D1
:1017600000B970BD94F839C2ACF12901012945D9FD
:1017700094F83932602B4FF000021CBF202384F80C
:101780003932C4F82C2284F83A22D4F8FC010168DA
:1017900021F400630360D4F8FC613268120555D56A
:1017A000706820F400617160D4F83002002855D0D0
:1017B00090F835304D4E0665022B54D0802343659A
:1017C000FEF79AFF94F83962282ECAD1D4F83C2249
:1017D0005307C6D500254648C4F828022021C4F87E
:1017E0002C5284F8391284F83A5270BDCD053FF579
:1017F00072AFB3E7C8053FF57AAFAFE700262825FB
:10180000C4F82C6284F83952BFE712F4823F7FF4A7
:101810006EAF95E700297FF478AF00F0F705212D32
:1018200005D028287FF471AF212E7FF46EAF94F895
:101830003962D4F828020428F5B21DD008281BD03C
:10184000212D32D06FF4806159616DE794F83952DF
:10185000602D04BF202584F83952B3E7D4F8340250
:101860000028A5D1AEE70268052580F8355010683C
:1018700020F001011160A5E7282DE1D11C4DC4F82D
:10188000285259686FF4806021F4E0665E60586108
:101890001D6825F48061196000202023C4F82C0203
:1018A00084F8393284F83A023EE7114EC4F82862CF
:1018B00094F839C294F83A520CF003000543202101
:1018C0000026C4F82C5284F8391284F83A625D6814
:1018D0006FF4806025F4E061596058611E6806402D
:1018E0001E6021E74000012000010100F906000808
:1018F0000000FFFF024BD3F83402FEF7C5BC00BF67
:1019000040000120024BD3F83002FEF7BDBC00BFFF
:1019100040000120034AD2F850320133C2F850325D
:10192000704700BF4000012038B5104A92F8543289
:10193000112B00D938BD0E480E4D41690133DCB280
:1019400081F4807C4CF08073836115F8141082F868
:101950005442002001F06CFC05EB44020120517858
:1019600001F066FC0448047338BD00BF400001204C
:10197000000802408C9C00080000002038B5104A86
:1019800092F8543203B938BD0E4841695C1EE4B286
:1019900081F4007545F00073122C82F85442836183
:1019A000F1D8094D002015F8141001F041FC05EBA9
:1019B00044020120517801F03BFC0448047338BD17
:1019C00040000120000802408C9C0008000000201C
:1019D00008B5234B2349D3F850224FF080600132E1
:1019E000C3F850228861D3F85812D3F85C22914290
:1019F00024D0D3F85802D3F85C1288421BD0D3F815
:101A00005C22D0B2043003EB400EBEF858C2D3F8CB
:101A10005C1201311FFA8CFCC3F85C121248A3F867
:101A200060C4FEF7CFFF114A536983F0200040F4F1
:101A30000011916108BD4FF6FF7CEFE793F8623427
:101A400053B90B48FEF7BEFF0848416981F04002D8
:101A500042F48003836108BD0648FEF7B3FFF3E755
:101A60004000012000040240A004012000080240C0
:101A7000B49C0008B29C000838B5234C94F8632449
:101A8000D4F85032054652B1D4F8640438B1D4F8D1
:101A900068145A1A142A2FD90023C4F86434D4F8CD
:101AA0006C04D4F87014D4F8742401309142C4F852
:101AB0006C0423D0D4F87434D9B2043104EB41025D
:101AC000B2F87004D4F8743401331FFA80FCC4F8FF
:101AD000743400B2D4F878260C49288001320C4DB9
:101AE0000869C4F87826C2F30E0405EB4403A0F895
:101AF00000C00B61012038BD8047CDE74FF0FF30BB
:101B00004FF6FF7CE6E700BF400001200000002008
:101B1000400000200120704701207047024B93F8DD
:101B20007F160170012070474000012000EB010C7E
:101B300002464BF6AD21002012F8013B80EA032358
:101B400018B20028ABBF5B0081EA40009BB283B2B1
:101B500018B20028ABBF5B0081EA40009BB283B2A1
:101B600018B20028ABBF5B0081EA40009BB283B291
:101B700018B20028ABBF5B0081EA40009BB283B281
:101B800018B20028ABBF5B0081EA40009BB283B271
:101B900018B20028ABBF5B0081EA40009BB283B261
:101BA00018B20028ABBF5B0081EA40009BB283B251
:101BB00018B20028ABBF5B0081EA400098B280B247
:101BC0009445B9D1704700BF70B4194D040C012C75
:101BD000D5F8FC6104D113E02C68E41AA2421BD3AF
:101BE000B46920EA0404A4B2B4FA84F464098C420F
:101BF000F2D0002070BC70472C68E41AA2420BD3CC
:101C0000746920EA040C1FFA8CF4B4FA84F46409B1
:101C10008C42F1D00020EDE700232022C5F82C32C1
:101C200085F8383285F83922032070BC704700BF30
:101C30004000012010B41849D1F8FC41636913F049
:101C4000800326D1626912F4806211D10B681B1ADD
:101C5000012BF3D9D1F83C0281F83822202420430B
:101C6000C1F83C02C1F82C22032081F839420DE072
:101C70006FF48062626104202024C1F83C0281F884
:101C80003832C1F82C32012081F839425DF8044B1A
:101C900070470020FAE700BF40000120024BB3F874
:101CA0004C10018002207047400001200120704745
:101CB0000020704708B5024B024A1A60FEF7A0FAEE
:101CC00000C00120AD700DB00020704708B5FEF7D0
:101CD00097FA00BF0020704700207047024B93F82E
:101CE0008016017001207047400001204379012BCC
:101CF00001D00120704780790228FAD8084A0128CB
:101D000082F88006F5D192F8811621B105494FF489
:101D100000628A61EDE7034B4FF000609861E8E7ED
:101D20004000012000080240084B5969642202FB70
:101D300001F111F5001304D503F57F1C0CF57F5359
:101D40003F339A1502700120704700BF0000002049
:101D50004379012B01D0012070478079421E632A0C
:101D6000F9D8054A054983053233A2FB032042090D
:101D70004A610120704700BF1F85EB510000002021
:101D8000024B197E01700120704700BF0000002047
:101D90004379012B01D0012070478079421E072A28
:101DA0009CBF024A10760120704700BF000000204F
:101DB000064B4FF0000C197F5B7F80F800C00122BA
:101DC00041708270C3700420704700BF0000002083
:101DD000084B997FDB7F002261F3070263F30F2238
:101DE0008908013361F317429B1063F31F6202609D
:101DF00004207047000000204379022B01D001200D
:101E0000704710B483799A08911E06290BD80F4C9D
:101E1000E17F013103F0FC03B2EB910FA377BCBF6C
:101E200003F1FF33E377C07901308408A21E062A4C
:101E300007D80648837FB4EB930F02D8A1004C1E4D
:101E4000C47701205DF8044B704700BF00000020FC
:101E5000024B93F863140170012070474000012089
:101E600000B50B4B93F8201093F821C093F828206D
:101E7000417093F8293080F802C04FF0000E012124
:101E800080F800E0C1700271437106205DF804FB28
:101E900000000020034B0B2193F882260270417052
:101EA00002207047400001204379012B01D001201E
:101EB000704780790A289CBF024A82F88206012076
:101EC000704700BF4000012010B5134BB3F830C07D
:101ED00004464FEA4C10B0EB0C0162EB02025302D5
:101EE000480210EB0C0043EAD15141F1000293018A
:101EF000810143EA906E081A6EEB020E10EB0C00A3
:101F0000064A4FF000034EF1000104F0CFFB0246F9
:101F10002280022010BD00BF00000020400D030001
:101F20004379022B01D001207047C0880649074A37
:101F300001FB00F09042F6D8054B0649A3FB0020B8
:101F4000820C0A8601207047400D03003F62B007F3
:101F500083DE1B43000000204379012B01D00120C8
:101F60007047807905289CBF024A82F883060120C9
:101F7000704700BF40000120054B06495B6B064AD5
:101F8000591A8B1002FB03F303700120704700BF46
:101F900000000020B89C0008ABAAAAAA0120704744
:101FA000034B13211A7B027041700220704700BF5F
:101FB000000000201B4B93F88426032A30D810B56C
:101FC00019491A4C0A69B0F807E090F806C083F87E
:101FD00084C6141B6210002183F88516C3F8881686
:101FE000C3F87826B0F80910A3F88C161EF4004F39
:101FF0001FFA8EF01CBF4FF4004E70468CB208BF23
:102000008646844288BFA3F88C06BCF1010FA3F872
:102010008EE604BF83F885C6C3F88826012010BD6C
:1020200000207047400001200000002040000020F8
:10203000002070474379012B01D00120704782793D
:1020400022B10549012081F890367047024880F896
:1020500090260120704700BF40000120044B93F8F8
:10206000901602460B1E18BF012301201370704703
:1020700040000120074B084AD3F894364FF47A7198
:1020800001FB03F39909A2FB01239A0902600420D2
:10209000704700BF40000120632D3E054379042BAB
:1020A00001D001207047D0F806000649064A01FB1E
:1020B00000F0A2FB002305499809C1F8940601200D
:1020C000704700BF400D0300D34D62104000012057
:1020D00000207047002070470020704700207047A4
:1020E0000120704701207047114BB3F898260280F9
:1020F000B3F89A164180B3F89C268280B3F89E16F6
:10210000C180B3F8A0260281B3F8A2164181B3F8CA
:10211000A4268281B3F8A616C181B3F8A82602824C
:10212000B3F8AA164182B3F8AC3683821620704702
:1021300040000120012070470020704701207047B7
:1021400030B5334BDC7F002C59D014F00701314AF5
:102150004FF000032BD0012922D002291BD00329E4
:1021600014D004290DD0052906D006294BD132F808
:1021700002CB20F813C0013332F8021B20F81310F1
:10218000013332F8025B20F81350013332F802CBEE
:1021900020F813C0013332F8021B20F8131001336A
:1021A00032F8025B20F813500133A34227D01146C6
:1021B00003F1010C31F802EB20F813E0558820F808
:1021C0001C5003F1020E498820F81E10DD1CD18836
:1021D00020F815101D1D118920F815105D1D51895D
:1021E00020F815109D1D918920F81510DD1D08336C
:1021F000D18920F81510A34202F11002D7D1600056
:1022000000F0FE0030BD32F8025B05800123AEE72E
:1022100000000020F00601200020704701207047D8
:10222000184BDA7F997F01328B1A48BF03339A101B
:10223000013212F0FF0321D0134A012BB2F8F0163D
:1022400001801BD0B2F8F2164180022B16D0B2F8F2
:10225000F4168180032B11D0B2F8F616C180042B3E
:102260000CD0B2F8F8160181052B07D0B2F8FA1697
:102270004181062B1CBFB2F8FC268281580000F079
:10228000FE00704700000020400001200020704741
:102290002DE9F84381FB0141A50B5B0045EA81462E
:1022A000B6FBF2F7C11B4FEAE07060F10008A1FB3A
:1022B000030403FB0841002304F0A8F9002976DB9E
:1022C000B0F1004F71F1000474DB0B4606460121AA
:1022D000B50845EA8376B6F1004F4FEAA3034FEA0B
:1022E000410773F10000F9B2F2DA9803002440EAE2
:1022F0009645B20300234FF0804E9E0846EA8E7347
:102300009A424FEAAE0E75EB0E00F6DB53EA0E0072
:102310004DD04FF00008464613EB080046EB0E0C7C
:10232000824275EB0C094FEA93070BDBB2EB000915
:1023300065EB0C05DB184EEB0E0213EB080846EBC1
:1023400002064A464FEA580047EA8E734FEAAE0E3D
:1023500040EAC67853EA0E004FEA6606DCD14FEA3F
:10236000E87708FB04F4A8FB012C01FB074695184D
:10237000664446EB0601AB1846EB010778015D01A8
:1023800040EAD3645B1947EB04019A1846EB010657
:10239000002E0CDB12F5005746F10009B80B40EA9D
:1023A0008944FF2C28BFFF24E0B2BDE8F883002059
:1023B000BDE8F8838A0342EA9045012182030024A4
:1023C00098E700BF2DE9F0410026154C82B0804609
:1023D0004FF400753746D4F87024D4F874349A4218
:1023E0000DF10600F7D0FFF747FB0028F3D0BDF949
:1023F0000600013D00FB00F1ADB207EBA13706443A
:10240000002DE8D1314601234FF400723846FFF722
:102410003FFF0646012088F8006002B0BDE8F08169
:102420004000012030B5374D034605F11002002071
:10243000698803EA010414F00F0E05F1020C0CD0B8
:102440005FEA5E0555D05FEA9E048EEA050102D080
:10245000614081EADE0101F0010EBCF8025040004B
:1024600081B21D4041EA0E0015F00F010AD04C0860
:1024700041D08D0881EA040402D06C4084EAD10482
:1024800004F00101BCF8045044001D40A0B215F056
:102490000F0E40EA01000CD05FEA5E012DD05FEA2A
:1024A0009E048EEA010502D0654085EADE0505F04E
:1024B000010EBCF8061044001940A5B211F00F013E
:1024C00045EA0E000CF106050CD04C0817D05FEA67
:1024D000910C81EA040E03D08CEA0E0484EAD10E3A
:1024E0000EF001014400A0B2954240EA01009FD1E4
:1024F00030BD0121AFE70124C2E70125D7E74FF046
:10250000010EEDE7CE9C0008224910B5864601F188
:102510002004002031F8023F0EEA0302C2F30A034E
:102520007BB35A0834D05FEA930C82EA030226D0C8
:102530008CEA02025FEAD30C21D082EA0C025FEA45
:10254000131C1CD082EA0C025FEA531C17D082EAEB
:102550000C025FEA931C12D082EA0C025FEAD31CE1
:102560000DD082EA0C025FEA132C08D082EA0C023A
:102570005FEA532C03D082EA932383EA0C0202F031
:102580000103400082B2A14242EA0300C2D110BD61
:102590000122F4E7DE9C000870B5334C0D4604F1CF
:1025A000080E114600223EF8023D0340520013F08F
:1025B000FF0392B21CD05E0824D083EA060C9E086A
:1025C00013D08CEA060CDE080FD08CEA060C1E092C
:1025D0000BD08CEA060C5E0907D08CEA060C9E092B
:1025E00003D08CEAD31383EA060C0CF001063243C5
:1025F000A645D8D10AB3072A07D84FF6FF7008803E
:10260000002070BD4FF0010CEFE7A2F1080414F0B8
:10261000FF0221D1C0F34014C0F3C00242EA4406D5
:10262000C0F3800343EA4604C0F3400040EA440696
:1026300001220A802E80012070BDC0F3401CC0F32F
:10264000C003C0F3800443EA4C0644EA4606C0F3E4
:10265000400040EA4606ECE7C2F108060123B34019
:10266000434098B2D6E700BF009D00082DE9F04135
:10267000DFF898C105460F4616469CE8070084B06F
:1026800001AB984603C30DF10E0E00241A803EF8EC
:10269000020D640015EA0001A4B240D04A084BD0F4
:1026A000880881EA020337D05FEAD10C83EA00038D
:1026B00032D00A0983EA0C032ED0480983EA0203C8
:1026C0002AD05FEA911C83EA000325D0CA0983EA75
:1026D0000C0321D0080A83EA02031DD05FEA512CC3
:1026E00083EA000318D08A0A83EA0C0314D0C80ACC
:1026F00083EA020310D05FEA113C83EA00030BD0A7
:102700004A0B83EA0C0307D0880B83EA020303D049
:1027100083EAD13181EA000303F001031C43F04551
:10272000B5D1002C40D00F2C08D84FF6FF750020F3
:10273000358004B0BDE8F0810123EDE7A4F1100875
:1027400018F0FF045BD1C5F34031C5F3C02343EA61
:102750004104C5F3802242EA4400C5F3402141EA26
:102760004004C5F3C01C4CEA4408C5F3801343EA97
:102770004802C5F3401040EA4201C5F3001444EAA0
:10278000410CC5F3C008C5F3800248EA4C0342EA95
:102790004300C5F3400545EA40010124012034808F
:1027A000398004B0BDE8F081C5F3403CC5F3C023D7
:1027B00043EA4C08C5F3802242EA4800C5F34021B1
:1027C00041EA400CC5F3C01343EA4C00C5F380183E
:1027D00048EA4002C5F3401141EA420CC5F3001338
:1027E00043EA4C00C5F3C00242EA4001C5F380034E
:1027F00043EA4100C5F3400545EA4001CEE7C4F194
:10280000100201209040684085B29CE7089D0008B6
:102810001C491D4A4B6992F805C783F0400343F4F5
:1028200080038B6192F804178C4502D092F8303700
:1028300003B9704792F806C7D2F8001741F82C0088
:1028400092F8061792F8040701315FFA81FC92F8BA
:10285000051782F806C760458CBF0131013103F1CD
:10286000FF3398BF00205FFA81FCD9B298BF82F88D
:10287000060702EB810082F805C7D0F8080782F846
:1028800030177047000002404000012010B4194C7E
:10289000D4F8FC1107E04A6912F0100C0BD1236840
:1028A0001A1A012A18D84B6913F04003F3D00020FC
:1028B0005DF8044B70476FF010004FF0200C48613A
:1028C000C4F83C3284F83832C4F82C3284F839C267
:1028D00001205DF8044B7047D4F83C0284F838C2FC
:1028E00020210843C4F83C0284F8391203205DF823
:1028F000044B70474000012070B41B4ED6F8FC51C9
:1029000007E06C6914F4806316D13468A41AA142FC
:1029100008D36B6920EA0304A3B2002BF1D1184657
:1029200070BC70472022C6F82C3286F8383286F800
:102930003922032070BC7047286840F40071296078
:10294000D6F8FC5100246FF48063042220216B61CF
:10295000C6F83C2286F83842C6F82C4286F839126E
:10296000012070BC704700BF40000120F8B5254C25
:10297000D4F82832042B16460746D4F8FC210D461D
:1029800008D0012B06D013F5803F03D0D4F82C02D9
:10299000122803D1116841F480731360D4F8FC212C
:1029A00003E02068811B8D4214D35069C307F8D51A
:1029B000D4F80C12B1F5804F17D117611248324686
:1029C0002946FFF799FF20B1D4F83C42042C0AD1E4
:1029D0000120F8BD00234FF0200CC4F82C3284F8FD
:1029E000383284F839C20320F8BDF0231361074858
:1029F00032462946FFF780FF0028E5D1D4F8FC21B4
:102A00001761DBE74000012002000100080001001F
:102A100010B51E4CD4F83407C36823F00101C1601F
:102A2000036A41F2111213420AD1026A40F2444190
:102A30000A4205D1036823F001020260D4F834078A
:102A400013491123C4F84037FDF76CFED4F834273E
:102A5000D4F83C07136823F070030343D4F8440709
:102A600023F4407303431360D4F83437D4F8400799
:102A7000D4F83847D86201219C625961DA680A4368
:102A8000DA6018680843186010BD00BF40000120DC
:102A90007807012030B4454902680C6800250223FC
:102AA00080F8353080F83450156825F00103136044
:102AB000026803E00B681D1B052D4DD81568ED0756
:102AC000F8D4D0E90134C1682343D0E904540B435E
:102AD0002B432343D0E906412343046A15680B4383
:102AE00023433349446A2940042C43EA010303D1B8
:102AF000D0E90B5425432B4313600168426A4B69AC
:102B0000042A23F0070545EA020508D1826A846990
:102B1000154344BB012A43D0022A2BD052B34D6146
:102B2000036824495FFA83FCACF110021824B2FB5D
:102B3000F4F529446FF3090391F88810C1655F2A01
:102B400088BF04333F228A400024012583659A60B0
:102B5000446580F8355004E020210322416580F867
:102B6000352030BC7047B4F5005F0CD0022A04D980
:102B7000032AD4D1C26AD201D1D5402101254165B1
:102B800080F83550EDE7032AC9D801A454F822F0A3
:102B90007B2B0008752B00087B2B0008A12B00085D
:102BA000C36AB3F1C07FBAD1E7E700BF400001209C
:102BB0003F8010F08C9C00080D4B0E4A1868A2FB59
:102BC00000218B09013BB3F1807F0BD24FF0E02253
:102BD000094853614FF0F00C0021072380F823C00F
:102BE0009161136100220F214FF0FF30FDF71ABBF6
:102BF00000000020D34D621000ED00E030B4174B10
:102C0000D3F85822D3F85C12501AB0F5807F10D157
:102C1000134D14498024AC610A6922F00400086154
:102C200030BFD3F85822D3F85C02121AB2F5807F75
:102C3000F1D0D3F85852E9B2043103EB410C4FF410
:102C40000044ACF85842D3F85822054D4FF4000028
:102C50000132C3F85822A86130BC704740000120FF
:102C60000008024000ED00E0B0F5804F70B438DAA3
:102C700010F5804F32DB00F5804290B241001FFA20
:102C800081FC194AD2F85832D2F85C421D1BB5F5C6
:102C9000807F10D1154E16488021B161036923F061
:102CA0000404046130BFD2F85852D2F85C32EC1AF6
:102CB000B4F5807FF1D0D2F858620C48F1B20431FB
:102CC00002EB41054FF40004A5F858C2D2F858327F
:102CD0000133C2F85832846170BC70474FF0000C69
:102CE000CFE74FF6FF7CCCE7400001200008024010
:102CF00000ED00E0094B4FF4E052986892FAA2F31D
:102D00000749B3FA83F200F4E053D3400B4405487B
:102D100093F890100068C840704700BF0038024028
:102D20008C9C000800000020094B4FF4604298681A
:102D300092FAA2F30749B3FA83F200F46043D34056
:102D40000B44054893F890100068C840704700BFD6
:102D5000003802408C9C00080000002010B4644938
:102D6000644A4B6983F0800040F4000483B08C61B6
:102D7000D2F850120131C2F85012B2F8A83098B20D
:102D8000C4001FFA84FCACF580410BB2002B88B262
:102D900092F87017D2F85042BCBFCCF5804C0FFAB5
:102DA0008CF302EB410C013101F03F0182F8701706
:102DB000BCF97417ACF874375B1AD2F8F4170B44EB
:102DC000D2F8F817C2F8F4378B4254DAB2F8FE376B
:102DD00003F1FF3C21211FFA8CF3A2F8FC17A2F8A3
:102DE000FE37002B6BD0D2F87044D2F87434E11A5D
:102DF000B1F5807F31D13E48446984F4806C4CF059
:102E0000806383613C4B3D4C4FF0007199613C4BBA
:102E10001168C2F88040116D1068C2F8883003E074
:102E200013681C1A642C54D88C68A307F8D54AF68A
:102E3000AA220020CA600190CB6801938C6801949B
:102E4000019B4A6842F0400048600B6843F0400430
:102E50000C6003B05DF8044B7047D2F87014CCB22C
:102E6000043402EB440CACF87004D2F87004013066
:102E7000C2F87004C6E7D2F800188B4217DDB2F82A
:102E8000FC3703F1FF3C40F201211FFA8CF3A2F85A
:102E9000FE17A2F8FC37002BA5D11A49C2F86844E6
:102EA0004FF0210CC2F86414A2F8FCC79BE7212460
:102EB00040F2012CA2F8FC47A2F8FEC793E71249A2
:102EC000C2F8684440F2012CC2F86414A2F8FEC7AC
:102ED00089E70E4B08249C614FF40062402080215A
:102EE0004FF480549A61986199619C61FEE700BF3C
:102EF0000008024040000120000402402C9D000810
:102F0000E80001207D19000829190008000002408E
:102F10002DE9F043654C94F83932202B83B003D06F
:102F2000002003B0BDE8F08300220092226894F8EC
:102F300039620D78497884F804580227202E84F8E5
:102F4000051884F80479EBD1594B5A4E1D68E908ED
:102F5000A6FB01173B0A03EB830808EB8806D4F8AD
:102F6000FC51009603E0AB6913F002030CD0009F04
:102F7000791E0091002FF6D12026C4F82C7284F817
:102F8000387284F83962CBE794F83862012EC7D0E2
:102F90004FF0010C84F838C22F68474E27F40061C7
:102FA0002960D4F83012454FD4F8FC810B654FF0FE
:102FB00021094FF0100E84F8399284F83AE2C4F8EF
:102FC0003C32022591F834E0A4F82652C4F8287265
:102FD0003B4FCF63E6453B4FD1F858900B64C1E9B6
:102FE0001133A4F82452C4F82062CF6407D091F8BA
:102FF00035E081F834C0E64522D081F83430400015
:1030000080B22321FFF7B2FC064628B10020D4F895
:103010003C2284F8380283E7D4F8FC2101905369FC
:103020000193916901910199556845F48077576042
:10303000536843F400615160012084F8386270E7FE
:10304000D1F800C081F835504B65DCF8007027F4EA
:103050008027CCF800700F687D608D680F68402D68
:1030600008F110031ED0BE600E68F360CD6D3F27DF
:10307000AF40C9F808700E68336843F01605356034
:103080000F687E6946F080037B610D6C25B10F6887
:103090003E6846F008033B6009680D6845F001078B
:1030A0000F60ACE7BB600B68DE60DFE7400001202B
:1030B0000000002089B5F814440801200000FFFF3B
:1030C00051060008D106000870B53B4B3B4C082266
:1030D00082B09A61D4F85052FFF79AFC72B6384E1B
:1030E0003848706062B672B60021C4F85812C4F84D
:1030F0005C1262B6344B4FF4803202209A619861C0
:10310000D4F85012D4F850325A1AB2F5487F0BD284
:103110002E48036923F00402026130BFD4F8503214
:103120005A1AB2F5487FF4D394F882C6284961440C
:10313000002091F8A4E08DF8040001A92D208DF85D
:1031400005E0FFF7E5FE226D116841F00200106016
:10315000226D012384F86234136843F00101116089
:10316000FFF756FC72B61B48706062B6D4F8506226
:10317000721BB2F5166F15D205F51665AE1B11D090
:10318000D4F85002D4F85032191A8E420AD90F4A94
:10319000156925F00403136130BFD4F850120D1ADD
:1031A000AE42F5D8084C044E04204FF40022A06132
:1031B000B26102B070BD00BF0008024040000120B3
:1031C00000000020151900080000024000ED00E09A
:1031D0008C9C0008D1190008012804D80B4620B99E
:1031E000012911D970470020704710B50E4C82B0EC
:1031F000002201A92C2063778DF804208DF805307A
:10320000FFF786FE02B010BD0748017741B901F112
:10321000804C0CF502304FF48032826101207047FF
:10322000024901238B61F9E70000002000080240F9
:10323000012800D9704738B5094D05EBC0050C468B
:1032400095F82110A14200D838BD6A6A12F83410EE
:10325000FFF7C2FF0028F7D085F8204038BD00BF37
:1032600000000020134B144901229A61D1F850024A
:10327000D1F850321A1AB2F5C87F0BD20F4A13692F
:1032800023F00403136130BFD1F850321B1AB3F599
:10329000C87FF4D391F8630458B910B5084C94F87A
:1032A0002010FFF7C5FF94F828100120BDE810405A
:1032B000BEE77047000002404000012000ED00E042
:1032C0000000002070B54479012C01D0012070BDB0
:1032D0008579122DFAD8084E002016F81510FFF740
:1032E000A7FF06EB450120464978FFF7A1FF034BF6
:1032F0001D73012070BD00BF8C9C000800000020E1
:10330000F8B51C4C94F86334A3B194F8545215BB2F
:103310000122194E84F85422114617461546002002
:10332000FFF786FF06EB470101204978FFF780FF92
:10333000124B1D73124D134EC4F8005840F2012772
:1033400040200022A4F8FE77A4F8FC07C4F8642407
:10335000C4F8F867F8BD112D07D91120064E84F87E
:103360005402074601210546D9E7034E2F4616F8B9
:103370001510D4E7400001208C9C000800000020BC
:10338000DB1B0400B9A201004F4B082270B59A6103
:1033900072B64E4C0020C4F87004C4F8740462B6CF
:1033A00094F86214002968D0D4F85052D4F850022E
:1033B000D4F850321A1A632A0AD845490E6926F001
:1033C00004030B6130BFD4F85022161A632EF5D9CE
:1033D0003D48404B4FF400214FF4802281619A61B7
:1033E000D4F85062D4F85002831B632B0AD83849B2
:1033F0000A6922F00400086130BFD4F850329A1BE9
:10340000632AF5D9FFF72EFF2F48324E082181613C
:103410004FF400334FF480220020B36184F862043B
:10342000B261FFF7F5FA72B62B4E2C49716062B6A5
:103430002B4B2C484FF080629A61FDF7C3FAD4F809
:103440005002411BB1F5166F25D394F86354FDB9B2
:10345000206D036843F002020260246D216821F0B0
:1034600001052560FFF7D4FA72B61F48706062B696
:10347000154E4FF40023B36170BD164D4FF48026F6
:10348000AE61FFF7EFFE94F86354134E002DDFD0CA
:10349000FFF736FFDCE705F5166CBCEB000ED4D069
:1034A000D4F85052D4F850325A1B9645CDD908481A
:1034B000016921F00403036130BFD4F85022511B8D
:1034C0008E45F5D8C1E700BF00080240400001204A
:1034D00000ED00E000000240000000201519000887
:1034E00000040240B49C00085D2D00084379022BC3
:1034F00072D12DE9F0418479302C6FD8C579002D37
:1035000077D0642D6DD9424F424E4FF4804507EB82
:103510008404FFF7D9FDD4F8FC72BC1E07F2FE3715
:10352000B4F9022005FB02F242F38F30FFF79CFB57
:10353000B4F9040005FB00F040F38F30FFF794FB73
:10354000B4F9061005FB01F141F38F30FFF78CFB56
:10355000B4F9083005FB03F343F38F30FFF784FB26
:10356000B4F90A2005FB02F242F38F30FFF77CFB2F
:10357000B4F90C0005FB00F040F38F30FFF774FB4B
:10358000B4F90E1005FB01F141F38F30FFF76CFB2E
:1035900034F9103F05FB03F343F38F30FFF764FB6F
:1035A000A742BDD1FFF72AFBD6F85852D6F85C42A5
:1035B000A54208D0184F1020B861D6F85822D6F886
:1035C0005C128A42F8D1144E4FF48013B361FFF7B6
:1035D000DBFE0120BDE8F081002070470020BDE83F
:1035E000F0810E4A0A4F0B4EA803A2FB00214D09A1
:1035F0008DE7084E064F96F88386C8EBC80CCCEBD7
:10360000CC0EA64407EB4E03B3F9B0507FE700BFE2
:103610008C9C000840000120000802401F85EB51EF
:103620002DE9F84F4379022B02D00020BDE8F88F36
:103630000546714EDFF8CC81FFF746FDA979D6F833
:1036400000B000273846A6F53F7900296BD1FFF777
:103650000BFB0424BBF9020033E0FFF705FBB4F5D4
:10366000806F47D0A9793BF90400D6F800B0023446
:10367000002940F09880FFF7F7FAA9793BF9040098
:10368000D6F800A004F1020B00297CD1FFF7ECFA78
:10369000AA793AF90B00D6F800A004F1040B002A2D
:1036A00061D1FFF7E1FAAB793AF90B00D6F800A047
:1036B00004F1060B002B46D1FFF7D6FA3AF90B00BE
:1036C0000834AB79D6F800B0002BC6D098F8831632
:1036D000C1EBC102C2EBC20ABA4409EB4A0CBCF806
:1036E000B0E01EFB00F040F38F30FFF7BDFAB4F5F9
:1036F000806FB7D1EB7900243BB1FFF77FFA01343B
:10370000E979A4B2B4EB412FF7DB3C4A964207F1CA
:10371000010758D056F8043FA979B3F90000D6F84C
:1037200000B0002993D098F88326C2EBC204C4EB02
:10373000C40ABA4409EB4A0CBCF8B0E01EFB00F026
:1037400040F38F3083E798F88316C1EBC102C2EBD8
:10375000C20CBC4409EB4C0EBEF8B03013FB00F0B9
:1037600040F38F30A8E798F883C6CCEBCC0ECEEBB5
:10377000CE033B4409EB4301B1F8B02012FB00F04B
:1037800040F38F308DE798F88326C2EBC20CCCEB68
:10379000CC0EBE4409EB4E03B3F8B01011FB00F0A1
:1037A00040F38F3072E798F88326C2EBC20ACAEB67
:1037B000CA0CBC4409EB4C0EBEF8B03013FB00F051
:1037C00040F38F3057E7D8F85852D8F85C62AE42D1
:1037D00008D00B4F1023BB61D8F85802D8F85C1200
:1037E0008842F8D1064C4FF48012A261FFF7CCFD5D
:1037F0000120BDE8F88F00BF889F000848A000089E
:1038000000080240400001204379012B57D12DE9E7
:10381000F04132498079324A01FB00F0A2FB0024DA
:10382000A50905F58076B6F5006F4FEA562748D210
:10383000FFF74AFC4FF004082A4E00272A4CB4F93F
:103840000200FFF711FAB4F90400FFF70DFAB4F91A
:103850000600FFF709FAB4F90800FFF705FAB4F912
:103860000A00FFF701FAB4F90C00FFF7FDF9B4F90B
:103870000E00FFF7F9F934F9100FFFF7F5F9B4422C
:10388000DDD101374745D9D1FFF7B8F9174BD3F848
:103890005802D3F85C12814208D0154D1024AC6157
:1038A000D3F85862D3F85C229642F8D1104F4FF407
:1038B0008013BB61FFF768FD0120BDE8F0810020A7
:1038C000704740F2D138474502D9FFF7FDFBB3E717
:1038D0001FFA87F8FFF7F8FBAEE700BF80841E00F1
:1038E000D34D62104AA400084AA0000840000120FD
:1038F000000802402DE9F04FC279ADF20C4D0346AD
:10390000002A00F0DC801446197A09B901201872E7
:103910009D79002D00F0CB806B4A6C4E92F8831697
:1039200000924FF0000BC1EBC100C0EBC0055A463E
:10393000AF1806EB47092244B9F9B0A092B2302A79
:10394000D344F5D9624F019302A94FEAEB7A07F20B
:10395000FE390DF106060020C1F10208A7F5F86551
:10396000302C08EB060C98BF23460AD805EB830ED3
:103970002344DEF8FC229BB232F90C10302B0844B1
:10398000F4D9C3179A0342EA9041534680035A463A
:1039900002F03CFEB94526F8020F02D037F9020FBB
:1039A000DEE7FFF791FB0198047A002C61D0002735
:1039B0000DF2064680460DF10605711B8B1E5A0856
:1039C000013212F007000DF106042AD0012822D09E
:1039D00002281CD0032816D0042810D005280AD0AD
:1039E000062804D0BDF9080002ACFFF73DF934F910
:1039F000020FFFF739F934F9020FFFF735F934F9FF
:103A0000020FFFF731F934F9020FFFF72DF934F9FE
:103A1000020FFFF729F934F9020FFFF725F9B44235
:103A200021D0B4F90200FFF71FF9B4F90400FFF741
:103A30001BF9B4F90600FFF717F9B4F90800FFF70E
:103A400013F9B4F90A00FFF70FF9B4F90C00FFF706
:103A50000BF9B4F90E00FFF707F934F9100FFFF76F
:103A600003F9B442DDD198F808500137B9B28D425C
:103A7000A1D8FFF7C3F8009FD7F85862D7F85C3297
:103A80009E4209D013481025BC468561DCF8584297
:103A9000DCF85C229442F8D10E494FF480178F6114
:103AA000FFF772FC01200DF20C4DBDE8F08F064EC1
:103AB00000963127B7FBF2F84FEA883B42E7012234
:103AC0001446C27120E700BF400001208C9C000812
:103AD0004CA40008000802404379032B00D109E7F9
:103AE0000020704708B54379012B01D0012008BDA3
:103AF00082794AB109490A4A8020886182F8633490
:103B0000FFF7FEFB012008BD0548044B80F8632445
:103B10004FF400019961012008BD00BF0000024080
:103B20004000012038B54379022B01D0012038BD77
:103B30008179C5790129F9D8084C04EBC10494F8BE
:103B40002120AA42F2D9636A084613F83510FFF71C
:103B500043FB0028EAD084F82050E7E7000000206B
:103B60004379022B01D00120704781790129FAD8CD
:103B7000C27949B9012AF6D80D480E4B0277A2B98D
:103B80004FF480329A61EEE710B5094C82B04FF0E5
:103B9000000C01A92C2062778DF804C08DF8052057
:103BA000FFF7B6F9012002B010BD01219961DAE7F3
:103BB000000000200008024010B4094C84460FCCDD
:103BC000CCF8000020788CF81000CCF80410CCF869
:103BD0000820CCF80C3011205DF8044B704700BF72
:103BE0002CF202084379012B01D0012070472DE906
:103BF000F04180798B4C020211B2002986B084F822
:103C00007F06BABF4BF6AD2080EA4100400285B284
:103C10002EB2002EBABF4BF6AD2585EA46056D00E3
:103C2000AFB23BB2002BBABF4BF6AD2787EA4307D2
:103C30007F00B8B202B2002ABABF4BF6AD2080EACC
:103C40004200400081B20DB2002DBABF4BF6AD214B
:103C500081EA450149008EB237B2002FB6BF4BF65C
:103C6000AD26760086EA4706B3B218B20028B6BF82
:103C70004BF6AD235B0083EA400399B20AB2002AF7
:103C8000BABF4BF6AD2181EA42014900B4F87D6626
:103C90008DB2AE4210D094F83932A4F87D56FF2789
:103CA00084F87C76D4F87C06CDF805004FF0000847
:103CB000202B8DF8048003D0012006B0BDE8F081F0
:103CC0000DF1040CDCE90001D4F8008094F83922ED
:103CD000C4F804080525202A84F8045984F8081833
:103CE000EAD1D4F8FC6104E02768A7EB08001928A2
:103CF00025D8B169CF4317F00203F5D094F8380204
:103D00000128D9D0012184F83812326822F40065E4
:103D100035602127444E84F839721023002542462D
:103D2000A02084F83A32C4F83C52C4F82862FEF766
:103D30001DFE60B1D4F83C3284F83852BCE7202133
:103D4000C4F82C3284F8383284F83912B4E7D4F845
:103D5000FC31009059690091986900900099334FA7
:103D600005265A6912F080052BD1596911F480603B
:103D70001AD12568A5EB0802012AF2D9D4F83C62D1
:103D800020273E43C4F83C62C4F82C0284F8397200
:103D9000D4F83C520022042D84F838228CD11C68BF
:103DA00044F400761E6087E76FF4806004214FF0D2
:103DB000200C5861C4F83C12C4F82C5284F839C263
:103DC000E6E7BE46751E1EF8010B18615A695207D8
:103DD000A9B224D519B37D781D61023EB6B202376F
:103DE000596911F0040509D1596911F48060DBD1DA
:103DF0002568A5EB0802012AF2D9BFE7002EB0D151
:103E00001F68202047F400721A6084F839020120EC
:103E100084F8386284F83A6206B0BDE8F0810E4654
:103E20007746DDE7400001200000FFFF4408012045
:103E30002C4A2D49034630B42C4D10680C6818608C
:103E400003CD2B4AC3F80340C3F80A10C3F8060099
:103E500003CA284C1861596103CCB5F800C0264C40
:103E6000264D9861D961286825492568C3F8220044
:103E70003A22C3F82550234DA08883F8202031240E
:103E80000A68A3F80EC083F82140C3F82B20A3F8DA
:103E9000290007CD1C4CC3F82E00C3F8321003CC08
:103EA000C3F83620194AC3F83B00C3F83F10184D39
:103EB00024782D8883F8434003CAC3F84910A3F837
:103EC0004C5093F84C10C3F845004FF02C0C614552
:103ED00083F83AC083F844C014BF4D204C2030BC56
:103EE000704700BF40F2020844F2020848F202089C
:103EF00054F2020860F2020870F202086CF2020842
:103F000078F202087CF202088CF2020898F20208A9
:103F1000A0F2020808B5094B094993F8832600F876
:103F2000012B01EB820C7E22DCF8C01B05F0B2FBFA
:103F300002F086FC0130C0B208BD00BF4000012085
:103F40008C9C00082DE9F04FAB4AAC49AC4BAD4C12
:103F5000AD4DB1B0824602F50060CDE90D130C9273
:103F6000099001F5006603F500678022002110A882
:103F700008940F950A960B9705F03AFBA34C4FF463
:103F80000075D4F87024D4F874148A42F9D00DF175
:103F90001E00FDF771FD0028F3D0DDE908C066467C
:103FA000BDF91EB0BCF8021036F8043B0896DDE9F6
:103FB0000A72119EB0F8029011FB0BF141F38F3899
:103FC000464430F8041B11967E88099011FB0BF0D3
:103FD00037F8041B0A9719FB0BFC159F16FB0BF90E
:103FE00049F38F3640F38F3811FB0BF0518813FBE8
:103FF0000BF3374443F38F3E15974CF38F3311FB8C
:104000000BF740F38F3C109932F8040B0B9271447C
:1040100010FB0BF2DDE913E042F38F399E44DDE93A
:10402000163247F38F36129F1091B84484444B44A4
:104030003244CDE9128ECDF850C0CDE91632DDE91B
:104040000C86B8F8027038F8043BCDF8308013FBCA
:104050000BF917FB0BF7209BDDE90E0149F38F32BB
:1040600047F38F3C219FB0F802901A447388209246
:10407000BC4436F8047B0D9613FB0BF343F38F3EE1
:1040800017FB0BF34E88CDF884C019FB0BF243F3FA
:104090008F3830F8043B0E9042F38F3931F8042BFF
:1040A0000F9113FB0BF016FB0BF7279B47F38F3693
:1040B00012FB0BFB40F38F3C4BF38F313344DDE9B4
:1040C000242BDDE92260269F2793013D0F444644BF
:1040D00070446244CB44ADB2CDE92260CDE9242BDB
:1040E0002697002D7FF44DAF5646CAF800500DF1CB
:1040F000400C46F8045FDFF818A12F464FF0640922
:10410000E046331F4146CDF814801D46CDE90361DA
:10411000A8468E46AC1CAB463E46DEE9007080FBEE
:10412000002C87FB0771930BB80B43EA8C4540EAE0
:104130008142AB185ED49D1498034FF08041002358
:104140009F0847EA817398424FEAA10175EB01028B
:10415000F6DB53EA01024FF000022ED0CDE9008BCE
:104160001746CDF808E013EB020C41EB070E604553
:1041700075EB0E0B4FEA930809DBB0EB0C0065EB17
:104180000E05DB1841EB010B9A1847EB0B0748EAC9
:1041900081738910520853EA010C42EAC7724FEA50
:1041A0006707E0D109FB02F00028DDE9008BB8BF0A
:1041B0005044DDF808E0C0F3875208F8012B44456D
:1041C0000EF1080EA9D13746039E0499A64201F1CB
:1041D000100101D0254699E7DDF814C002375D468D
:1041E000042F05F106060CF140088AD1082031B0F1
:1041F000BDE8F08F0022E0E764B0000864C000086A
:1042000064D0000864A8000864E0000840000120B1
:10421000FFFF3F0007490023C1F89836C1F89C36DC
:10422000C1F8A036C1F8A436C1F8A836A1F8AC365A
:10423000012070474000012008B5402200210248BB
:1042400005F0D6F9012008BDF0060120054900233C
:10425000C1F8F036C1F8F436C1F8F836A1F8FC36EA
:10426000012070474000012070B5A6B00646982294
:10427000144C0021684605F0BBF9FE220123256895
:104280008DF802208DF805308DF8066003E0206877
:10429000411B642907D807216846FCF785FC0028E4
:1042A000F5D026B070BD084E08234FF400624024BC
:1042B00080254FF48050B361B261B461B561B061E3
:1042C000FEE700BF40000120000002402DE9F04F52
:1042D000724D95F80C6995F80D39B34285B00446D6
:1042E0003BD095F83007C0B3E17801F00303012B10
:1042F00000F08780022B00F09F80A1787F2930D0CA
:1043000095F80E29D5F8081995F8807641F82240DD
:1043100095F80E4995F80D0995F80C6901345FFA86
:1043200084FB5E4598BF4FF0000B013085F80EB955
:1043300085F80D09012F05D1594B85F881764FF489
:1043400000629A6195F830473CB1611ECFB205EB2F
:10435000870885F83077D8F80847204605B0BDE8CB
:10436000F08F6379002BCBD0677895F87F96B945AD
:1043700001D0FF2FC4D1D4F890B0D5F8ACA9494AE8
:10438000D4F80690ABEB0A00A0FB02010023464ADA
:1043900002F08CF9A0EB090808EBD8714B10A3F1DF
:1043A000220727EAE77095F88076022F6BD0D5F8C0
:1043B00050823D4A0090A8EB0A0CDFF8E8A00023E9
:1043C000ACFB0A0102F072F9A8EB0B01364A01902E
:1043D0000023A1FB0A0102F069F9CDE902091020CE
:1043E000E9466071B9E80F0095F80DE9C4F80600D8
:1043F000B645C4F80A10C4F80E20C4F8123099D09B
:104400007EE795F87F0694F8018080457FF475AFCC
:104410009822002105F6141085F8103905F0E8F807
:1044200085F814892778237985F815797F2685F80A
:10443000166985F8183963E795F87F766278BA428D
:1044400002D0FF2A7FF459AF95F8901600297FF427
:1044500054AF98221548012685F8106905F0C8F870
:1044600085F814792378277985F815397F20042178
:1044700085F8160985F8187985F81919D4F8942063
:10448000C5F81A293CE706494A6982F4006343F0FB
:1044900000628A61D4F890B089E700BF4000012033
:1044A0000008024040420F00400D03005409012063
:1044B0002DE9F04FDFF8E082B349D8F83890202298
:1044C000ADF2DC4D8A6199F805B0BBF1000F07D160
:1044D0004FF40010886101200DF2DC4DBDE8F08F33
:1044E00099F80300A94F10F0040F14BF0C26002602
:1044F000C0F38003B91903EB4304A7F12C0606EBC4
:10450000840ABBF10C0F9AF82CC09AF82D70009118
:104510008CBF022501255D440CEBC505B4AC6A1EB9
:10452000C8F83410B2FBFCF500216A0020461FFADF
:1045300085FA05F05DF8002F00F09C800AF1FF304D
:104540001FFA80FE0DF2D223914ACDF8049003EBBE
:104550004E0C00208023002D00F08680ACEB040977
:10456000A9F102014E08013616F00306214633D0A8
:10457000012E20D0022E0FD0218892F800E04E00AC
:1045800013EA0E0F214618BF46F0010621F8026B10
:104590005B0804BF013280230E8892F800907600F9
:1045A00013EA090F18BF46F0010621F8026B5B08F9
:1045B00004BF013280230E8892F800E0760013EAEF
:1045C0000E0F18BF46F001065B0821F8026B01D1FF
:1045D00001328023614547D0B1F800E092F80090A5
:1045E0000E4613EA090F4FEA4E0118BF41F00101D0
:1045F00026F8021B5B08B64608BF01323EF8021BD4
:1046000092F8009008BF802313EA090F4FEA410196
:1046100018BF41F001015B082EF8021C01D1802374
:104620000132718892F800904FEA410E13EA090FA7
:1046300018BF4EF0010E5B0808BF013206F10601FB
:10464000A6F802E092F80090B68808BF802313EA2B
:10465000090F4FEA460618BF46F001065B0821F82D
:10466000026CB5D06145B7D10130B8427FF473AF69
:10467000DDF80490002D00F071820AF1FF318EB256
:104680000DF2D22B0BEB460A32AF1AF0020F414D5E
:10469000DFF8F4904FEA4606BB4616D02088009C0F
:1046A0000DF14202A36839460DF2D2249847002842
:1046B00058D0BDF84200002840F03A82D8F83420A3
:1046C0000092A24507F1020B69D0009B41E0BDF8C2
:1046D00042300BF1020B0DF142025946A3B1B5F87D
:1046E000A8C6D8F838E05CFA83F09EF888C0A5F830
:1046F000A80663448EF88830D9F8143083F040005F
:1047000040F48003C9F81830D8F83400836834F8CE
:10471000020B984730B3BDF842000BF1020BA0B179
:10472000D8F83810B5F8A82691F888E052FA80F346
:10473000704481F88800A5F8A836D9F8140080F0F4
:10474000400141F48002C9F81820A245D8F834305D
:1047500024D09B6834F8020B0DF142025946984769
:104760000028B4D1084D0B4E6B69B6F8AA7683F0D9
:10477000800242F400010137A961A6F8AA76002060
:104780000DF2DC4DBDE8F08F00080240B89C000837
:10479000FE090120400001200000002000930DF1DF
:1047A000440A82220021504604F022FF009DCDF8E9
:1047B0003CA095F80090012009F1FF34A04081B29F
:1047C000B1FA81F2C0F30B14C0F34A11C2F11F0316
:1047D000BD1CC0F3891203940491C0F3C814C0F344
:1047E0000721AE1905920694C0F34622C0F3852432
:1047F0000791C0F3C42102930096002386B2C0F350
:104800004E0CC0F38D0EC0F3CC0B08920994C0F38C
:104810000332C0F342340A91C0F38131C0F3C03097
:104820000B920C940D910E901A465446019600E09E
:104830000235019E002E00F0688139885F000E422B
:1048400018BF47F001073BB202F00707072F02F13C
:10485000010008BF04F8013B80B20CBF00239BB2EB
:10486000BCF1000F00F04E8111EA0C0F4FEA430338
:1048700018BF43F0010300F0070A1BB2BAF1070F9B
:1048800002F1020608BF04F8013BB6B20CBF0023D8
:104890009BB2BEF1000F00F0358111EA0E0F4FEA16
:1048A000430318BF43F0010306F007061BB2072EAF
:1048B00002F1030908BF04F8013B1FFA89FA0CBF93
:1048C00000239BB2BBF1000F00F01C810AF0070629
:1048D00011EA0B0F4FEA430318BF43F00103072E01
:1048E000039E1BB202F1040908BF04F8013B1FFA42
:1048F00089FA0CBF00239BB2002E00F003813142E5
:104900004FEA43030AF0070618BF43F00103072EDE
:10491000049E1BB202F1050908BF04F8013B1FFA0F
:1049200089FA0CBF00239BB2002E00F0EB803142CD
:104930004FEA43030AF0070618BF43F00103072EAE
:10494000059E1BB202F1060908BF04F8013B1FFADD
:1049500089FA0CBF00239BB2002E00F0D3803142B5
:104960004FEA43030AF0070618BF43F00103072E7E
:10497000069E1BB202F1070908BF04F8013B1FFAAB
:1049800089FA0CBF00239BB2002E00F0BB8031429D
:104990004FEA43030AF0070618BF43F00103072E4E
:1049A000079E1BB20ABF04F8013B9BB20023002EF6
:1049B00000F0A88031424FEA430318BF43F00103DF
:1049C000072F089F1BB202F1090608BF04F8013B3C
:1049D0001FFA86F90CBF00239BB2002F00F09280D3
:1049E00039424FEA430318BF43F0010309F00706B9
:1049F000099F1BB2072E02F10A0A08BF04F8013B07
:104A00001FFA8AF90CBF00239BB2002F7AD03942DB
:104A100009F007064FEA430318BF43F00103072ECE
:104A20000A9E1BB202F10B0708BF04F8013BBFB29C
:104A30000CBF00239BB2002E64D031424FEA4303E7
:104A400018BF43F0010307F007060B9F1BB2072EA8
:104A500002F10C0A08BF04F8013B1FFA8AF90CBFE7
:104A600000239BB2002F4DD0394209F007064FEAD0
:104A7000430318BF43F00103072E0C9E1BB202F143
:104A80000D0708BF04F8013BBFB20CBF00239BB267
:104A9000002E37D031424FEA430318BF43F00103E1
:104AA00007F007060D9F1BB2072E02F10E0A08BF82
:104AB00004F8013B1FFA8AF90CBF00239BB20FB325
:104AC00039424FEA430318BF43F0010309F00706D8
:104AD0000E9F1BB2072E02F10F0208BF04F8013B24
:104AE00092B20CBF00239BB267B101F0010141EA11
:104AF000430602F00702072A37B20ABF04F8017B17
:104B0000BBB200230299084482B2009885422F4626
:104B10007FF48EAED8F83890DDF83CA099F805B057
:104B2000BBF10C0F24D8BBF1000F79D16949CFE458
:104B3000D8F83810B5F8A8E691F888C05EFA80F287
:104B4000604481F88800A5F8A826D9F8143083F0CD
:104B5000400040F48001C9F81810AFE50DF1440A97
:104B600082222946504604F043FDBBF10C0F57D971
:104B70000DF14605D04605EB0B0C00234BF6AD249A
:104B800018F8016B83EA06273BB2002BB9B2B3BF1A
:104B900084EA430349008BB29BB21AB2002AABBF2E
:104BA0005B0084EA42029BB293B218B20028ABBF0A
:104BB0005B0084EA40009BB283B21DB2002DABBF04
:104BC0005B0084EA45059BB2ABB21EB2002EABBFC0
:104BD0005B0084EA46069BB2B3B21FB2002FABBFA4
:104BE0005B0084EA47079BB2BBB219B20029ABBF96
:104BF0005B0084EA41019BB28BB21AB2002AABBFC0
:104C00005B0084EA42029BB293B2C445B8D1002B48
:104C100059D03148B0F8A6460134A0F8A646AEE512
:104C20000BF1010400235FFA84F8D4461A463FE0F2
:104C30004500EEB274B2002CBABF660086F097064B
:104C40007600F0B243B2002BBABF580080F0970054
:104C50004000C5B26EB2002EBABF750085F0970550
:104C60006D00EFB279B20029BABF4F0087F0970705
:104C70007F00F8B244B2002CBABF600080F0970009
:104C80004000C3B25DB2002DBABF6B0083F0970342
:104C90005B00DEB277B2002F02F10102B8BF7E00E6
:104CA000D2B2ACBF760086F097064245F3B2AED2E0
:104CB0001CF8010B584043B2002BB9DA5F0087F0B3
:104CC0009701CEB2B6E75A46514609F1060001F007
:104CD00007FD2BE700080240400001202DE9F04FBE
:104CE000C178DFF83491447911F0040F14BF0C231C
:104CF0000023ADF2A44D09F12C051D4403AF454B33
:104D00000646C1F380082246811D38465D6301F0E6
:104D1000E7FC0C2C00F28280002C00F05E82BE4684
:104D20003A19002026E04800C1B24BB2002B2EDB1E
:104D30004900CBB258B2002830DB5B00D9B248B290
:104D4000002832DB4900CBB258B2002834DB5B00CC
:104D5000D9B248B2002836DB4900CBB258B200289D
:104D600038DB5B00D9B248B200283ADB49009645EF
:104D7000C8B23DD01EF8011B41404BB2002BD2DA25
:104D80005B0083F09700C1B24BB2002BD0DA580021
:104D900080F09701CBB258B20028CEDA400080F004
:104DA0009703D9B248B20028CCDA400080F09701CE
:104DB000CBB258B20028CADA400080F09703D9B2CB
:104DC00048B20028C8DA400080F09701CBB258B250
:104DD0000028C6DA400080F09703D9B248B2002814
:104DE000C4DA430083F0970A96455FFA8AF0C1D18E
:104DF0000DF1900B38554FF402720021584604F023
:104E0000F7FB08EB480209EB82094FF0010899F81B
:104E10002CC066E0000000208C9C0008601E0DF194
:104E20000D0212FA80FABB4600234BF6AD211BF8A7
:104E3000010B83EA00231AB2002AABBF5B0081EAB0
:104E400042029BB293B218B20028ABBF5B0081EA6A
:104E500040009BB283B21AB2002AABBF5B0081EA6A
:104E600042029BB293B218B20028ABBF5B0081EA4A
:104E700040009BB283B21AB2002AABBF5B0081EA4A
:104E800042029BB293B218B20028ABBF5B0081EA2A
:104E900040009BB283B21AB2002AABBF5B0081EA2A
:104EA00042029BB293B218B20028ABBF5B0081EA0A
:104EB00040009BB283B2DA45B9D13A19190A0DF113
:104EC000900B39555846537000214FF4027204F08C
:104ED0008FFB08EB480309EB83094FF0020899F8B0
:104EE0002CC03878A0444FEAC801614401F1FF3E6C
:104EF0009EFBFCF3002B40F3B38000224FF0800AAE
:104F0000009401956446D9469646D4461D464FF016
:104F1000000129F8021B002C00F09980002314F0F6
:104F2000030A194640D0BAF1010F27D0BAF1020F97
:104F300010D01CEA000F14BF012300235FEA5C0CB1
:104F400007D10132D2B290458CBFB85C60464FF0B9
:104F5000800C01211CEA000F4FEA430318BF43F005
:104F600001035FEA5C0C9BB207D10132D2B29045DB
:104F70008CBFB85C60464FF0800C01311CEA000F1A
:104F80004FEA430318BF43F001035FEA5C0C9BB296
:104F900007D10132D2B290458CBFB85C60464FF069
:104FA000800C0131A14250D01CEA000F4FEA4303AC
:104FB00018BF43F001035FEA5C0C9BB207D10132DA
:104FC000D2B290458CBFB85C60464FF0800C1CEAB2
:104FD000000F4FEA430318BF43F001035FEA5C0A86
:104FE00001F101019BB207D10132D2B290458CBFD1
:104FF000B85C50464FF0800A1AEA000F4FEA4303AC
:1050000018BF43F001035FEA5A0C9BB207D101328B
:10501000D2B290458CBFB85C60464FF0800C1CEA61
:10502000000F4FEA430318BF43F001035FEA5C0C33
:105030009BB207D10132D2B290458CBFB85C6046BA
:105040004FF0800C0331A142AED129F8023C0EF1A1
:1050500001011FFA81FE75453FF759AFDDE90045B3
:10506000A6AF4FF402720021384604F0C1FAB946E7
:105070004FF000082CB10C2C8CBF022301231C44E0
:10508000E4002A781319581E90FBF2F141450BDD1C
:105090006A683BF8020B9047594B29F8020B747968
:1050A0005D6B08F10108E5E76E780125741EA540E7
:1050B000ACB288B2002C00F08C80421E1FFA82FB3A
:1050C000BB1C504A03EB4B05002300287ED0E91B94
:1050D0008E1E7108013111F003013E4638D00129BE
:1050E00023D0022910D0117836F802AB013314EA2C
:1050F0000A0FDBB24FEA410118BF41F00101082B52
:10510000117004BF00230132117836F802CB01334D
:1051100014EA0C0FDBB24FEA410118BF41F0010164
:10512000082B117004BF00230132117836F8028B6E
:10513000490014EA080F03F10103DBB218BF41F084
:105140000101082B117004BF00230132B5423DD08C
:105150003146167831F8029B0133DBB214EA090FAD
:105160004FEA460618BF46F00106082B167004BF2A
:10517000013200231678B1F800E0013314EA0E0F73
:105180004FEA4606DBB218BF46F00106082B167040
:1051900001D1002301321678B1F802B0B1F804A0B1
:1051A000013314EA0B0FDBB24FEA460618BF46F094
:1051B0000106082B167008BF013201F106061178AE
:1051C00008BF0023490014EA0A0FB4E764087FF41B
:1051D0007CAF0DF2A44DBDE8F08F0DF1900B214690
:1051E0004FF4027258463C7004F002FA08EB480093
:1051F00009EB8008214698F82CC02046A04674E6AA
:1052000000000020120B01202DE9F843374A384DE9
:105210005369384F064683F0020040F40031916133
:1052200005F6D83000214FF42A7204F0E1F9002489
:10523000B000314B314E324985F8804EA5F8844E8E
:1052400005F6886C05F6986EA7F5FF68DCF8042073
:10525000DCF80090034401449342CCF8001041D0A4
:10526000CCF804300021CEE90011CEE90211A6F5F8
:105270000053C3E90011C3E90411C3E90811C3E9EC
:105280000C11C3E91011C3E91411C3E91811C3E9E2
:105290001C118033B342ECD19CB957F8044FA1786C
:1052A00094F8009008EB810308EB8902D3F80038EA
:1052B000D2F800180CF1080C08360EF1100E01247B
:1052C000C4E70A4C0F4810490422A2616669C5F878
:1052D000000886F0020747F40033C5F8F817A36109
:1052E000BDE8F8834945D7D0BCE700BF00080240BD
:1052F0004000012064E8000864C80008544401200C
:1053000064A80008DB1B0400B9A201002DE9F04FDE
:10531000114D124AB5F8983604464FF40061A3B017
:105320000133916105F6C4204FF489720021A5F87C
:105330009836002604F05CF9FDF7C6FEA7882068C1
:10534000ADF84C70A5F8B86E12900DF148090DF14A
:105350004E0A374608E000BF40000120000002402E
:105360005300CA45DFB243D019F8012B7A4055B239
:10537000002DBABF6A0082F097025200D3B259B230
:105380000029BABF4B0083F097035B00DEB270B216
:105390000028BABF460086F097067600F7B27AB2C8
:1053A000002ABABF570087F097077F00FDB26BB2A3
:1053B000002BBABF5D0085F097056D00E9B24EB2D3
:1053C000002EBABF710081F097014900CFB278B2C8
:1053D0000028BABF470087F097077F00FAB255B29E
:1053E000002DBDDA690081F09706CA45F7B2BBD13E
:1053F0000023CDE91B33CDE91D33CDE91F338DF8F3
:105400004E700DF16A0B9DF8487021930DF18600E6
:10541000D9464FF0800C07EA0C02D5B2291ECCF316
:10542000470E18BF0121BEF1000F40F05D8101332E
:10543000DBB2062B4FEA410109D803F188080DEBD6
:10544000080717F9406C17F840EC41EAD671CEF323
:10545000801545EA41084FF0200C1EEA0C0F4FEA78
:10546000480218BF42F001025FEA5C0792B240F0C6
:1054700094850133DBB2062B4FF0800C05D803F185
:1054800088070DEB070616F8407C29F8022F4845DF
:10549000C1D10023CDE91433CDE91633CDE918335A
:1054A000C24D1A933BF8022FDFF80893002139F818
:1054B000027F02EA070616F00F030CD05F0887EAA6
:1054C000030700F06E819E0887EA060601D086EA8F
:1054D000D30707F00103490089B2A94541EA030156
:1054E000E5D183452AF8021FDCD1BDF85000BDF894
:1054F0005250BDF85A70BDF85E60BDF86230BDF81C
:105500005620BDF8661005900495029706960793FD
:105510000820BDF85480BDF858E0BDF85CC0BDF867
:105520006070BDF86460BDF86850BDF86AB0A04B0B
:105530000392089100228021019005980842187872
:105540004FEA400018BF40F001005FFA80FA04986B
:1055500008424FEA4A0018BF40F001001870901C42
:10556000C0B2082840F02881587818EA010F14BF0B
:105570000122002242EA40025A70013301220398BC
:10558000084218784FEA400018BF40F00100187038
:10559000501C5FFA80F9B9F1080F40F04E815A783B
:1055A0001EEA010F4FEA420018BF40F00100587098
:1055B0000122013302980842187814BF4FF0010904
:1055C0004FF0000949EA40001870501CC0B208288A
:1055D00040F0258193F8019011EA0C0F14BF0122CD
:1055E000002242EA49025A70013301220698014220
:1055F000187814BF4FF001094FF0000949EA400044
:105600001870501CC0B2082840F0FC8093F801903C
:105610000F4214BF0122002242EA49025A700133AC
:10562000012207980142187814BF4FF001094FF08A
:10563000000949EA40001870501CC0B2082840F028
:10564000D48093F80190314214BF0122002242EA33
:10565000490058700122013308980142187814BF9C
:105660004FF001094FF0000949EA40001870501C42
:10567000C0B2082840F0AD805A7829424FEA420073
:1056800018BF40F0010058700122013318781BEA5E
:10569000010F4FEA400018BF40F001000132D2B2C2
:1056A00018700198082A04BF0133002201384FEA1C
:1056B000510101907FF441AFA77866797F2F00F008
:1056C000CA80002E00F0CA802046FFF707FB6479ED
:1056D000002C00F0C3800C2C8CBF4FF002084FF060
:1056E00001084444E500BAE007EA0E06F2B24D00B4
:1056F000002A18BF45F001051CF47F7FCCF3870E0C
:105700001DD10133DBB2062B16D803F188020DEB55
:10571000020E1EF9401C1EF8407CCE0F46EA4506DC
:10572000C7F3801545EA460229F8022F48454FF095
:10573000200C7FF470AEACE66E007746F0E717EA17
:105740000E0F4FEA4501CCF3C70C0CBF884641F061
:105750000108BCF1000F40F01D840133DBB2062BC1
:1057600013D84FF0400C03EB0C0648360DEB060245
:1057700012F9405C12F8407CE90F41EA480229F82E
:10578000022F48457FF447AE83E64FEA4807BAB296
:1057900029F8022F484567464FF0400C7FF43BAE96
:1057A00077E6012707F0010395E600BFDE9C0008BD
:1057B000040B0120CE9C0008187818EA010F4FEA6C
:1057C000400002F1030218BF40F00100D2B218708D
:1057D000D5E693F800A0294214BF01200020023230
:1057E00040EA4A00D2B2187050E793F800A0314264
:1057F00014BF01200020023240EA4A09D2B283F8E5
:10580000009029E718780F424FEA400902F102029E
:1058100018BF49F00109D2B283F8009001E7187867
:1058200011EA0C0F4FEA400902F1020218BF49F0D9
:105830000109D2B283F80090D8E618781EEA010F69
:105840004FEA400902F1020218BF49F00109D2B241
:1058500083F80090AEE6002E40F07C830025D74808
:10586000436B847F93F800E05978D54801947544E0
:105870006A1E92FBFEF711FB07F67036B6B290F87F
:105880008356A0F8B86E002C00F07F83C5EBC501ED
:10589000CC4CCD4F0297CDE904654FF0000AC1EB27
:1058A000C1024FEAC50C0392202104F5806B01234D
:1058B000D046D146CDF818C0039DEE18029B03EBED
:1058C000460E6818BEF9B02003EB4001D717B1F9B6
:1058D000B050BE0346EA92415619F3179003324680
:1058E000079300F093FE0746E8178103079B3246B3
:1058F00041EA9541A80300F089FE0BF2FE33ABF1BB
:1059000002050646C346023C9846B4F90200B5F9C2
:1059100002C006FB00F007FB0C02A91CA31C42F30B
:105920008F3008910793FDF79FF90798089AB0F90F
:105930000210B2F9023006FB01F107FB031040F33D
:105940008F30FDF791F9B4F90610B5F9062006FB82
:1059500001F107FB021343F38F30FDF785F9B4F92A
:105960000800B5F9081006FB00F007FB010242F33E
:105970008F30FDF779F9B4F90A30B5F90A0006FB62
:1059800003F307FB003141F38F30FDF76DF9B4F9F4
:105990000C30B5F90C2006FB03F307FB023040F393
:1059A0008F30FDF761F9B4F90E10B5F90E3006FB32
:1059B00001F107FB031242F38F30FDF755F934F97B
:1059C000100F35F9101F06FB00F007FB010343F32E
:1059D0008F30FDF749F9454597D1D846B9F1000F09
:1059E0001BD14FF00109019E0AF1010AB24523D0F3
:1059F000764F029D07EB8902D2F8F80710F80830BD
:105A000000EB080605EB830CB178DCF8FC4205EBF3
:105A1000810EA346DEF8FC424EE70BF101075FFA68
:105A200087F8B8F1010F4FF00009DCD9019E0AF1A7
:105A3000010AB245C846DBD1DDE90465DDF818E0AE
:105A4000DFF890910496AEEB0504C4EBC402002786
:105A500001970392A9F5006AA9F580640E214FF021
:105A6000130C0595F046039846180299844401EBFF
:105A7000460B01EB4C0CBBF9B030BCF9B050DA1757
:105A80005E19900340EA934132469803F317069358
:105A900000F0BCFDE9178346880340EA9541324691
:105AA000A803069B00F0B2FDAAF102050646023CDF
:105AB0000AF2FE3AB4F90220B5F902E006FB02F25E
:105AC0000BFB0E23A91CA21C43F38F3007910692F7
:105AD000FDF7CAF80698079BB0F90210B3F9022047
:105AE00006FB01F10BFB021040F38F30FDF7BCF811
:105AF000B4F90610B5F9063006FB01F10BFB0312F1
:105B000042F38F30FDF7B0F8B4F90800B5F908108A
:105B100006FB00F00BFB010343F38F30FDF7A4F805
:105B2000B4F90A20B5F90A0006FB02F20BFB0021CA
:105B300041F38F30FDF798F8B4F90C20B5F90C302B
:105B400006FB02F20BFB032040F38F30FDF78CF8CD
:105B5000B4F90E10B5F90E2006FB01F10BFB021390
:105B600043F38F30FDF780F834F9100F35F9101F2B
:105B700006FB00F00BFB010242F38F30FDF774F8D7
:105B8000554597D1019E3EBB01240194104B994588
:105B90002CD019F8010F0D4B029C03EB800ADAF8A8
:105BA000F867F519F15D95F802C004EB810B04EB81
:105BB0008C0EDBF8FCA2DEF8FC4254E7000000206B
:105BC0004000012030E900088C9C00086CE00008CF
:105BD00033F9000830F900080137FFB2012F40F215
:105BE000B681CB4B002799450197D2D1C94ADDE94F
:105BF0000461147E0794002E00F04E81A8EB01058D
:105C0000C5EBC5070D97C44C002701974FF0800BDB
:105C100094F800C01BEA0C0F14BF012000205FEABB
:105C20005B0340F0648162784FF02009D1090134B0
:105C3000C2F38012237819EA030F14BF0123002353
:105C40005FEA590B02D101344FF0800B079D0437F6
:105C5000BFB2002D00F01D81B04D05EB800A05EBB1
:105C6000810E05EB820805EB830CCDE90E67CDE9CB
:105C7000104BDAF8D007DEF8D017D8F8D027DCF8C8
:105C8000D037029C099000250A910B920C93049541
:105C9000019EA24B099F0A980B990C9D334493F8DF
:105CA000D89793F8DBA793F8DE8793F8E12793F86A
:105CB000E46709EB490B0AEB4A0E08EB480C02EBD0
:105CC000420986448C4493F8E70793F8EA1793F85F
:105CD000ED37A944BB441CF801501BF8067019F8B5
:105CE00003201EF800600D990392C8198B19039ABE
:105CF000089504EB430E04EB400B4D1904EB4508EB
:105D000004EB870A1144BEF9B090BBF9B000DAF891
:105D1000FC72B8F9B0B0059704EB410C09EB000335
:105D2000BCF9B0705B44FD18C2174FEAE5789103E7
:105D300043462A4641EA9041800300F067FC8246D0
:105D40004FEAE970830343EA99412A4643464FEA02
:105D5000893000F05BFC4FEAEB72910343462A4620
:105D600041EA9B4181464FEA8B3000F04FFC2A46C6
:105D7000FD170690A803434640EA9741B80300F098
:105D800045FC089F039B04EB870804EB860604EBA5
:105D90008302D6F8FC128346D8F8FC02D2F8FC52F3
:105DA000059B0394069C8F1E861E023DA3F10208EC
:105DB00003F2FE31B7F90220B8F90200B6F902E0A9
:105DC000089109FB02F1B5F902C00AFB001204FBBD
:105DD0000E210BFB0C1308F10202B11C43F38F30B0
:105DE00006920591FCF740FF069BB7F90400059960
:105DF000B3F90220B1F9023009FB00F00AFB0202FC
:105E000004FB0321B5F904300BFB031040F38F3082
:105E1000FCF72AFFB7F90620B8F9063009FB02F1B2
:105E2000B6F906200AFB0310B5F9063004FB02019F
:105E30000BFB031040F38F30FCF716FF37F9082FE8
:105E400038F9083F09FB02F136F9082F0AFB031065
:105E500035F9083F04FB02010BFB031040F38F30C0
:105E6000FCF702FF08994145A4D1019F049D079AC0
:105E7000039C0137FEB2032E05F1010508BF002681
:105E80009542049501967FF403AFDDE90E67DDE9E5
:105E9000104BBE423FF6BCAEFCF7B0FE2049D1F835
:105EA0005802D1F85C3298420FD01E4F1E4E10257A
:105EB000BD61346924F00402326130BF1849D1F861
:105EC0005802D1F85C329842F2D1164F144A174E5C
:105ED0004FF48015BD61D2F850124FF00064B461E8
:105EE000C2F8AC1923B0BDE8F04FFDF74DBA13EA84
:105EF0000C0F14BF012100215FEA9B0218D16378C7
:105F00004FF0200BDA090134C3F380139EE600BF83
:105F100033F9000800000020040B012064F10008A0
:105F2000400001200008024000ED00E000000240B7
:105F300012EA0C0F14BF012200225FEADB097FF492
:105F400079AE65784FF0400BEB0901347EE6002511
:105F500001951BE6134E2046D6F85052FEF7BEFEC2
:105F6000D6F85032D4F806200F49C5EB4300871A03
:105F7000A7FB01010D4A002300F098FB6679C4F8E5
:105F80000600002E7FF4A0AB68E4094B02934FEAB1
:105F9000C50E55E5BE46FFF760BABC467746FFF72B
:105FA00074BA00BF4000012040420F00400D0300C2
:105FB0008C9C00082DE9F04F4B4C94F8BB3E00221E
:105FC000A3B084F8BA2E002B00F00F83474800F5E9
:105FD0007F68CDF81C80464994F8C07E0D7B94F80C
:105FE000C19ED4F8BC6EAF4228BF2F46A94538BF2A
:105FF000A94640222E44002112A8C4F8BC6E84F8A1
:10600000C07E84F8C19E03F0F3FA94F8C22E94F88F
:10601000C30E0132D3B2984284F8C23E00F0CF8260
:106020003249344E344ACD1895F8D8A795F8E4B7DC
:106030000AEB4A0CB444DC449CF8F8769CF804E77C
:1060400002EB870802EB8E09D8F80018D9F800088F
:10605000264D284E2B44CDE90A1093F8DBA793F880
:10606000DEC793F8E72793F8E1E793F8EA9793F808
:10607000ED370AEB4A0BB34493440CEB4C07F01991
:106080000EEB4E089BF804179BF8F8764844B04492
:10609000194E984406EB810A06EB870B90F804171B
:1060A00090F8F876DAF80028DBF800380D9206EB65
:1060B000870006EB810C98F8F87698F80417DCF85E
:1060C00000280C9306EB870806EB810ED0F8003809
:1060D000DEF80068D8F800080F924FF400750E93B0
:1060E0001196109010E000BF4000012064F10008FC
:1060F000000000205C0201086CE00008D148026941
:1061000022F00401016130BFD4F87024D4F8743453
:106110009A42F3D00DF12600FBF7AEFC0028EDD03B
:10612000DDE90A6CBDF926307188BCF80200DDE9B2
:106130000C2B11FB03F747F38F39578810FB03F142
:1061400017FB03F041F38F3E40F38F3136F8040B19
:106150000A9610FB03F63CF8040BCDF82CC05F4602
:1061600046F38F3A10FB03F646F38F3832F8040BF0
:1061700037F8046B0C9210FB03F216FB03F0D4F813
:10618000C86E42F38F3C40F38F3212981E44C4F81D
:10619000C86E0AEB000613980596129609EB0006E6
:1061A00014980696139608EB000615980496149614
:1061B0000EEB00061698039615960CEB0006029659
:1061C000169617980D970144BBF80270019117912C
:1061D000189917FB03F01144DDE9107CD4F8C42EA4
:1061E000B7F802A0189103FB03F902EBA93640F3BC
:1061F0008F3BDDE90E201AFB03F8518832F804AB1F
:10620000C4F8C46E0E9211FB03F61AFB03F2418828
:1062100042F38F3A30F8042B0F9046F38F3911FB7D
:1062200003F612FB03F046F38F3E37F8042B10976A
:10623000664612FB03F736F8042B48F38F3140F320
:106240008F3847F38F3012FB03F747F38F32199FD4
:106250005F4419971A9F57441A971B9F4F441B97E7
:106260001C9F47441C971D9F77441D971E9F1196A6
:1062700007441F98BCF802601E97084420991F909D
:10628000114416FB03F3219A2091013D43F38F3B08
:106290005A44ADB22192002D7FF436AF6A4F94F884
:1062A000CCBE0825BD6194F8BA6EBBF1000F00F0BA
:1062B00083800598069D80FB001C85FB05798B0B70
:1062C000B80B049940EA894A039843EA8C4281FB5F
:1062D00001359F0B80FB003847EA85419D0B04EB9D
:1062E000461945EA884C52446144BBF1010FC9F894
:1062F000D02EC9F8D41E5FD0019981FB0105029907
:10630000830B43EA854081FB0153A90BDDE9182784
:1063100041EA834A5044C9F8D80E87FB0770BD0B89
:1063200082FB0227910B45EA804341EA87484344B8
:10633000BBF1020FC9F8DC3E3ED0DDE91A02DDE90F
:106340001CA582FB0237990B80FB000341EA8742C0
:10635000870B47EA834C85FB05588AFB0A03624496
:10636000A90B870BC9F8E02E47EA834A41EA884225
:106370005244BBF1030FC9F8E42E1DD0DDE91E2CF9
:106380008CFB0C138F0BDDE9200547EA834182FB70
:106390000223970B47EA8348414480FB000A85FBB0
:1063A000053CC9F8E81E9D0B810B41EA8A4245EA8B
:1063B0008C473A44C9F8EC2E94F8BB8E224801363B
:1063C0005FFA86F94FF40021C84584F8BA9E8161CE
:1063D0003FF601AE1C4B10229A61BBF1000F00F09A
:1063E000E780DFF86CE0B4F8D85FDFF868C09EF8AB
:1063F0001870D4F8D00FDCF804200297013503950B
:106400000026ACF5807ADEF83C5001960AEB47177F
:1064100002998946002900F0A9800C4B03EBC608BD
:10642000A7EB0809A9F12001490901314FF0000942
:1064300011F003014FEAC60A4B4649D0012933D077
:106440000AE000BF00ED00E000080240100F01204C
:106450000000002010100120022913D0644951F8D7
:106460000AA0D8F804105145ABBFA1EB0A01AAEB72
:1064700001014FF0010ACA460029C4BFD1460B46AC
:1064800008F12008D8E900A15145ABBFA1EB0A01F2
:10649000AAEB01014FF0010A4FF0000A9942C4BF74
:1064A000D1460B4608F12008D8E900A15145ABBF01
:1064B000A1EB0A01AAEB01014FF0010A4FF0000A1B
:1064C00008F120089942C4BFD1460B46B8454AD0CE
:1064D00041462BE0A3EB09034FF000095345D6BF1B
:1064E0005346CA46C246D1E90889C145ABBFA9EBAC
:1064F0000808A8EB09084FF001094FF0000998457A
:10650000DCBF9846D146D1E9103A9A45ABBFAAEB19
:106510000303A3EB0A034FF0010A4FF0000A6031B6
:106520004345CCBFD1464346B9421CD0D1E9008A8D
:10653000C245B5BFA8EB0A0AAAEB080A4FF000084B
:106540004FF001089A45D8BF9A4601F120010B6827
:10655000D8BFC846D1F804909945BBDBA9EB03032B
:106560004FF00109BAE7181842EBE372297849EABB
:10657000410303992B7031441FFA81F8490707D171
:106580001C4B0135E91AB1F5897F1ED20123019315
:106590000136B34507F108077FF43AAF019EA4F82E
:1065A000D88F0EB1CEF83C50C4F8D00FCCF80420F0
:1065B000114C4FF48015A56123B0BDE8F08F002386
:1065C0000E48079984F8C23E42E5B4F8AC76CEF89E
:1065D0003C500137A4F8D88FC4F8D00FCCF8042071
:1065E000A4F8AC7623B0BDE8F08F94F8CCBEF1E609
:1065F000100F0120F00901200008024054F90008A2
:10660000014BC3F8F8017047400001207BB972B913
:106610000029BEBF00204FF0004106E008BF00285F
:106620001CBF6FF000414FF0FF3000F057B8ADF1E4
:10663000080C6DE904CE002909DB002B1ADB02F0FF
:1066400079FEDDF804E0DDE9022304B07047404242
:1066500061EB4101002B1BDB02F06CFEDDF804E076
:10666000DDE9022304B0404261EB4101524263EB99
:1066700043037047524263EB430302F05BFEDDF8D5
:1066800004E0DDE9022304B0404261EB41017047C0
:10669000524263EB430302F04DFEDDF804E0DDE916
:1066A000022304B0524263EB4303704753B94AB923
:1066B000002908BF00281CBF4FF0FF314FF0FF300A
:1066C00000F00CB8ADF1080C6DE904CE02F032FE1A
:1066D000DDF804E0DDE9022304B07047704700BF35
:1066E000844641EA000313F003036DD1403A41D3DD
:1066F00051F8043B40F8043B51F8043B40F8043B9C
:1067000051F8043B40F8043B51F8043B40F8043B8B
:1067100051F8043B40F8043B51F8043B40F8043B7B
:1067200051F8043B40F8043B51F8043B40F8043B6B
:1067300051F8043B40F8043B51F8043B40F8043B5B
:1067400051F8043B40F8043B51F8043B40F8043B4B
:1067500051F8043B40F8043B51F8043B40F8043B3B
:1067600051F8043B40F8043B51F8043B40F8043B2B
:10677000403ABDD2303211D351F8043B40F8043BCB
:1067800051F8043B40F8043B51F8043B40F8043B0B
:1067900051F8043B40F8043B103AEDD20C3205D3DB
:1067A00051F8043B40F8043B043AF9D2043208D0D3
:1067B000D2071CBF11F8013B00F8013B01D30B8845
:1067C00003806046704700BF082A13D38B078DD023
:1067D00010F003038AD0C3F10403D21ADB071CBFF5
:1067E00011F8013B00F8013B80D331F8023B20F85F
:1067F000023B7BE7043AD9D3013A11F8013B00F898
:10680000013BF9D20B7803704B7843708B7883701F
:10681000604670470000000000000000000000001B
:106820000000000000000000000000000000000068
:106830000000000000000000000000000000000058
:1068400030B490F800F020F007016FF0000C10F069
:10685000070491F820F040F048804FF000046FF0FA
:106860000700D1E9002391F840F000F1080082FA16
:106870004CF2A4FA8CF283FA4CF3A2FA8CF34BBBE1
:10688000D1E9022382FA4CF200F10800A4FA8CF25A
:1068900083FA4CF3A2FA8CF3E3B9D1E9042382FA28
:1068A0004CF200F10800A4FA8CF283FA4CF3A2FA3D
:1068B0008CF37BB9D1E9062301F1200182FA4CF275
:1068C00000F10800A4FA8CF283FA4CF3A2FA8CF3DC
:1068D000002BC6D0002A04BF04301A4612BAB2FAFE
:1068E00082F200EBD20030BC7047D1E9002304F003
:1068F0000305C4F100004FEAC50514F0040F91F838
:1069000040F00CFA05F562EA05021CBF63EA0503D4
:1069100062464FF00004AAE72DE98048D1B072B674
:10692000CD4CDFF8488300250E95236B43F0010022
:106930002063216B01F001020E920E9B0D95266BD8
:1069400046F002072763236B03F002000D900D9BB6
:106950000C95216B41F004022263266B2C9506F006
:1069600004070C97BD4F0C9B2D952AA9384601268C
:106970002B962A96F9F772FD4FF48033BB614FF0E6
:10698000020ACDF8A8A0F9F769FD4FF40032BA6108
:106990004FF00409CDF8A890F9F760FD4FF480207E
:1069A000B8614FF4006340464FF0006B2A93F9F74B
:1069B00055FD3846C8F818B008222A92F9F74EFD5E
:1069C0004FF40023BB614FF400622A92F9F746FDB1
:1069D000C7F818B04FF0400BCDF8A8B0F9F73EFD5E
:1069E0004FF48003BB6180272A97F9F737FD4FF4F6
:1069F00000024FF4805C8261CDF8A8C0F9F72EFD4B
:106A00004FF0805383610B95206B40EA09022263AB
:106A1000236B2E9503EA09000B904FF480620B98CC
:106A20002A924046CDE92C562B96F9F717FDCDF862
:106A3000A8A0F9F713FDCDF8A890F9F70FFD0823EA
:106A40002A93F9F70BFD10222A92F9F707FD20236C
:106A5000DFF81C822A93F9F701FDCDF8A8B0F9F709
:106A6000FDFC2A974FF48077F9F7F8FC2A97F9F79D
:106A7000F5FC4FF400722A924FF40027F9F7EEFC70
:106A8000C8F84457C8F83C574FF400314FF08065C0
:106A90004FF480234FF48012856181614FF400151B
:106AA00083614FF4800187614FF4000382614FF0EE
:106AB00080774FF0007285618161836187618261B7
:106AC00098F86D574FF0804011211823C8F834070B
:106AD000C8F84017C8F83837002D00F040856049E5
:106AE000022588F86D57F9F71DFE5E48C8F860501A
:106AF00001214AF6C8764FF4FA7388F86D1786625A
:106B0000C362C16001600024072698F8A170C8F82C
:106B1000584000F55053C8E91C44C8F86440C8F810
:106B200078404FF482724FF400640820C8F87C600B
:106B30004FF40076C8F85C40C8F85030C8F85420CC
:106B4000C8F86C00C8F8686007F0FF04002F00F078
:106B500095854FF0020988F8A1901C6824F0400741
:106B60001F60D8E91556D8F85C00D8F86010D8F83E
:106B70006430D8F86C40D8F87070D8F8502035439D
:106B800005430D431D43D8F87860D8F868002543C5
:106B90003D4300F4007135430D431560B8F86A5069
:106BA000D8F87440D8F8502005F00403234353600C
:106BB000D7692D4C002127F400660120D661C8F862
:106BC000A41088F8A10098F8E520C8F8BC104FF48C
:106BD000E1350C23C8E92D11C8E93111C8E92B456D
:106BE000C8F8C03002F0FF07002A00F0FB8424261A
:106BF00088F8E560E26822F40050E0602769D8F880
:106C0000B83027F440561E432661D8E92F72E06859
:106C10001743D8F8C82020F41646174326F00C0373
:106C20000F431F43E7606169D8F8C40021F440773F
:106C300007436761D8F8C860B6F5004F00F091854A
:106C4000094B9C424FEA850500F0B48403F580624D
:106C5000944200F0AF840DE0003802400000024092
:106C600078070120000400400010014000080240A5
:106C700040000120FCF73EF88346FCF73BF84FF05C
:106C8000190909FB00F1B1FBF5F6FCF733F8824670
:106C9000FCF730F809FB00F7B7FBF5F7FCF72AF82B
:106CA000642109FB00FE09FB0BFBBEFBF5F209FBAF
:106CB0000AFCB2FBF1F3BCFBF5F901FB1377B9FB5E
:106CC000F1F001FB106630013A0132303232B0FB94
:106CD000F1F6B2FBF1F7BBFBF5F507F00F03B5FBDF
:106CE000F1F506F0F001194301EB0510A0602069F1
:106CF00020F4904525616769CA48C8F8FC0127F06F
:106D00002A066661E168002241F400532027E3600F
:106D1000C8F8E82088F8E57088F8E67098F83952E5
:106D2000C149C8F810225E244FF48046C8E9862283
:106D3000FE22C8F80842C8F81422C8F80C62C8F845
:106D40000462C8F8001205F0FF04002D01F0C680AF
:106D5000B64B0093242388F839320268B44D22F0F0
:106D600001010160FBF7C6FFD8F8FC61A5FB001428
:106D7000A70C7760D8F800328346AE48834201F210
:106D800091800137376240F6FC775C00BBFBF4F57D
:106D90003D4208BF0425F561D8E9863003433360DE
:106DA000D8E98261D8F8FC513143A960D8E984243C
:106DB0002243EA602F68A04A002047F00103202602
:106DC0002B60C8F83C0288F83962C8F82C0288F8B1
:106DD0003A02D8F84450994FC8F8047001214FF492
:106DE0008034C8F80C00C8F81400C8F81C00C8F8B3
:106DF0002400C8F83000C8F81000C8F83400C8F8FB
:106E00001810C8F82C20C8F80840002D01F0218087
:106E1000D8F84440E20640F19587002501241D95ED
:106E200088F840403A69009922F0E0633B61386994
:106E300041F8584C40F000723A617B6B23F01F0020
:106E400078637A6B082632437A637D4F88F8405026
:106E5000022541F85C6C41F8545CBE614FF4006659
:106E6000BE61802140264FF48053BE61B961BB6191
:106E700098F83902202800F09A84724C00222046AB
:106E80000121FF2488F87F2688F87C46FAF74EFE19
:106E9000A8F87D066A4E4FF480014FF00060B161A2
:106EA000B061FBF7B5FD72B6674D684B6B6062B6BB
:106EB0004FF4803700244FF400314FF48022B76143
:106EC00088F8824688F86244B161B261B761B16105
:106ED000B26172B6C8F85842C8F85C4262B672B67F
:106EE000C8F87044C8F8744462B6FCF74DFA4FF025
:106EF00080554FF400204FF40003B061B361B561D9
:106F0000009E16F84C7C3FBB0099514CC8F80047D6
:106F10004FF0010B052201F84CBCC8F804273B4692
:106F2000D8F8000740F82730013798F80457FEB228
:106F3000B542F5D8474FC8F8087905240023C8F8AA
:106F40000C491A46D8F8081941F82320013398F85B
:106F50000CE9D8B28645F5D83F4DC8F8085705F179
:106F60009806C8F80C6705F5987705F5E47405F5FB
:106F7000187305F53E7205F5647105F5856005F534
:106F8000986605F5AB65C8F81077C8F82C570A273E
:106F9000009DC8F81447C8F81837C8F81C27C8F867
:106FA0002017C8F82407C8F8286788F830772B4CD2
:106FB0002B4B2C4A2C492D482D4E2E4FC5F8A84559
:106FC000C5F8B435C5F8B825C5F8BC15C5F8C00571
:106FD000C5F8C465C5F8C875274C284B284A294907
:106FE00029482A4E2A4FC5F8CC45C5F8F835C5F8CA
:106FF000FC25C5F80016C5F80406C5F80866C5F8EE
:107000000C76244C244B254A25492648264E274FEA
:10701000C5F81046C5F81436C5F81826C5F81C166C
:1070200046E000BF00540040801A060038110120DD
:1070300083DE1B43A08601000100000F00200140F9
:1070400000000240BF0601200000002015190008C2
:10705000E41A0120F81A0120F0100120151B000885
:10706000191B0008E53B0008AD1C0008B51C000812
:10707000CD1C0008D51C0008ED1C0008511D00089F
:10708000911D0008613B0008F91D0008E53A000861
:10709000253B0008A91E0008211F0008591F0008F1
:1070A0009D1F0008C5320008B51F000835200008E4
:1070B000C5F82006C5F82866864CC5F82C76864BA0
:1070C000864A87498748884E884FC5F84846C5F89C
:1070D0006C36C5F87026C5F87416C5F87806C5F87C
:1070E0008866C5F88C76824C824B834A83498448F3
:1070F000844E854FC5F8A846C5F8AC36C5F8B0260D
:10710000C5F8B416C5F8B806C5F8BC66C5F8A877C2
:107110007E4C7F4B7F4A80498048814E814FC5F825
:10712000B447C5F8B837C5F8BC27C5F8C017C5F8C7
:10713000C407C5F8C867C5F8CC777B4C7B4B7C4A45
:107140007C497D487D4E7E4FC5F8F847C5F8FC3731
:10715000C5F80028C5F80418C5F80808C5F80C6873
:10716000C5F81078774C784B784A794979487A4E47
:107170007A4FC5F81448C5F81838C5F81C28C5F862
:107180002018774CC5F82808764B774A7749784815
:10719000C5F82C68C5F84878764E774FC5F86C4826
:1071A000C5F87038754C764BC5F87428C5F8781852
:1071B000744A7549C5F88808C5F88C687348744ED8
:1071C000C5F8A878734FC5F8AC48C5F8B038C5F80D
:1071D000B428C5F8B818C5F8BC08C5F8A869C8F837
:1071E000F87162B66C4CDFF8B8B16C4E4FF0010A22
:1071F000802388F863A40022A36188F85422FCF756
:107200007FF8FCF7C1F888F8AAA0AA469AF8D459E2
:10721000002D00F07285012D00F0D883022D01F0C1
:10722000BD8098F88516002900F02B83D8F8884691
:10723000D8F87826B8F88C56131B9FB2AF42C0F02E
:107240002083781B2C44B8F88E562918B1F5004FCE
:10725000A4EB050488BF24184FF098024FF00001FA
:107260002AA888BFA8F88C7602F0C2F9052798F8FA
:107270008426B8F88C968DF8AD70A023D8F80070ED
:10728000ADF8AF508DF8AE20ADF8B1908DF8AA30C2
:1072900005E0D8F80020D31B642B00F2D6820B2126
:1072A0002AA8F9F781FC0028F3D0C4F30E04002DBE
:1072B00000F0D9820027BD4200F286803B46D8B25A
:1072C000D8F800208DF8AD000630A946C1B2254699
:1072D00014466DE09D200008ED34000821360008BA
:1072E000D93A000809380008E1200008E520000824
:1072F00035210008154200083D21000839420008E8
:107300001D2200084D420008B93B0008313E00082C
:107310001D1B00089D1C0008B11C0008C91C0008AA
:10732000D91C0008DD1C0008291D0008811D00086B
:10733000B11D0008D11D0008511E0008611E000883
:10734000951E0008C91E0008153F0008791F000897
:10735000A11F0008312000085D20000875200008EA
:10736000D1200008D5200008D9200008DD20000821
:10737000C5230008453F0008E9200008392100081E
:107380004121000819220008212200088D2200084E
:10739000CD420008112800080000024000ED00E086
:1073A00030220120D8F80020131B642B00F29784B0
:1073B0002AA80091F9F7F8FB00990028F2D0B94506
:1073C0002C464D4640F24F822AA800230090A74940
:1073D000009A31F81400D0710134023314F4004FD4
:1073E0009BB24FEA1021A4B207F1010718BF002495
:1073F000802B9171BFB203F102013FF460AF04F141
:107400000109BD4207F1010E1FFA89FC02F10200D9
:107410003FF455AF954B1A4633F81430C37119F445
:10742000004F1FFA8EF74FEA132383710CBF644697
:1074300000248BB2BD4203F1020100F1020007F10A
:1074400001093FF43CAF32F814E080F807E0013462
:1074500014F4004F4FEA1E2C1FFA89F7A4B280F8EB
:1074600006C018BF002400988BB204F10109BD4288
:1074700003F1020107F1010E1FFA89FC00F1060079
:107480003FF41DAF32F81430C37119F4004F4FEAC6
:10749000132308BF64461FFA8EF7837118BF0024B8
:1074A0008BB2009904F10109BD4203F1020007F11A
:1074B000010E1FFA89FC01F108013FF400AF32F818
:1074C0001430CB7119F4004F4FEA132308BF644600
:1074D0001FFA8EF78B7118BF0024009983B204F154
:1074E0000109BD4203F1020007F1010E1FFA89FCF8
:1074F00001F10A013FF4E3AE32F8143001921A0AA6
:1075000019F4004F8A71009ACB7108BF64461FFAC4
:107510008EF718BF002483B204F1010902F10C01B7
:10752000BD4202F10E0203F1020007F1010E1FFA43
:1075300089FC00923FF4C3AE4C4F37F81430CB7146
:1075400019F4004F1FFA8EF74FEA13220CBF64465E
:107550000024BD428A7183B27FF439AFAFE605F0F3
:10756000FF07109788F86C77206C30432064226CFA
:107570003240109231463A461C20109BF8F752FEDA
:1075800032463B4E4FF0805535600F97216C41EAF3
:107590000A032364246C04EA0A070F971D200921BB
:1075A0000F9BF8F73FFE4FF00052D8F834073260D7
:1075B000FFF795BAFBF7B8FB8346FBF7B5FB4FF037
:1075C000190909FB00F0B0FBF5F6FBF7ADFB8246AD
:1075D000FBF7AAFB09FB00F3B3FBF5F7FBF7A4FBF2
:1075E000FFF75EBB234E189788F8E470326B0243B6
:1075F0003263346B04401894189A1797356B05431F
:107600003563336B03401793179A1697716C41F0EB
:1076100010027264766C06F01004CDE92C7016949A
:107620001548169B2AA907254FF4007B2E95CDE916
:107630002AB94FF0120AF8F711FF4FF48062CDE932
:107640002A2AF8F70BFF3A4603212520F8F7EAFD2E
:107650000748D8F8AC4020274760E368D8F8B41052
:10766000D8F8B0503B43E360FFF7C1BA40000020B8
:1076700000E100E0003802400000024003F5003E57
:10768000159488F8A040DEF830302B43CEF8303027
:1076900007F1804ADEF830702F401597159A149440
:1076A000DEF830202A43CEF83020DEF830302B4090
:1076B0001493149A1394DEF830702F43CEF8307080
:1076C000DEF830202A401392139A1294DEF83030FC
:1076D0002B43CEF83030DEF830702F401297129ADC
:1076E0001194DEF8402042F48043CEF84030DEF8BA
:1076F00040702A9607F480420AF501301192119BDE
:107700002B91CDE92C412AA9F8F7A8FE86614FF408
:1077100080662A964FF48057F8F7A0FE86612A9774
:10772000F8F79CFE052387612B954FF400552E93A7
:107730002A954FF48046F8F791FE4FF400422A92C2
:10774000F8F78CFE2A96F8F789FE21462420224677
:10775000F8F768FD9548D8F8503010214160FFF7E0
:10776000F8B906F1804A0AF5104C64454FEA45061F
:1077700000F05F850CF58062944200F05A85FBF7BB
:10778000B9FA8346FBF7B6FA4FF0190909FB00F77F
:10779000FBF7B0FAB7FBF6F78246FBF7ABFA09FB4B
:1077A00000F5B5FBF6F5FBF7A5FA00F058BDD8F8E3
:1077B000007098F83922202A7FF45FAB21467C487C
:1077C0003B461922FAF700FA014600287FF455AB30
:1077D00098F83852012D3FF450ABD8F8FC2188F8C6
:1077E00038421368734823F400651560D8F8FC210B
:1077F0004FF0220A88F839A288F83A62C8F83C1299
:10780000C8F82802166846F480601060D8F8FC5169
:107810002A6842F480763B462E6022464FF00110E3
:10782000FAF7D2F9002841F0AF84D8F8FC11624889
:10783000A0230B613A462146FBF75EF8002801F0D1
:107840008584D8F83C3201F09FBC5C4E08244FF48C
:107850000065402080214FF48057B461B561B0616C
:10786000B161B761FEE7564D564F2C69E31B00210D
:107870005810C8F8780688F88516C8F8881688F869
:10788000841698F80D29002A3ED098F80F4998F8E8
:107890000C59D8F80819631CD8B202F1FF3E854292
:1078A00098BF002088F80DE988F80F0951F82440A6
:1078B00094F805C0D4F88670A444CCF80670B4F8E7
:1078C0008A20D8F80050ACF80A2005E0D8F800204B
:1078D000531B642B00F27F8463790C332046D9B2AA
:1078E000F9F762F90028F1D098F83057092D06D839
:1078F00008EB85090135C9F8084788F8305798F82A
:107900000D49002C00F0D58498F81059002D40F056
:10791000708498F80527002A3FF478AC98F8077728
:1079200098F80447D8F800177B1CD8B2844298BF57
:10793000002002F1FF3C88F805C788F8070751F8D6
:10794000277097F90220B878002AC0F2C28429462D
:1079500095220DF1AB0001F04BFEFF2598F87F4614
:107960008DF8AA508DF8A84097F801908DF8A9904D
:107970003B79D8F800508DF8AC3005E0D8F80040DD
:10798000631B642B01F2898406212AA8F9F70CF9FC
:107990000028F3D098F87F0638703846FDF7B6FC1B
:1079A000094980228A6101F05CBC00BF00E100E06F
:1079B000020010000000FFFF020001000000024072
:1079C000000000204000002000080240D74D6F69F1
:1079D000EC7F2B8E0594002FBCBF07F57F573F37F8
:1079E000BA13049303924FF00009D8F87014D8F832
:1079F000740481423FF415AC2AA8FAF73DF8002838
:107A00003FF40FAC98F8803ED8F86C54BBF8E440D3
:107A1000009563B103F1FF3E0EEB8E0708EB870C78
:107A2000DCF8E42BA91AB1F5806F00F27881D8F860
:107A3000887EBF483D46BA1CC8F8882E35F804EB4E
:107A4000C8F8885E7F88BDF9A82000EB041117FBF9
:107A500002F51EFB02FC45F38F3EB1F90250A1F87E
:107A600002E02701AEEB050EB14D4CF38F3035F936
:107A700007C0E853A0EB0C05D8F8980ED8F88C7E18
:107A8000B1F904C02844D8F89C5EC8F8980E0EEBF3
:107A90000500C8F89C0EBD1C3846C8F88C5E30F84E
:107AA00004EBC8F88C0E7F881EFB02F017FB02F572
:107AB00040F38F37B1F906008F8045F38F35CD80C5
:107AC0002D1AD8F8A00EA7EB0C0E7044C8F8A00E23
:107AD000D8F8A40ED8F8907E0544C8F8A45E3846BD
:107AE000BD1CC8F8905E30F804CBC8F8900E7F88B3
:107AF0001CFB02F017FB02FEB1F908C0069340F32D
:107B00008F37B1F90A000F814EF38F354D812D1A51
:107B1000D8F8A80EA7EB0C0E7044C8F8A80ED8F839
:107B2000AC0ED8F8947E0544C8F8AC5E3846BD1C4F
:107B3000C8F8945E30F804CBC8F8940E7F881CFB1C
:107B400002FE17FB02F04EF38F3540F38F3E82FBAF
:107B50000220920B42EA80420AEB8407B1F90C0042
:107B60008D812D1AB1F90E00A1F80EE0D7F8D819C1
:107B7000C7F8D829571AD8F8B02E1544C8F8B05EFF
:107B8000D8F8B45EAEEB00002844C8F8B40EDBF8B9
:107B9000E000074407F58071CBF8E0705F1C0291AC
:107BA0009C46019719460CE0D7F8E01B0131C7F855
:107BB000E01B019F0CF101051FFA85FCBC456146E5
:107BC00051DC0CF0010308EB031E01EB8102DEF82F
:107BD000985EDEF89C3EDEF8A00E08EB8207DEF829
:107BE000A42E85FB055EAD0B45EA8E4583FB033E67
:107BF0009B0B43EA8E4E754482FB022E930B43EAA5
:107C00008E4380FB000E820B42EA8E4003441D44EB
:107C1000029B95FBF3F0D7F8D85BA8425FFA8CF390
:107C20004FEA8102C0DD15B9009DC7F8E85B0A4440
:107C300008EB82070199C7F8D80B0133DBB2009833
:107C4000C7F8E40B994287F8DC9BC7F8E09BB0DBF0
:107C500003EB830E013308EB8E02DBB28B42C2F8DA
:107C6000D89BF5DDA5E7069B039D03EB830008EB9E
:107C7000800EDEF8D82B954240F30E820134C4F317
:107C80000804ABF8E440002C7FF4AFAE294898F824
:107C9000847E98F885CE284D0744844497F81037A1
:107CA00097F812279CF814079CF816C705EB830178
:107CB00005EB820E05EB8C0305EB8002D1F8004842
:107CC000DEF80078D2F80058D3F80018C8F8884ECB
:107CD000C8F88C7EC8F8905EC8F8941E85E6174EEA
:107CE00008274FF40064402080214FF48055B7618D
:107CF000B461B061B161B561FEE74FF4006229463D
:107D00000F4801F075FC2846CBF8E050FDF77CFAEF
:107D100001208AF8D409FBF737FBFFF782BA204627
:107D2000FDF772FA98F8803E81E600BF000000205F
:107D3000542401205C0201086CE0000800000240AD
:107D4000101B0120D8F84430CB4DD8F8084023F45C
:107D5000885020F0020646F00202C8F84420696804
:107D600021F440336B606868204368607E6826F4C5
:107D700080727A607D68D8F8144045EA0421796001
:107D80007B6823F0407078607E68D8F80C20BB4890
:107D900016437E60BD6825F40064BC60BB68D8F8FB
:107DA00010100B43BB60BA68D8F82C6022F07065E5
:107DB000BD608642BC6800F0D782D8F82C100C4316
:107DC000BC60B86820F04056BE60BA68D8F8305041
:107DD0002A43BA60BC6824F00203BB60B868D8F8D4
:107DE0001C1040EA4106BE60D8F82420002A40F06A
:107DF000A5827D6825F400647C60FE6AD8F8204086
:107E000026F47002FA62FD6A631E45EA0350F862C6
:107E1000B96821F40076BE60BA68D8F8345042EAF6
:107E20004524BC60BB6823F48060B860BE68D8F8A5
:107E30001810002546EA8122BA60C8F84850D8F8E0
:107E4000444024F0030343F00100C8F84400FEF767
:107E5000E4BF07F58C3CC8F8485088F840501E95A0
:107E6000DCF8443043F48070CCF84400DCF8446023
:107E700083482A9106F480721E9203272D912AA925
:107E80001E9B2B972C95F8F7E9FA2A460921122018
:107E9000F8F7C8F97B494FF480250D60D8F80470D5
:107EA000FEF7B6BF4FF49672D8F8041202FB07F73C
:107EB0004FF47A7EB7FBFEF501353562002940F0BC
:107EC000CE8003EB4300BBFBF0F1C1F30B02002AB1
:107ED00000F0CF8041F40045FEF75DBF00F5F23CB5
:107EE0001C9488F83842DCF8300040F00202CCF8EC
:107EF0003020DCF8305005F002061C961C9A1B94CA
:107F0000DCF8301041F00203CCF83030DCF83000FF
:107F100000F002021B921B9A1A94DCF8405045F4C0
:107F20000016CCF84060DCF8401001F400131A93FE
:107F30001A9A1994DCF8300040F40012CCF8302082
:107F4000DCF830504E482C9405F400161221199696
:107F5000402501262B914FF0040B2AA9CDE92D6B6A
:107F6000199B2A95F8F77AFA80232A93F8F776FA7C
:107F7000C8F8E45F444D454AC8F8E84FA5F124002D
:107F80004FF000714FF480634FF0030A4FF4000983
:107F90004FF4001BC5E901A9C8F8F04FC8F8F44F29
:107FA000C8F8F84FC8F8FC4F2C60C8F8DC2FC8F8A8
:107FB000E01FC8F8EC3FC5F80CB0FAF76BFD344A87
:107FC000C8F830024FF4806311464FF0007042F859
:107FD000AC3C42E9249B42E92D4442E92A4442F860
:107FE000B80C42F894ACA2F1BC00924642F8A04C06
:107FF00042F8984C0092274A41F8BC2CA5F6046937
:108000004FF400314AF89C1CC5F81490FAF742FD71
:108010003246C8F8340202212F204AF8849CF8F72F
:1080200001F92246174C4FF40040606002210B20FA
:10803000F8F7F8F838464FF4006732460221276017
:10804000F8F7F0F8022266601F2011464FF0004654
:10805000F8F7E8F82660D8F8FC01FEF77BBE192493
:1080600004FB03F3BBFBF3F7C7F30B03002B40F058
:1080700061810125FEF78FBE002301400100000F42
:108080000004024000E100E040100120B86002401E
:108090003811012010600240DEF8E02B0498B4494A
:1080A000B44FC8F800188242C8F8F8770BD2002BFA
:1080B0003FF4E4ADD8F8E42B009D5902AA1A8031B0
:1080C0008A427FF6DBAD13F0010CAB4FAB4914BF16
:1080D00004224FF4802208EB0C0EBA619EF8845EF5
:1080E0000135EAB201EB8C00022AD0F8F87708BF1C
:1080F00000228EF8842EB85C01EB800E0134DEF88D
:10810000001808EBCC00C4F308053A4401EB8507DE
:10811000C0F8887E9278994901EB820E984ADEF881
:108120000078984907EB8505C0F88C5E02EBCC0718
:108130000FFA8CF001EBCC05C7E90099C7E9049967
:10814000C7E90899C7E90C99C7E91099C7E91499D3
:10815000C7E91899C7E91C998037BD42ECD18A4F0D
:1081600007EB001C00011F2B47F80090CCE9019998
:10817000CCF80C9006D808EB4303B3F8B0260132D4
:10818000A3F8B0269DF80430059D88F8803E1421A0
:1081900001FB038EAB42CEF8E09BFFF470AD0021F3
:1081A000D8F8E42B794C8E4602E0E568AF1ABE445D
:1081B0000131CFB2BB4204F11404F6D8BEFBF3F98F
:1081C000013302EB03244C440220CBF8E8408AF848
:1081D000D409FFF726B86E4E08274FF400644020FC
:1081E00080214FF48055B761B461B061B161B56170
:1081F000FEE7D8F89436002188F810198BB1D8F82A
:108200005072D8F85052E81B98420AD2614C226949
:1082100022F00401216130BFD8F85052E81B83429C
:10822000F5D85D48FDF772F8534B80279F61FEF744
:10823000EDBFFAF779FD8346FAF776FD4FF019099D
:1082400009FB00F1B1FBF6F7FAF76EFD8246FAF78B
:108250006BFD09FB00F3B3FBF6F5FAF765FD64214E
:1082600009FB0AFE09FB00F0BEFBF6F209FB0BFC62
:10827000B2FBF1F3B0FBF6FB01FB1377BBFBF1F9AB
:1082800001FB1955E800FA0032303232B0FBF1F54B
:10829000B2FBF1F705F0070A7B0003F4F87EBCFBA4
:1082A000F6F6B6FBF1F60AEB06117144A160FEF793
:1082B0001EBD98F8800601287FF426AB04F1804E9D
:1082C0000EF502314FF0006788F881468F61FFF7A5
:1082D0001BBB80F0800E0AEB8E09D9F8A845002C54
:1082E00000F0BD873846A047002800F0E487294603
:1082F00098222AA801F07CF9BD78D9F8A8378DF822
:10830000AA500DF1AE009847D8F800408DF8AD00A6
:1083100005E0D8F800100B1B642B00F2B0879DF825
:10832000AD2006322AA8D1B2F8F73EFC0028F0D0E2
:1083300000F097BF47F44045FEF72DBD7B6843F43E
:1083400000607860796821F460467E604FF4604296
:1083500092FAA2F5D8F828307968B5FA85F4581E53
:10836000A0400843786048E524F04053BB6031E505
:10837000DB1B0400B9A20100000802406CE0000809
:108380005424012054440120D80E0120180C01204F
:108390000000024000ED00E054090120D8F87014FC
:1083A000D8F87404814202D02AA8F9F765FBDBF8FB
:1083B000E870D8F86C44A7427EF433AFB8F89A3628
:1083C00098F88456874901334FF0000C4FF40002AF
:1083D000022DA8F89A368AF8D4C98A6100F0E98299
:1083E000814B8048DD7F9A7F804C0135571B4FF0D1
:1083F00002017D4D81616969219448BF03370029DD
:10840000B8BF01F57F514FEAA703B8BF3F31DAB2D9
:108410008813FF2A059000F0D980754B754FCDF871
:1084200010A04FF00009964601254FF0000A21AC3C
:108430000295CDF8189003945546F146CDE9237383
:108440000027CDE92A77CDE92C77CBF8E0704FF4FF
:10845000007404E0316921F00400306130BFD8F8C5
:108460007014D8F8743499420DF12A00F2D0F9F75B
:1084700003FB0028EED02398BDF92A302A9ADDF8B4
:1084800090C00746013C37F804EB23971EFB03F12D
:1084900041F38F318A182A924088009210FB03FE24
:1084A0002B9A4EF38F3160468A182B9230F804EBEA
:1084B0002C9901921EFB03F242F38F320A442C9254
:1084C000BCF802E0249083FB031C2D981EFB03F3F1
:1084D0008F0BDBF8E01047EA8C4E43F38F33714487
:1084E0000344A4B2CBF8E0102D93002CB7D18C46F6
:1084F0000CF5807E82FB022CDDE90010970B47EA29
:108500008C4783FB033C9A0B42EA8C4381FB01219D
:108510001F44930B80FB002043EA814C910B41EAFE
:108520008043029A05989C44674497FBFEF7B84243
:10853000C8BF00220292BAF1000F1CD14FF0010A0D
:1085400003990DF187048C4220D00C462A4914F877
:10855000012F039401EB820EDEF8F807471910F89B
:1085600005C0BC7801EB8C0301EB8402D3F80078E2
:10857000D2F8003862E70135EDB2012D22D9039916
:108580002546A2460DF187048C42DED1029DDDF81E
:1085900018A0CE46002D35D1F2450AF1010913D0BD
:1085A000154F9DF884C007EB8C03D3F8F82710789B
:1085B000947807EB800A07EB8401DAF80078D1F8A9
:1085C000003831E7A246BBE7DDF810A0054F0B4AA3
:1085D0000B48C8F800284FF40033C8F8F807BB610F
:1085E000FEF71FBE0008024000000020010000014D
:1085F00064D0000864B000086CE00008DB1B0400D5
:10860000B9A20100B8F89C56D1465FFA89F201354B
:10861000062ADDF810A0A8F89C5606D808EB490EEB
:10862000BEF8F0060130AEF8F006D8F85042D8F89F
:108630007014D8F87474484A2744484C7B1A4FF495
:108640000035CBF8EC30A5619146906B0021982263
:1086500000F0CEFF4FF489720021414800F0C8FFBE
:108660003F49C9F83C104FF400274FF480134FF4F2
:1086700000154FF480024FF40001A761A361A561CA
:108680000423A261A1610222364999F81800D8F8A2
:108690006C7488F8CC3E002488F8C22E0023002297
:1086A0004FF0FF090325A8F8D84FC8F8C44EC8F802
:1086B000C84EC8F8BC4E88F8C14EC1E90023CBF8BB
:1086C000F07088F8BB0E88F8C09E88F8C35EFDF78E
:1086D00071FC1B24013CA7B2FDF76CFCFDF76AFCA2
:1086E000781E1FFA80F9FDF765FC09F1FF339DB292
:1086F000FDF760FC6A1E94B2FDF75CFC611E8FB250
:10870000FDF758FC781E1FFA80F9FDF753FC09F1BC
:10871000FF339DB2FDF74EFC6A1E94B2FDF74AFC92
:10872000611E8CB2002CD5D10C4F0D49202008229F
:10873000B861A6460792CDE90044CDE90344A446BA
:1087400027462546204602940694089480220594E4
:10875000CDF824A093E000BF0000002000080240F4
:10876000F009012010100120069A4B784FEA420AC6
:10877000039AC3F3801949EA42039AB291F901308E
:1087800003924AEAD37293B2069301312022049BEA
:1087900091F800A05B0012EA0A0F18BF43F0010332
:1087A0009BB25208049340F09880029A4B784FEAAB
:1087B0004209019AC3F3801A4AEA42039AB291F934
:1087C0000130019249EAD37293B20293013120221F
:1087D000009B91F800905B0012EA090F18BF43F06C
:1087E00001039BB25FEA520A009340F09A8091F82D
:1087F000019091F901204000C9F3801A40EAD27338
:108800004AEA440498B2A4B2013120230A786D00E8
:10881000134218BF45F001055B08ADB240F09C80E3
:108820004B7891F901A07F00C3F3801949EA4C0C01
:1088300047EADA721FFA8CFC97B2013120234FEA23
:108840004E0291F800E013EA0E0F18BF42F0010249
:108850005FEA530A1FFA82FE40F09B80059B91F964
:1088600001905B0043EAD97293B205930131402233
:10887000079B013B13F0FF03079300F02381089B44
:1088800091F800905B0019EA020F18BF43F0010352
:108890009BB2089353083FF467AF13EA090F069B96
:1088A0004FEA430318BF43F001039BB206939308BA
:1088B00040F08C80039A4B784FEA420A049AC3F343
:1088C000801949EA42039AB291F9013004924AEAC6
:1088D000D37293B2039301312022029B91F800904E
:1088E0005B0012EA090F18BF43F001039BB2520864
:1088F000029340F08D80019B91F801A04FEA43095B
:10890000009BCAF3801242EA430A91F901301FFA30
:108910008AF2009249EAD37293B2019301314FF087
:10892000200A0A7840001AEA020F18BF40F001003E
:108930005FEA5A0380B240F08A8091F8019091F981
:1089400001206400C9F3801A44EAD2734AEA45055B
:108950009CB2ADB2013120230A787F00134218BFC8
:1089600047F001075B08BFB240F08A804FEA4C0332
:1089700091F801C091F901A0CCF3801943EADA72B1
:1089800049EA4E0E1FFA8EFE1FFA82FC01314FF0AB
:10899000200A059B5A000B781AEA030F18BF42F011
:1089A000010292B205925FEA5A0204BF01318022AD
:1089B0005EE798F8850600287FF412ADD8F878763F
:1089C000C8F88876012488F8854609E513EA090F76
:1089D000039B4FEA430318BF43F001039BB2D20845
:1089E00003937FF4D4AE049B91F801904FEA430ABD
:1089F000029BC9F3801242EA430991F901301FFA40
:108A000089F202924AEAD37293B20493013120228E
:108A1000019B91F800A05B0012EA0A0F18BF43F017
:108A200001039BB2520801937FF4D2AE009B91F9EF
:108A3000012091F801905B0043EAD273C9F3801AD8
:108A40009AB24AEA400080B20092013120230A78AB
:108A50006400134218BF44F001045B08A4B27FF421
:108A6000D5AE91F8019091F901206D00C9F3801AFB
:108A700045EAD2734AEA47079DB2BFB201312023CB
:108A80004FEA4C0291F800C013EA0C0F18BF42F0F5
:108A900001025B081FFA82FC7FF4D1AE91F80190CD
:108AA000059AC9F3801A4AEA42039AB291F9013051
:108AB00005924FEA4E0E4EEAD3721FFA82FE013142
:108AC0002022D5E60599039AADF89A000098069BF6
:108AD000ADF8A610ADF8A070ADF89E50049F029DB1
:108AE000ADF89C40ADF89800019C0898ADF8902036
:108AF0002AA90DF12A02ADF89640ADF89270DDF882
:108B000024A0974CADF8A4E0ADF8A2C0ADF8945005
:108B1000ADF88E30ADF88C000DF18E07F9F73CFD05
:108B2000002800F00481BDF82A5095B18D49B8F8AD
:108B3000A2C68A6B92F888905CFA85FEA944A8F8D0
:108B4000A2E682F88890636983F0400040F48005D3
:108B5000A5610DF1AA05BDF88E000DF12A02294686
:108B60000237F9F719FD002800F0E180BDF82A204E
:108B700092B17C49B8F8A2C6886B90F888905CFAEC
:108B800082FE9144A8F8A2E680F88890636983F099
:108B9000400242F48001A161023537F8020B0DF169
:108BA0002A022946F9F7F8FC002800F0C080BDF839
:108BB0002A0090B16B4BB8F8A2169A6B92F888E035
:108BC00051FA80FC8644A8F8A2C682F888E0606961
:108BD00080F0400949F48003A361023538880DF123
:108BE0002A022946F9F7D8FC002800F0A080BDF839
:108BF0002A2092B15B49B8F8A2C6886B90F8889099
:108C00005CFA82FE9144A8F8A2E680F88890636935
:108C100083F0400242F48001A16178880DF12A02BC
:108C2000A91CF9F7B9FC002800F08180BDF82A00E2
:108C300090B14C4BB8F8A2169A6B92F888E051FAB2
:108C400080FC8644A8F8A2C682F888E0606980F0BB
:108C5000400949F48003A361B8880DF12A02291D57
:108C60000637F9F799FC002861D0BDF82A2092B1A7
:108C70003C49B8F8A2C6886B90F888905CFA82FEEE
:108C80009144A8F8A2E680F88890636983F04002D6
:108C900042F48001A1612AA8B84205F106057FF4DB
:108CA0007CAF002321930DF1A604CDF88730184640
:108CB0000DF1840C04E08BB20435A8B238284BD0F7
:108CC0006588A71CC5F3C00444EA4303C5F3800EBE
:108CD0004EEA4309C5F3400242EA490105F00105A5
:108CE000430745EA4104B3F1004F0FFA84FE2ED04A
:108CF0001FFA8EF97A88BC1CC2F3C00747EA490301
:108D0000C2F38001043041EA4303C2F3400E85B24E
:108D10004EEA4309400702F0010242EA4907B0F176
:108D2000004F39B2C7D10CF8011B0023C4E7B8F8D3
:108D3000A4060B4A0130A8F8A406536983F0800703
:108D400047F400049461064902258D613EE40CF865
:108D500001EB4FF00009CDE707990DF1830C09E015
:108D600000080240000000200DF18A056700AC45B4
:108D7000F9B246D01CF8014F4C4062B2002ABABF8B
:108D8000540084F097046400E7B279B20029BABFB6
:108D90004F0087F097077F00FBB25DB2002DBABF8E
:108DA0006B0083F097035B00D8B244B2002CBABFCB
:108DB000600080F097004000C2B257B2002FBABFE7
:108DC0007A0082F097025200D3B259B20029BABF9A
:108DD0004B0083F097035B00DDB268B20028BABF96
:108DE000450085F097056D00ECB262B2002ABBDA4F
:108DF00053000DF18A0583F0970EAC455FFA8EF1B2
:108E0000B8D1079129B1B8F8A0560135A8F8A056F5
:108E100099E7CA48CA4A846B219FBDF88830A3806D
:108E20004FF40015276095616179002900F07D817C
:108E30000C298CBF022201221144C800BF4C626B76
:108E400092F8009057784844431E93FBF9F517FBBE
:108E500005F1703188B2B0F5096F3FF674AF98F83C
:108E6000CC2E8418671E97FBF2FCACF11C039CB25D
:108E7000002C41D0651E05F007070125FDF79AF883
:108E8000A54239D239B21FB301291BD0022916D00D
:108E9000032911D004290CD0052907D0062902D0B6
:108EA000FDF788F80225FDF785F80135FDF782F812
:108EB0000135FDF77FF80135FDF77CF80135FDF749
:108EC00079F801350135FDF775F8A8B2A04213D243
:108ED0000835FDF76FF8FDF76DF8FDF76BF8FDF756
:108EE00069F8FDF767F8FDF765F8FDF763F8FDF73A
:108EF00061F8AAB2A242EBD3FBF7DAFA00283FF4FA
:108F000022AFD8F86C44DBF8F03098F8CC5ED8F893
:108F1000C81E8A4FD8F8C40EE21A2B46F9F7B8F9E2
:108F2000BC6BB8F8D89F874984F8860000234A466E
:108F3000D1E90001FDF76AFB00290A4607460B4606
:108F4000C0F2F780B0F1004F72F100024FF0010E55
:108F50000DDBB80840EA8377B7F1004F4FEAA3036F
:108F60004FEA4E0173F100025FFA81FEF1DA9A03D3
:108F700042EA9740BF03009700234FF08041009AD8
:108F80009B0843EA81739A424FEAA10170EB010208
:108F9000F5DB53EA010227D0CDE902541A4600233B
:108FA0001F4694080194009CD51841EB070CAC4275
:108FB00070EB0C040ADB009C651B60EB0C00921844
:108FC00041EB0104D318009544EB0707019A5D08B3
:108FD00042EA8172891045EAC77352EA01054FEAF5
:108FE0006707DED1DDE902548EFB03ECA5FB0E2002
:108FF000C82705FB0C01A2FB073E6FF4FF7007FBBF
:1090000001E2834272F1FF31C0F29180002A04DA5A
:1090100040F2FF115B1842F100025F0A47EAC25CAE
:109020001CF500504FEA622141F1000E830B43EA28
:109030008E42424F98F8BBEEB87FD8F8BC3EFF2A6C
:1090400028BFFF2284F88720DBF8EC20C4F88C20AE
:109050000430A2EB40210EFB09F705FB03F3B3FB41
:10906000F7F0637998F8C19EC4F8901098F8C01E84
:1090700084F8890084F88A1084F88B903BB10C2B1B
:109080008CBF4FF002094FF001094B44DB002B4F1E
:10909000796B91F800C04F78634403F1FF3999FB75
:1090A000FCF307FB03F3681E7033DAF8A8790EFBB4
:1090B0000301B1FBF5F502EB4522C4F8942057B14A
:1090C0002046214C636983F0080141F40025A56125
:1090D000B8471A4A9063B8F89E0698F88446184F25
:1090E00001304FF40023A8F89E064FF48011BB61B5
:1090F0004FF400154FF480024FF400000223032CBC
:10910000B961BD61BA61B861BB617FF45FAA98F8CB
:109110008576002F7FF45AAAD8F87846C8F8884692
:10912000012188F88516FFF751BA079886E60022D4
:109130007FE74FF0FF3EF44658E700BF00000020F5
:10914000000802401010012000000240D8F8FC5135
:1091500020906A692092AE6920963846209BF8F7E5
:1091600069FD38B9D8F8FC1108613846F8F762FD96
:10917000014688B1D8F83C12042905D1D8F8FC0181
:10918000036843F4007505600027D8F83C22634C5F
:1091900088F83872FDF772BED8F8FC01056845F40E
:1091A000807202603B4622464FF00110F8F70CFD3A
:1091B0000028E9D12146D8F8FC415948A123236170
:1091C0003A46F9F799FB00287EF43BABD8F8FC113E
:1091D00000261F964D691F958A691F9238461F9B6E
:1091E000F9F754FB0146002840F09180D8F8FC01C3
:1091F0000469436988F87C4613F0040962D0046965
:10920000484888F87D463B460122474CF8F7DCFC8D
:10921000002854D1D8F8FC71396841F400703860E6
:10922000D8F8FC311E6926701D69657098F87C2697
:1092300000242027FF2A88F8397288F8384288F8F5
:109240003A42364C7DF41AAE01212046F8F76EFC06
:10925000B8F87D6686427DF411AEFDF71BBEFBF7C4
:1092600003F898F8300709283DF6D0AF08EB800CDA
:109270000130CCF8087788F83007FDF7C7BF2B4ED0
:1092800008274FF40065402080244FF48052B761D6
:10929000B561B061B461B261FEE7244E08254FF4B8
:1092A0000062402080214FF48057B561B261B06107
:1092B000B161B761FEE7B878FAF7D6FFD1E70134BC
:1092C000FDF7DCBD17481A4C49463B460122F8F72A
:1092D0007BFC00BB3B46D8F8FC7112483E6826F484
:1092E00080653D60D8F8FC21176927700122F8F7E6
:1092F0006BFC80B9D8F8FC11086840F400730B606F
:10930000D8F8FC61356965703269A2708EE7D8F8CB
:109310003C32FDF7B2BD0234FDF7B0BDBF060120FF
:109320000200010004000100BE060120000002400E
:10933000BD0601202DE9F047089D0E4604460F4664
:10934000002B4AD194468C45B2FA82F260D942B1E0
:10935000C2F12003974020FA03F30CFA02FC1F43EA
:1093600094404FEA1C4E1FFA8CF6B7FBFEF1230C1B
:109370000EFB117743EA074301FB06F098420AD936
:109380001CEB030301F1FF3780F01581984240F296
:109390001281023963441B1AA4B2B3FBFEF00EFB28
:1093A000103344EA034400FB06F6A6420AD91CEB3C
:1093B000040400F1FF3380F00081A64240F2FD80FA
:1093C0006444023840EA0140A41B00211DB1D4408E
:1093D0000023C5E90043BDE8F0878B4205D90DB1F4
:1093E000C5E9000100210846F5E7B3FA83F1002939
:1093F00046D1B34202D3824200F2F580841A66EB72
:10940000030201201746002DE5D0C5E90047E2E739
:10941000002A40F09380A1EB0C034FEA1C471FFA8F
:109420008CFE0121B3FBF7F607FB1630230C43EA51
:1094300000430EFB06F0984208D91CEB030306F12B
:10944000FF3802D2984200F2D08046461B1AA4B2DE
:10945000B3FBF7F007FB103344EA03440EFB00FEB6
:10946000A64508D91CEB040400F1FF3302D2A6453F
:1094700000F2B6801846A4EB0E0440EA0640A5E7C9
:10948000C1F120078B4022FA07FC4CEA030C06FAD4
:1094900001FE20FA07F426FA07F344EA0E0400FA64
:1094A00001F84FEA1C404FEA1449B3FBF0FE1FFAE3
:1094B0008CF600FB1E3349EA03430EFB06F999457F
:1094C00002FA01F20BD91CEB03030EF1FF3A80F014
:1094D0008580994540F28280AEF1020E6344A3EB91
:1094E0000909A4B2B9FBF0F300FB139944EA09445B
:1094F00003FB06F6A64208D91CEB040403F1FF3077
:1095000068D2A64266D9023B644443EA0E40A41BDB
:10951000A0FB02E6B4427346B14652D34FD05DB1D0
:10952000B8EB030264EB090404FA07F722FA01F32B
:109530001F43CC40C5E9007400214CE7C2F1200173
:1095400020FA01F30CFA02FC26FA01F196403343AB
:109550004FEA1C471FFA8CFEB1FBF7F007FB101611
:10956000190C41EA064100FB0EF68E4204FA02F4A1
:1095700008D91CEB010100F1FF382DD28E422BD906
:1095800002386144891B9BB2B1FBF7F607FB161149
:1095900043EA014306FB0EF1994208D91CEB030391
:1095A00006F1FF3814D2994212D9023E63445B1A85
:1095B00046EA004136E73946EDE6184602E7F0454F
:1095C000ADD2BEEB020366EB0C060138B146A6E74E
:1095D0004646ECE7034698E74046D3E7D6467EE7A3
:1095E0006444023847E708460DE7023E63442DE72E
:1095F000830730B547D0541E002A3ED0CAB2034676
:1096000001E0013C39D303F8012B9D07F9D1032C6C
:109610002CD9CDB205EB05250F2C05EB054535D929
:10962000A4F1100222F00F0C03F1100EE6444FEAF1
:10963000121C1A46C2E90055C2E9025510327245A1
:10964000F8D10CF1010214F00C0F03EB021204F03C
:109650000F0C13D0ACF1040323F0030304331344C1
:1096600042F8045B9342FBD10CF003042CB1C9B265
:109670001C4403F8011BA342FBD130BD64461346D2
:10968000002CF4D1F9E703461446C0E71A46A44675
:10969000E0E700BF40EA01039B0710B501D1032AB0
:1096A00017D8844601F1FF3E07E01EF8011F03F8BA
:1096B000011B541E29B19C4622466346002AF4D160
:1096C00010BD9444002CFBD003F8011B6345FBD173
:1096D00010BD8E468446DEF80040A4F1013323EA33
:1096E000040313F0803F71460EF1040EDAD1043A00
:0C96F000032A4CF8044BEED87146D3E777
:1096FC0008B5F6F77FFD00BF024A1368013313600B
:10970C00704700BF4000012080B56F4B6F4A84B09A
:10971C001968914200AF0AD16D4D6E4E1D6086F3F3
:10972C000888A3F5303CDCF80440A047FEE76A4EFD
:10973C006A4BD6F8884044F47005C6F888501A680D
:10974C00674C002042F00101196098601D6825F0FB
:10975C00847222F4803119605C601D68614C25F4C0
:10976C0080224FF000611A60D860B160B460D6F806
:10977C0088505D485D4B45F470049842C6F88840AB
:10978C0007D25E1E321A22F0030259490432FCF74A
:10979C00A1FF58485849884207D24D1E2B1A23F076
:1097AC00030204320021FFF71DFF544E4A48326871
:1097BC0042F4007131603568514A45F4806333607E
:1097CC00316841F480753560C6684FF6FF04264059
:1097DC003243C260F9F7EAF900244048FC60026C9D
:1097EC00484B42F080510164056C474905F08056A6
:1097FC00FE60FA68BC601C6844F440421A601B6846
:10980C0003F44046BE600125BB68CD64846804F057
:10981C000C01042927D0826802F00C03082B1FD0FE
:10982C002E4DAE6806F00C040C2C00F020822B4A56
:10983C00364C01239370206803E02668311A6429A2
:10984C006DD81568AE03F8D5244A956805F00C0060
:10985C00082864D02C4C2D4900262666086809E09F
:10986C0040684202DCD51D4B1B68EDE70C68251ADD
:10987C00022D54D813689D01F8D447F6C07595FA9B
:10988C00A5F04FF44036B0FA80F496FAA6F34FF0F8
:10989C00706393FAA3F54FF0E046B5FA85F896FAA3
:1098AC00A6F307204FF4B473A34000FA08F4234343
:1098BC00154D43F4800646F01003012053602866D2
:1098CC000D68064A28E000BF00C00120AD700DB045
:1098DC00EFBEADDEF82A002000ED00E000380240BB
:1098EC00103000240000000800000020400001207F
:1098FC00F0F202084000012054440120003C0240D8
:10990C000003FA05007000400000474240000120AF
:10991C000E68731B022B02D81468A401F8D5A24957
:10992C000E6806F00F03042B00F2D380052008709C
:10993C000A6802F00F04052C00F0CB809B4D9C4C68
:10994C00A16801F00C03082B00F01881994E984B7C
:10995C0099499868994AC0F3031E714491F81847C5
:10996C00E640974C2E60151BAE10002D7E604BDD33
:10997C00711E54F8043B01F00706984778680125DE
:10998C00A84241DD3EB3012E1ED0022E18D0032E6C
:10999C0012D0042E0CD0052E06D0062E40F062817B
:1099AC0054F8041B8847013554F8043B984701359B
:1099BC0054F8046BB047013554F8040B804701355B
:1099CC0054F8042B9047013554F8041B88477B68E6
:1099DC000135AB4218DDA046083558F8046BB0478A
:1099EC0060688047D8F804209047E168884723696D
:1099FC0098476669B047A0698047E26990477968E3
:109A0C00A94204F12004E6DC6E4C6F4D631B002B65
:109A1C004FEAA3065BDD701E55F8042B00F007041B
:109A2C00904701218E42884651DD94B3012C28D0F9
:109A3C00022C20D0032C18D0042C10D0052C08D0CC
:109A4C00062C40F0098155F8040B80474246013240
:109A5C00904655F8044BA04741460131884655F8CD
:109A6C00043B984740460130804655F8042B444649
:109A7C0090470134A04655F8041B884743460133F0
:109A8C00984655F8040B8047424601329642904660
:109A9C001DDD2C46203554F8041B884755F81C3C1A
:109AAC0098476068804755F8142C904755F8104C2F
:109ABC00A04755F80C1C884755F8083C984755F8B2
:109ACC00040C80474246083296429046E1DCFCF793
:109ADC001DFF374B9D6825F0F00199601E68B2019F
:109AEC007FF52CAF9868394920F0030C4CF002023A
:109AFC009A60086841F2883804E00E68321A4245D0
:109B0C003FF61CAF9D6805F00C06082EF5D1264CCF
:109B1C00236803F00F01052907D90520207022685E
:109B2C0002F00F05052D7FF409AF214EB46824F423
:109B3C00E05343F4A051B160B06820F4604E4EF491
:109B4C000042B260B56805F00C04082C62D00C2CF5
:109B5C0040D0184E164DF024AB6894FAA4FE1C4865
:109B6C00124DBEFA8EF103F0F002CA40024492F894
:109B7C009040E6402E60F9F719F8E0E663680C4E69
:109B8C00606864680B4A00F03F0C7068B2FBFCF331
:109B9C00C4F38811C0F30144013403FB01F16200EA
:109BAC00B1FBF2F6D3E600BF003C024000000020FF
:109BBC00003802400024F4005C020108F0F20208B4
:109BCC00F0F20208F0F20208F0F202084000012064
:109BDC008C9C000874687168766804F03F0847F63E
:109BEC00C07393FAA3F0244C244AB2FBF8F5B0FAF4
:109BFC0080F11E40CE40606805FB06F64FF0E04356
:109C0C0093FAA3FCBCFA8CF100F0E042CA40B6FB1C
:109C1C00F2F69FE773687168766803F03F0847F6C1
:109C2C00C07090FAA0FC144C144AB2FBF8F5BCFAC4
:109C3C008CF10640CE40606805FB06F64FF44033CD
:109C4C0093FAA3FEBEFA8EF100F44032CA40013200
:109C5C005500B6FBF5F67DE755F8043B98474FF0F9
:109C6C000208F0E654F8042B9047022598E6696840
:109C7C004B027FF5DCADF6E5003802400024F40021
:109C8C0001000101010201030104010501060107A4
:109C9C0001080109010A010B010C010D010E010F54
:109CAC0001100111011200800000000004080000E6
:109CBC0025240008992500080B1000000925000830
:109CCC006D2600080D000B000800070004000200C0
:109CDC0001000E00D506B30500048F03000200013D
:109CEC0080007F00400020001000080004000200EB
:109CFC0001006907AA0066001E00FF00AAAA66669A
:109D0C001E1EFE01FFFF00000006101600061016B6
:109D1C000000000001020304010203040607080905
:109D2C00AAAA0000055085ABC5D8E5EEF5FAFD00F2
:109D3C0000402C37D72F7428A622981ED41A9F18AF
:109D4C003F168A1435133C12C0116811FC10CA104E
:109D5C005710F70FBC0FA80F920F670F740F200F3F
:109D6C00CC0E470EDD0D590DAD0C2D0C800BC90A18
:109D7C00140A5509B2083D08EE07D107B907C30705
:109D8C00B907C007AE0789076907B6079F070B0815
:109D9C0009080040CB377F30CB2ADB26CF2241206D
:109DAC00E21D231C001B901A631B9B1C6B1D291EA0
:109DBC00C61D1C1BD117CC145A129610720FEB0E29
:109DCC00E20E8D0FDB10741255138814BE15941609
:109DDC0047150011FE0DD50B1D0AF2081A086A076B
:109DEC000507DD06DB06FB06F8064D07B0074C0839
:109DFC000709A0090040DA3C403AB339123726363D
:109E0C0041359730812AB52681244A24BB24A225CA
:109E1C002324E820F21D6A1BFC18641600141F1280
:109E2C001010200E4C0C9B0A48096908AE070E074F
:109E3C00890621067505A3042204F203CA039103C3
:109E4C0066033E031503EF02D102B7029F028D0297
:109E5C007B02620256020040BC3B15380735583273
:109E6C00CC2F772D4C2B4C296A27A425F623632263
:109E7C00F3209C1F4F1E0B1DCB1B921A601943180D
:109E8C0033172F1636154E147513A212DB1122112F
:109E9C008110FB0F800F780EDA0D630DEA0C5F0C4E
:109EAC00D50B4B0BC80A4F0AE10979091609BA08F8
:109EBC0062081208CB078907C83E603A233C953FDD
:109ECC0000409536012C2924F71D6518D3141C135A
:109EDC004413CF14BE158A17C617B31611154413A5
:109EEC00A6110A10790E130D860B380A11091B08DE
:109EFC00E9079C074507E80686068206AB06E706D7
:109F0C00250757077C073A07BC064606A5058405B6
:109F1C009505CC056D069E063607E90C9C0BE60AEA
:109F2C003C0A9109BC08FB0744079606E405470563
:109F3C00C3045204F703A603640333030D03EA02BC
:109F4C00CD02B402A00294028F029602A802C702AC
:109F5C00F0022E037503CE033704B1044005EE0561
:109F6C00C806CE070209510ADF0BB30DFC0F101304
:109F7C003017851C3B23B42B173500404CA400082C
:109F8C0030ED000884ED020884E9020884E502083B
:109F9C0084E1020884DD020884D9020884D5020811
:109FAC0084D1020884CD020884C9020884C5020841
:109FBC0084C1020830F1000884BD020884B902088B
:109FCC0084B5020884B1020830F5000884AD02089B
:109FDC0084A9020884A5020884A10208849D0208B1
:109FEC00849902088495020884910208848D0208E1
:109FFC0084890208848502088481020830E90008FB
:10A00C00847D020884790208847502088471020830
:10A01C00846D020884690208846502088461020860
:10A02C00845D020884590208845502088451020890
:10A03C00844D0208844902088445020884410208C0
:10A04C000000640994125D1B8E23FA2A7931E536DF
:10A05C00203B143EB13FEC3FC53E423C7138673368
:10A06C00412D1F262B1E8F157C0C2303BBF974F07E
:10A07C0083E719DF67D795D0CACA26C6C2C2B2C059
:10A08C0000C0B2C0C2C226C6CACA95D067D719DFF3
:10A09C0083E774F0BBF923037C0C8F152B1E1F2652
:10A0AC00412D67337138423CC53EEC3FB13F143E05
:10A0BC00203BE5367931FA2A8E235D1B9412640914
:10A0CC0000009CF66CEDA3E472DC06D587CE1BC9B0
:10A0DC00E0C4ECC14FC014C03BC1BEC38FC799CC08
:10A0EC00BFD2E1D9D5E171EA84F3DDFC45068C0FD2
:10A0FC007D18E72099286B2F3635DA393E3D4E3FD7
:10A10C0000404E3F3E3DDA3936356B2F9928E7201B
:10A11C007D188C0F4506DDFC84F371EAD5E1E1D99D
:10A12C00BFD299CC8FC7BEC33BC114C04FC0ECC1CA
:10A13C00E0C41BC987CE06D572DCA3E46CED9CF69B
:10A14C000000640994125D1B8E23FA2A7931E536DE
:10A15C00203B143EB13FEC3FC53E423C7138673367
:10A16C00412D1F262B1E8F157C0C2303BBF974F07D
:10A17C0083E719DF67D795D0CACA26C6C2C2B2C058
:10A18C0000C0B2C0C2C226C6CACA95D067D719DFF2
:10A19C0083E774F0BBF923037C0C8F152B1E1F2651
:10A1AC00412D67337138423CC53EEC3FB13F143E04
:10A1BC00203BE5367931FA2A8E235D1B9412640913
:10A1CC0000009CF66CEDA3E472DC06D587CE1BC9AF
:10A1DC00E0C4ECC14FC014C03BC1BEC38FC799CC07
:10A1EC00BFD2E1D9D5E171EA84F3DDFC45068C0FD1
:10A1FC007D18E72099286B2F3635DA393E3D4E3FD6
:10A20C0000404E3F3E3DDA3936356B2F9928E7201A
:10A21C007D188C0F4506DDFC84F371EAD5E1E1D99C
:10A22C00BFD299CC8FC7BEC33BC114C04FC0ECC1C9
:10A23C00E0C41BC987CE06D572DCA3E46CED9CF69A
:10A24C000000640994125D1B8E23FA2A7931E536DD
:10A25C00203B143EB13FEC3FC53E423C7138673366
:10A26C00412D1F262B1E8F157C0C2303BBF974F07C
:10A27C0083E719DF67D795D0CACA26C6C2C2B2C057
:10A28C0000C0B2C0C2C226C6CACA95D067D719DFF1
:10A29C0083E774F0BBF923037C0C8F152B1E1F2650
:10A2AC00412D67337138423CC53EEC3FB13F143E03
:10A2BC00203BE5367931FA2A8E235D1B9412640912
:10A2CC0000009CF66CEDA3E472DC06D587CE1BC9AE
:10A2DC00E0C4ECC14FC014C03BC1BEC38FC799CC06
:10A2EC00BFD2E1D9D5E171EA84F3DDFC45068C0FD0
:10A2FC007D18E72099286B2F3635DA393E3D4E3FD5
:10A30C0000404E3F3E3DDA3936356B2F9928E72019
:10A31C007D188C0F4506DDFC84F371EAD5E1E1D99B
:10A32C00BFD299CC8FC7BEC33BC114C04FC0ECC1C8
:10A33C00E0C41BC987CE06D572DCA3E46CED9CF699
:10A34C000000640994125D1B8E23FA2A7931E536DC
:10A35C00203B143EB13FEC3FC53E423C7138673365
:10A36C00412D1F262B1E8F157C0C2303BBF974F07B
:10A37C0083E719DF67D795D0CACA26C6C2C2B2C056
:10A38C0000C0B2C0C2C226C6CACA95D067D719DFF0
:10A39C0083E774F0BBF923037C0C8F152B1E1F264F
:10A3AC00412D67337138423CC53EEC3FB13F143E02
:10A3BC00203BE5367931FA2A8E235D1B9412640911
:10A3CC0000009CF66CEDA3E472DC06D587CE1BC9AD
:10A3DC00E0C4ECC14FC014C03BC1BEC38FC799CC05
:10A3EC00BFD2E1D9D5E171EA84F3DDFC45068C0FCF
:10A3FC007D18E72099286B2F3635DA393E3D4E3FD4
:10A40C0000404E3F3E3DDA3936356B2F9928E72018
:10A41C007D188C0F4506DDFC84F371EAD5E1E1D99A
:10A42C00BFD299CC8FC7BEC33BC114C04FC0ECC1C7
:10A43C00E0C41BC987CE06D572DCA3E46CED9CF698
:10A44C000000412D0040412D0000BFD200C0BFD202
:10A45C000000412D0040412D0000BFD200C0BFD2F2
:10A46C000000412D0040412D0000BFD200C0BFD2E2
:10A47C000000412D0040412D0000BFD200C0BFD2D2
:10A48C000000412D0040412D0000BFD200C0BFD2C2
:10A49C000000412D0040412D0000BFD200C0BFD2B2
:10A4AC000000412D0040412D0000BFD200C0BFD2A2
:10A4BC000000412D0040412D0000BFD200C0BFD292
:10A4CC000000412D0040412D0000BFD200C0BFD282
:10A4DC000000412D0040412D0000BFD200C0BFD272
:10A4EC000000412D0040412D0000BFD200C0BFD262
:10A4FC000000412D0040412D0000BFD200C0BFD252
:10A50C000000412D0040412D0000BFD200C0BFD241
:10A51C000000412D0040412D0000BFD200C0BFD231
:10A52C000000412D0040412D0000BFD200C0BFD221
:10A53C000000412D0040412D0000BFD200C0BFD211
:10A54C000000412D0040412D0000BFD200C0BFD201
:10A55C000000412D0040412D0000BFD200C0BFD2F1
:10A56C000000412D0040412D0000BFD200C0BFD2E1
:10A57C000000412D0040412D0000BFD200C0BFD2D1
:10A58C000000412D0040412D0000BFD200C0BFD2C1
:10A59C000000412D0040412D0000BFD200C0BFD2B1
:10A5AC000000412D0040412D0000BFD200C0BFD2A1
:10A5BC000000412D0040412D0000BFD200C0BFD291
:10A5CC000000412D0040412D0000BFD200C0BFD281
:10A5DC000000412D0040412D0000BFD200C0BFD271
:10A5EC000000412D0040412D0000BFD200C0BFD261
:10A5FC000000412D0040412D0000BFD200C0BFD251
:10A60C000000412D0040412D0000BFD200C0BFD240
:10A61C000000412D0040412D0000BFD200C0BFD230
:10A62C000000412D0040412D0000BFD200C0BFD220
:10A63C000000412D0040412D0000BFD200C0BFD210
:10A64C000000412D0040412D0000BFD200C0BFD200
:10A65C000000412D0040412D0000BFD200C0BFD2F0
:10A66C000000412D0040412D0000BFD200C0BFD2E0
:10A67C000000412D0040412D0000BFD200C0BFD2D0
:10A68C000000412D0040412D0000BFD200C0BFD2C0
:10A69C000000412D0040412D0000BFD200C0BFD2B0
:10A6AC000000412D0040412D0000BFD200C0BFD2A0
:10A6BC000000412D0040412D0000BFD200C0BFD290
:10A6CC000000412D0040412D0000BFD200C0BFD280
:10A6DC000000412D0040412D0000BFD200C0BFD270
:10A6EC000000412D0040412D0000BFD200C0BFD260
:10A6FC000000412D0040412D0000BFD200C0BFD250
:10A70C000000412D0040412D0000BFD200C0BFD23F
:10A71C000000412D0040412D0000BFD200C0BFD22F
:10A72C000000412D0040412D0000BFD200C0BFD21F
:10A73C000000412D0040412D0000BFD200C0BFD20F
:10A74C000000412D0040412D0000BFD200C0BFD2FF
:10A75C000000412D0040412D0000BFD200C0BFD2EF
:10A76C000000412D0040412D0000BFD200C0BFD2DF
:10A77C000000412D0040412D0000BFD200C0BFD2CF
:10A78C000000412D0040412D0000BFD200C0BFD2BF
:10A79C000000412D0040412D0000BFD200C0BFD2AF
:10A7AC000000412D0040412D0000BFD200C0BFD29F
:10A7BC000000412D0040412D0000BFD200C0BFD28F
:10A7CC000000412D0040412D0000BFD200C0BFD27F
:10A7DC000000412D0040412D0000BFD200C0BFD26F
:10A7EC000000412D0040412D0000BFD200C0BFD25F
:10A7FC000000412D0040412D0000BFD200C0BFD24F
:10A80C000000412D0040412D0000BFD200C0BFD23E
:10A81C000000412D0040412D0000BFD200C0BFD22E
:10A82C000000412D0040412D0000BFD200C0BFD21E
:10A83C000000412D0040412D0000BFD200C0BFD20E
:10A84C00A4F20208A8F20208B4F20208BCF2020850
:10A85C00C8F20208D8F20208000000405A2E212C3F
:10A86C00EC3FDDFCCD298ACFBBF94FC08CCDA1D8F4
:10A87C00B2C0640926DB53347C0CC53E12363D2233
:10A88C00143E74F08B1F51C86CEDC2C2D6C63AE3AD
:10A89C00BEC38F1511E6823A7D18203BB63B0817D4
:10A8AC00DA39A3E413143BC3D5E18FC752C2EFEEE0
:10A8BC001BC9E720FBF1713E8E2336350E3FF10AA2
:10A8CC006733E1D9D5077CC067D787CE2DC04BFB4A
:10A8DC0095D0FA2A6EFEFB3F412D412DFB3F6EFEBB
:10A8EC00FA2A95D04BFB2DC087CE67D77CC0D507F5
:10A8FC00E1D96733F10A0E3F36358E23713EFBF1F9
:10A90C00E7201BC9EFEE52C28FC7D5E13BC313142E
:10A91C00A3E4DA390817B63B203B7D18823A11E6DE
:10A92C008F15BEC33AE3D6C6C2C26CED51C88B1F9D
:10A93C0074F0143E3D221236C53E7C0C533426DB9B
:10A94C006409B2C0A1D88CCD4FC0BBF98ACFCD2938
:10A95C00DDFCEC3F212C5A2E00400000212CA6D10E
:10A96C00DDFC14C08ACF33D64FC04506A1D8743253
:10A97C0064094E3F5334DA24C53E84F33D22EEC9BC
:10A98C0074F0ECC151C875E0C2C294123AE32A3992
:10A99C008F15423C823AEF19203B83E708174AC4D3
:10A9AC00A3E426C63BC3EDEB8FC72B1EEFEEAE3DEB
:10A9BC00E720E536713E050E363572DCF10AF2C041
:10A9CC00E1D999CC7CC02BF887CE99284BFBD33F8F
:10A9DC00FA2A6B2FFB3F9201412DBFD26EFE05C0B0
:10A9EC0095D006D52DC0B50467D77931D507843FEE
:10A9FC0067331F260E3F0FF58E23CACAFBF18FC19A
:10AA0C001BC919DF52C21111D5E171381314C53CA1
:10AA1C00DA395D1BB63BF8E87D18E0C411E67EC55B
:10AA2C00BEC371EAD6C6C61C6CED3E3D8B1FAF375C
:10AA3C00143E8C0F1236C3DD7C0C3BC126DBADCB38
:10AA4C00B2C09CF68CCD5F27BBF9B13FCD297630D7
:10AA5C00EC3F23035A2EDFD3000000C0A6D1DFD376
:10AA6C0014C0230333D676304506B13F74325F27CA
:10AA7C004E3F9CF6DA24ADCB84F33BC1EEC9C3DD6B
:10AA8C00ECC18C0F75E0AF3794123E3D2A39C61CD1
:10AA9C00423C71EAEF197EC583E7E0C44AC4F8E88A
:10AAAC0026C65D1BEDEBC53C2B1E7138AE3D11115E
:10AABC00E53619DF050E8FC172DCCACAF2C00FF57C
:10AACC0099CC1F262BF8843F99287931D33FB504B4
:10AADC006B2F06D5920105C0BFD2BFD205C0920123
:10AAEC0006D56B2FB504D33F79319928843F2BF8C9
:10AAFC001F2699CC0FF5F2C0CACA72DC8FC1050EA5
:10AB0C0019DFE5361111AE3D71382B1EC53CEDEB4E
:10AB1C005D1B26C6F8E84AC4E0C483E77EC5EF197E
:10AB2C0071EA423CC61C2A393E3D9412AF3775E09F
:10AB3C008C0FECC1C3DDEEC93BC184F3ADCBDA2481
:10AB4C009CF64E3F5F277432B13F4506763033D6C4
:10AB5C00230314C0DFD3A6D100C00000DFD35A2ECC
:10AB6C002303EC3F7630CD29B13FBBF95F278CCD69
:10AB7C009CF6B2C0ADCB26DB3BC17C0CC3DD1236E0
:10AB8C008C0F143EAF378B1F3E3D6CEDC61CD6C6EA
:10AB9C0071EABEC37EC511E6E0C47D18F8E8B63B89
:10ABAC005D1BDA39C53C13147138D5E1111152C251
:10ABBC0019DF1BC98FC1FBF1CACA8E230FF50E3FDB
:10ABCC001F266733843FD507793167D7B5042DC06D
:10ABDC0006D595D005C06EFEBFD2412D9201FB3F2C
:10ABEC006B2FFA2AD33F4BFB992887CE2BF87CC0CE
:10ABFC0099CCE1D9F2C0F10A72DC3635050E713E02
:10AC0C00E536E720AE3DEFEE2B1E8FC7EDEB3BC3D9
:10AC1C0026C6A3E44AC4081783E7203BEF19823AFF
:10AC2C00423C8F152A393AE39412C2C275E051C8DE
:10AC3C00ECC174F0EEC93D2284F3C53EDA245334E2
:10AC4C004E3F64097432A1D845064FC033D68ACF23
:10AC5C0014C0DDFCA6D1212C000000405A2E212C62
:10AC6C00EC3FDDFCCD298ACFBBF94FC08CCDA1D8F0
:10AC7C00B2C0640926DB53347C0CC53E12363D222F
:10AC8C00143E74F08B1F51C86CEDC2C2D6C63AE3A9
:10AC9C00BEC38F1511E6823A7D18203BB63B0817D0
:10ACAC00DA39A3E413143BC3D5E18FC752C2EFEEDC
:10ACBC001BC9E720FBF1713E8E2336350E3FF10A9E
:10ACCC006733E1D9D5077CC067D787CE2DC04BFB46
:10ACDC0095D0FA2A6EFEFB3F412D412DFB3F6EFEB7
:10ACEC00FA2A95D04BFB2DC087CE67D77CC0D507F1
:10ACFC00E1D96733F10A0E3F36358E23713EFBF1F5
:10AD0C00E7201BC9EFEE52C28FC7D5E13BC313142A
:10AD1C00A3E4DA390817B63B203B7D18823A11E6DA
:10AD2C008F15BEC33AE3D6C6C2C26CED51C88B1F99
:10AD3C0074F0143E3D221236C53E7C0C533426DB97
:10AD4C006409B2C0A1D88CCD4FC0BBF98ACFCD2934
:10AD5C00DDFCEC3F212C5A2E00400000212CA6D10A
:10AD6C00DDFC14C08ACF33D64FC04506A1D874324F
:10AD7C0064094E3F5334DA24C53E84F33D22EEC9B8
:10AD8C0074F0ECC151C875E0C2C294123AE32A398E
:10AD9C008F15423C823AEF19203B83E708174AC4CF
:10ADAC00A3E426C63BC3EDEB8FC72B1EEFEEAE3DE7
:10ADBC00E720E536713E050E363572DCF10AF2C03D
:10ADCC00E1D999CC7CC02BF887CE99284BFBD33F8B
:10ADDC00FA2A6B2FFB3F9201412DBFD26EFE05C0AC
:10ADEC0095D006D52DC0B50467D77931D507843FEA
:10ADFC0067331F260E3F0FF58E23CACAFBF18FC196
:10AE0C001BC919DF52C21111D5E171381314C53C9D
:10AE1C00DA395D1BB63BF8E87D18E0C411E67EC557
:10AE2C00BEC371EAD6C6C61C6CED3E3D8B1FAF3758
:10AE3C00143E8C0F1236C3DD7C0C3BC126DBADCB34
:10AE4C00B2C09CF68CCD5F27BBF9B13FCD297630D3
:10AE5C00EC3F23035A2EDFD3000000C0A6D1DFD372
:10AE6C0014C0230333D676304506B13F74325F27C6
:10AE7C004E3F9CF6DA24ADCB84F33BC1EEC9C3DD67
:10AE8C00ECC18C0F75E0AF3794123E3D2A39C61CCD
:10AE9C00423C71EAEF197EC583E7E0C44AC4F8E886
:10AEAC0026C65D1BEDEBC53C2B1E7138AE3D11115A
:10AEBC00E53619DF050E8FC172DCCACAF2C00FF578
:10AECC0099CC1F262BF8843F99287931D33FB504B0
:10AEDC006B2F06D5920105C0BFD2BFD205C092011F
:10AEEC0006D56B2FB504D33F79319928843F2BF8C5
:10AEFC001F2699CC0FF5F2C0CACA72DC8FC1050EA1
:10AF0C0019DFE5361111AE3D71382B1EC53CEDEB4A
:10AF1C005D1B26C6F8E84AC4E0C483E77EC5EF197A
:10AF2C0071EA423CC61C2A393E3D9412AF3775E09B
:10AF3C008C0FECC1C3DDEEC93BC184F3ADCBDA247D
:10AF4C009CF64E3F5F277432B13F4506763033D6C0
:10AF5C00230314C0DFD3A6D100C00000DFD35A2EC8
:10AF6C002303EC3F7630CD29B13FBBF95F278CCD65
:10AF7C009CF6B2C0ADCB26DB3BC17C0CC3DD1236DC
:10AF8C008C0F143EAF378B1F3E3D6CEDC61CD6C6E6
:10AF9C0071EABEC37EC511E6E0C47D18F8E8B63B85
:10AFAC005D1BDA39C53C13147138D5E1111152C24D
:10AFBC0019DF1BC98FC1FBF1CACA8E230FF50E3FD7
:10AFCC001F266733843FD507793167D7B5042DC069
:10AFDC0006D595D005C06EFEBFD2412D9201FB3F28
:10AFEC006B2FFA2AD33F4BFB992887CE2BF87CC0CA
:10AFFC0099CCE1D9F2C0F10A72DC3635050E713EFE
:10B00C00E536E720AE3DEFEE2B1E8FC7EDEB3BC3D5
:10B01C0026C6A3E44AC4081783E7203BEF19823AFB
:10B02C00423C8F152A393AE39412C2C275E051C8DA
:10B03C00ECC174F0EEC93D2284F3C53EDA245334DE
:10B04C004E3F64097432A1D845064FC033D68ACF1F
:10B05C0014C0DDFCA6D1212C00000040DA395D1BA8
:10B06C00793167D774F0ECC13BC184F3E1D9673314
:10B07C002B1E7138EC3FDDFC7D18E0C406D595D055
:10B08C00C2C294129CF64E3F36358E23E53619DF3C
:10B09C00BBF94FC0BEC371EABFD2412D8F15423CE4
:10B0AC00B13F4506E7201BC972DCCACAB2C06409AD
:10B0BC006CED3E3D6B2FFA2A203B83E7230314C033
:10B0CC008FC7D5E199CC1F267C0CC53E143E8C0F46
:10B0DC00992887CEA3E426C600C00000A3E4DA3981
:10B0EC0099287931143E74F07C0C3BC199CCE1D990
:10B0FC008FC72B1E2303EC3F203B7D186B2F06D5EF
:10B10C006CEDC2C2B2C09CF672DC3635E720E53677
:10B11C00B13FBBF98F15BEC3BFD2BFD2BEC38F1513
:10B12C00BBF9B13FE536E720363572DC9CF6B2C090
:10B13C00C2C26CED06D56B2F7D18203BEC3F230370
:10B14C002B1E8FC7E1D999CC3BC17C0C74F0143EFB
:10B15C0079319928DA39A3E4000000C026C6A3E4AB
:10B16C0087CE99288C0F143EC53E7C0C1F2699CC9B
:10B17C00D5E18FC714C0230383E7203BFA2A6B2F3A
:10B18C003E3D6CED6409B2C0CACA72DC1BC9E72033
:10B19C004506B13F423C8F15412DBFD271EABEC36B
:10B1AC004FC0BBF919DFE5368E2336354E3F9CF682
:10B1BC009412C2C295D006D5E0C47D18DDFCEC3FDC
:10B1CC0071382B1E6733E1D984F33BC1ECC174F0A9
:10B1DC0067D779315D1BDA39004000005D1B26C64C
:10B1EC0067D787CEECC18C0F84F3C53E67331F261F
:10B1FC007138D5E1DDFC14C0E0C483E795D0FA2AA0
:10B20C0094123E3D4E3F64098E23CACA19DF1BC9F6
:10B21C004FC0450671EA423C412D412D423C71EA3A
:10B22C0045064FC01BC919DFCACA8E2364094E3F9D
:10B23C003E3D9412FA2A95D083E7E0C414C0DDFC9D
:10B24C00D5E171381F266733C53E84F38C0FECC1F2
:10B25C0087CE67D726C65D1B00000040DA395D1B20
:10B26C00793167D774F0ECC13BC184F3E1D9673312
:10B27C002B1E7138EC3FDDFC7D18E0C406D595D053
:10B28C00C2C294129CF64E3F36358E23E53619DF3A
:10B29C00BBF94FC0BEC371EABFD2412D8F15423CE2
:10B2AC00B13F4506E7201BC972DCCACAB2C06409AB
:10B2BC006CED3E3D6B2FFA2A203B83E7230314C031
:10B2CC008FC7D5E199CC1F267C0CC53E143E8C0F44
:10B2DC00992887CEA3E426C600C00000A3E4DA397F
:10B2EC0099287931143E74F07C0C3BC199CCE1D98E
:10B2FC008FC72B1E2303EC3F203B7D186B2F06D5ED
:10B30C006CEDC2C2B2C09CF672DC3635E720E53675
:10B31C00B13FBBF98F15BEC3BFD2BFD2BEC38F1511
:10B32C00BBF9B13FE536E720363572DC9CF6B2C08E
:10B33C00C2C26CED06D56B2F7D18203BEC3F23036E
:10B34C002B1E8FC7E1D999CC3BC17C0C74F0143EF9
:10B35C0079319928DA39A3E4000000C026C6A3E4A9
:10B36C0087CE99288C0F143EC53E7C0C1F2699CC99
:10B37C00D5E18FC714C0230383E7203BFA2A6B2F38
:10B38C003E3D6CED6409B2C0CACA72DC1BC9E72031
:10B39C004506B13F423C8F15412DBFD271EABEC369
:10B3AC004FC0BBF919DFE5368E2336354E3F9CF680
:10B3BC009412C2C295D006D5E0C47D18DDFCEC3FDA
:10B3CC0071382B1E6733E1D984F33BC1ECC174F0A7
:10B3DC0067D779315D1BDA39004000005D1B26C64A
:10B3EC0067D787CEECC18C0F84F3C53E67331F261D
:10B3FC007138D5E1DDFC14C0E0C483E795D0FA2A9E
:10B40C0094123E3D4E3F64098E23CACA19DF1BC9F4
:10B41C004FC0450671EA423C412D412D423C71EA38
:10B42C0045064FC01BC919DFCACA8E2364094E3F9B
:10B43C003E3D9412FA2A95D083E7E0C414C0DDFC9B
:10B44C00D5E171381F266733C53E84F38C0FECC1F0
:10B45C0087CE67D726C65D1B00000040DA395D1B1E
:10B46C00793167D774F0ECC13BC184F3E1D9673310
:10B47C002B1E7138EC3FDDFC7D18E0C406D595D051
:10B48C00C2C294129CF64E3F36358E23E53619DF38
:10B49C00BBF94FC0BEC371EABFD2412D8F15423CE0
:10B4AC00B13F4506E7201BC972DCCACAB2C06409A9
:10B4BC006CED3E3D6B2FFA2A203B83E7230314C02F
:10B4CC008FC7D5E199CC1F267C0CC53E143E8C0F42
:10B4DC00992887CEA3E426C600C00000A3E4DA397D
:10B4EC0099287931143E74F07C0C3BC199CCE1D98C
:10B4FC008FC72B1E2303EC3F203B7D186B2F06D5EB
:10B50C006CEDC2C2B2C09CF672DC3635E720E53673
:10B51C00B13FBBF98F15BEC3BFD2BFD2BEC38F150F
:10B52C00BBF9B13FE536E720363572DC9CF6B2C08C
:10B53C00C2C26CED06D56B2F7D18203BEC3F23036C
:10B54C002B1E8FC7E1D999CC3BC17C0C74F0143EF7
:10B55C0079319928DA39A3E4000000C026C6A3E4A7
:10B56C0087CE99288C0F143EC53E7C0C1F2699CC97
:10B57C00D5E18FC714C0230383E7203BFA2A6B2F36
:10B58C003E3D6CED6409B2C0CACA72DC1BC9E7202F
:10B59C004506B13F423C8F15412DBFD271EABEC367
:10B5AC004FC0BBF919DFE5368E2336354E3F9CF67E
:10B5BC009412C2C295D006D5E0C47D18DDFCEC3FD8
:10B5CC0071382B1E6733E1D984F33BC1ECC174F0A5
:10B5DC0067D779315D1BDA39004000005D1B26C648
:10B5EC0067D787CEECC18C0F84F3C53E67331F261B
:10B5FC007138D5E1DDFC14C0E0C483E795D0FA2A9C
:10B60C0094123E3D4E3F64098E23CACA19DF1BC9F2
:10B61C004FC0450671EA423C412D412D423C71EA36
:10B62C0045064FC01BC919DFCACA8E2364094E3F99
:10B63C003E3D9412FA2A95D083E7E0C414C0DDFC99
:10B64C00D5E171381F266733C53E84F38C0FECC1EE
:10B65C0087CE67D726C65D1B00000040DA395D1B1C
:10B66C00793167D774F0ECC13BC184F3E1D967330E
:10B67C002B1E7138EC3FDDFC7D18E0C406D595D04F
:10B68C00C2C294129CF64E3F36358E23E53619DF36
:10B69C00BBF94FC0BEC371EABFD2412D8F15423CDE
:10B6AC00B13F4506E7201BC972DCCACAB2C06409A7
:10B6BC006CED3E3D6B2FFA2A203B83E7230314C02D
:10B6CC008FC7D5E199CC1F267C0CC53E143E8C0F40
:10B6DC00992887CEA3E426C600C00000A3E4DA397B
:10B6EC0099287931143E74F07C0C3BC199CCE1D98A
:10B6FC008FC72B1E2303EC3F203B7D186B2F06D5E9
:10B70C006CEDC2C2B2C09CF672DC3635E720E53671
:10B71C00B13FBBF98F15BEC3BFD2BFD2BEC38F150D
:10B72C00BBF9B13FE536E720363572DC9CF6B2C08A
:10B73C00C2C26CED06D56B2F7D18203BEC3F23036A
:10B74C002B1E8FC7E1D999CC3BC17C0C74F0143EF5
:10B75C0079319928DA39A3E4000000C026C6A3E4A5
:10B76C0087CE99288C0F143EC53E7C0C1F2699CC95
:10B77C00D5E18FC714C0230383E7203BFA2A6B2F34
:10B78C003E3D6CED6409B2C0CACA72DC1BC9E7202D
:10B79C004506B13F423C8F15412DBFD271EABEC365
:10B7AC004FC0BBF919DFE5368E2336354E3F9CF67C
:10B7BC009412C2C295D006D5E0C47D18DDFCEC3FD6
:10B7CC0071382B1E6733E1D984F33BC1ECC174F0A3
:10B7DC0067D779315D1BDA39004000005D1B26C646
:10B7EC0067D787CEECC18C0F84F3C53E67331F2619
:10B7FC007138D5E1DDFC14C0E0C483E795D0FA2A9A
:10B80C0094123E3D4E3F64098E23CACA19DF1BC9F0
:10B81C004FC0450671EA423C412D412D423C71EA34
:10B82C0045064FC01BC919DFCACA8E2364094E3F97
:10B83C003E3D9412FA2A95D083E7E0C414C0DDFC97
:10B84C00D5E171381F266733C53E84F38C0FECC1EC
:10B85C0087CE67D726C65D1B00000040793199283A
:10B86C00C53E84F32B1E8FC783E7E0C4C2C26CEDC8
:10B87C00CACA8E23BBF9B13F412D412DB13FBBF953
:10B88C008E23CACA6CEDC2C2E0C483E78FC72B1EDD
:10B89C0084F3C53E9928793100400000992887CE61
:10B8AC0084F33BC18FC7D5E1E0C47D186CED3E3D00
:10B8BC008E233635B13F4506412DBFD2BBF94FC063
:10B8CC00CACA72DCC2C2941283E7203B2B1E7138A9
:10B8DC00C53E7C0C793167D7000000C087CE67D796
:10B8EC003BC17C0CD5E171387D18203B3E3D941258
:10B8FC00363572DC45064FC0BFD2BFD24FC04506AD
:10B90C0072DC363594123E3D203B7D187138D5E102
:10B91C007C0C3BC167D787CE00C0000067D779315C
:10B92C007C0CC53E71382B1E203B83E79412C2C29F
:10B93C0072DCCACA4FC0BBF9BFD2412D4506B13F1C
:10B94C0036358E233E3D6CED7D18E0C4D5E18FC7B6
:10B95C003BC184F387CE99280000004079319928A7
:10B96C00C53E84F32B1E8FC783E7E0C4C2C26CEDC7
:10B97C00CACA8E23BBF9B13F412D412DB13FBBF952
:10B98C008E23CACA6CEDC2C2E0C483E78FC72B1EDC
:10B99C0084F3C53E9928793100400000992887CE60
:10B9AC0084F33BC18FC7D5E1E0C47D186CED3E3DFF
:10B9BC008E233635B13F4506412DBFD2BBF94FC062
:10B9CC00CACA72DCC2C2941283E7203B2B1E7138A8
:10B9DC00C53E7C0C793167D7000000C087CE67D795
:10B9EC003BC17C0CD5E171387D18203B3E3D941257
:10B9FC00363572DC45064FC0BFD2BFD24FC04506AC
:10BA0C0072DC363594123E3D203B7D187138D5E101
:10BA1C007C0C3BC167D787CE00C0000067D779315B
:10BA2C007C0CC53E71382B1E203B83E79412C2C29E
:10BA3C0072DCCACA4FC0BBF9BFD2412D4506B13F1B
:10BA4C0036358E233E3D6CED7D18E0C4D5E18FC7B5
:10BA5C003BC184F387CE99280000004079319928A6
:10BA6C00C53E84F32B1E8FC783E7E0C4C2C26CEDC6
:10BA7C00CACA8E23BBF9B13F412D412DB13FBBF951
:10BA8C008E23CACA6CEDC2C2E0C483E78FC72B1EDB
:10BA9C0084F3C53E9928793100400000992887CE5F
:10BAAC0084F33BC18FC7D5E1E0C47D186CED3E3DFE
:10BABC008E233635B13F4506412DBFD2BBF94FC061
:10BACC00CACA72DCC2C2941283E7203B2B1E7138A7
:10BADC00C53E7C0C793167D7000000C087CE67D794
:10BAEC003BC17C0CD5E171387D18203B3E3D941256
:10BAFC00363572DC45064FC0BFD2BFD24FC04506AB
:10BB0C0072DC363594123E3D203B7D187138D5E100
:10BB1C007C0C3BC167D787CE00C0000067D779315A
:10BB2C007C0CC53E71382B1E203B83E79412C2C29D
:10BB3C0072DCCACA4FC0BBF9BFD2412D4506B13F1A
:10BB4C0036358E233E3D6CED7D18E0C4D5E18FC7B4
:10BB5C003BC184F387CE99280000004079319928A5
:10BB6C00C53E84F32B1E8FC783E7E0C4C2C26CEDC5
:10BB7C00CACA8E23BBF9B13F412D412DB13FBBF950
:10BB8C008E23CACA6CEDC2C2E0C483E78FC72B1EDA
:10BB9C0084F3C53E9928793100400000992887CE5E
:10BBAC0084F33BC18FC7D5E1E0C47D186CED3E3DFD
:10BBBC008E233635B13F4506412DBFD2BBF94FC060
:10BBCC00CACA72DCC2C2941283E7203B2B1E7138A6
:10BBDC00C53E7C0C793167D7000000C087CE67D793
:10BBEC003BC17C0CD5E171387D18203B3E3D941255
:10BBFC00363572DC45064FC0BFD2BFD24FC04506AA
:10BC0C0072DC363594123E3D203B7D187138D5E1FF
:10BC1C007C0C3BC167D787CE00C0000067D7793159
:10BC2C007C0CC53E71382B1E203B83E79412C2C29C
:10BC3C0072DCCACA4FC0BBF9BFD2412D4506B13F19
:10BC4C0036358E233E3D6CED7D18E0C4D5E18FC7B3
:10BC5C003BC184F387CE99280000004079319928A4
:10BC6C00C53E84F32B1E8FC783E7E0C4C2C26CEDC4
:10BC7C00CACA8E23BBF9B13F412D412DB13FBBF94F
:10BC8C008E23CACA6CEDC2C2E0C483E78FC72B1ED9
:10BC9C0084F3C53E9928793100400000992887CE5D
:10BCAC0084F33BC18FC7D5E1E0C47D186CED3E3DFC
:10BCBC008E233635B13F4506412DBFD2BBF94FC05F
:10BCCC00CACA72DCC2C2941283E7203B2B1E7138A5
:10BCDC00C53E7C0C793167D7000000C087CE67D792
:10BCEC003BC17C0CD5E171387D18203B3E3D941254
:10BCFC00363572DC45064FC0BFD2BFD24FC04506A9
:10BD0C0072DC363594123E3D203B7D187138D5E1FE
:10BD1C007C0C3BC167D787CE00C0000067D7793158
:10BD2C007C0CC53E71382B1E203B83E79412C2C29B
:10BD3C0072DCCACA4FC0BBF9BFD2412D4506B13F18
:10BD4C0036358E233E3D6CED7D18E0C4D5E18FC7B2
:10BD5C003BC184F387CE99280000004079319928A3
:10BD6C00C53E84F32B1E8FC783E7E0C4C2C26CEDC3
:10BD7C00CACA8E23BBF9B13F412D412DB13FBBF94E
:10BD8C008E23CACA6CEDC2C2E0C483E78FC72B1ED8
:10BD9C0084F3C53E9928793100400000992887CE5C
:10BDAC0084F33BC18FC7D5E1E0C47D186CED3E3DFB
:10BDBC008E233635B13F4506412DBFD2BBF94FC05E
:10BDCC00CACA72DCC2C2941283E7203B2B1E7138A4
:10BDDC00C53E7C0C793167D7000000C087CE67D791
:10BDEC003BC17C0CD5E171387D18203B3E3D941253
:10BDFC00363572DC45064FC0BFD2BFD24FC04506A8
:10BE0C0072DC363594123E3D203B7D187138D5E1FD
:10BE1C007C0C3BC167D787CE00C0000067D7793157
:10BE2C007C0CC53E71382B1E203B83E79412C2C29A
:10BE3C0072DCCACA4FC0BBF9BFD2412D4506B13F17
:10BE4C0036358E233E3D6CED7D18E0C4D5E18FC7B1
:10BE5C003BC184F387CE99280000004079319928A2
:10BE6C00C53E84F32B1E8FC783E7E0C4C2C26CEDC2
:10BE7C00CACA8E23BBF9B13F412D412DB13FBBF94D
:10BE8C008E23CACA6CEDC2C2E0C483E78FC72B1ED7
:10BE9C0084F3C53E9928793100400000992887CE5B
:10BEAC0084F33BC18FC7D5E1E0C47D186CED3E3DFA
:10BEBC008E233635B13F4506412DBFD2BBF94FC05D
:10BECC00CACA72DCC2C2941283E7203B2B1E7138A3
:10BEDC00C53E7C0C793167D7000000C087CE67D790
:10BEEC003BC17C0CD5E171387D18203B3E3D941252
:10BEFC00363572DC45064FC0BFD2BFD24FC04506A7
:10BF0C0072DC363594123E3D203B7D187138D5E1FC
:10BF1C007C0C3BC167D787CE00C0000067D7793156
:10BF2C007C0CC53E71382B1E203B83E79412C2C299
:10BF3C0072DCCACA4FC0BBF9BFD2412D4506B13F16
:10BF4C0036358E233E3D6CED7D18E0C4D5E18FC7B0
:10BF5C003BC184F387CE99280000004079319928A1
:10BF6C00C53E84F32B1E8FC783E7E0C4C2C26CEDC1
:10BF7C00CACA8E23BBF9B13F412D412DB13FBBF94C
:10BF8C008E23CACA6CEDC2C2E0C483E78FC72B1ED6
:10BF9C0084F3C53E9928793100400000992887CE5A
:10BFAC0084F33BC18FC7D5E1E0C47D186CED3E3DF9
:10BFBC008E233635B13F4506412DBFD2BBF94FC05C
:10BFCC00CACA72DCC2C2941283E7203B2B1E7138A2
:10BFDC00C53E7C0C793167D7000000C087CE67D78F
:10BFEC003BC17C0CD5E171387D18203B3E3D941251
:10BFFC00363572DC45064FC0BFD2BFD24FC04506A6
:10C00C0072DC363594123E3D203B7D187138D5E1FB
:10C01C007C0C3BC167D787CE00C0000067D7793155
:10C02C007C0CC53E71382B1E203B83E79412C2C298
:10C03C0072DCCACA4FC0BBF9BFD2412D4506B13F15
:10C04C0036358E233E3D6CED7D18E0C4D5E18FC7AF
:10C05C003BC184F387CE99280000004012363D2264
:10C06C00DA39A3E4D5077CC087CE67D73BC313145A
:10C07C0074F0143E212C5A2EC53E84F308174AC482
:10C08C00E1D999CC2DC0B504D5E171388B1FAF37F0
:10C09C00EC3F2303DA24ADCB83E7E0C4F2C00FF509
:10C0AC0006D56B2F1111AE3D3E3D9412763033D632
:10C0BC009CF6B2C07EC511E6CACA8E239201FB3F24
:10C0CC00E536E7202A393AE345064FC08CCDA1D896
:10C0DC00BEC38F15FBF1713E412D412D713EFBF11D
:10C0EC008F15BEC3A1D88CCD4FC045063AE32A3973
:10C0FC00E720E536FB3F92018E23CACA11E67EC5C6
:10C10C00B2C09CF633D6763094123E3DAE3D111142
:10C11C006B2F06D50FF5F2C0E0C483E7ADCBDA2464
:10C12C002303EC3FAF378B1F7138D5E1B5042DC01D
:10C13C0099CCE1D94AC4081784F3C53E5A2E212C58
:10C14C00143E74F013143BC367D787CE7CC0D5075D
:10C15C00A3E4DA393D221236004000003D22EEC93C
:10C16C00A3E426C67CC02BF867D779311314C53CE1
:10C17C00143E8C0F5A2EDFD384F33BC14AC4F8E82B
:10C18C0099CC1F26B504D33F71382B1EAF3775E001
:10C19C00230314C0ADCB26DBE0C47D180FF50E3F96
:10C1AC006B2FFA2AAE3DEFEE9412C2C233D68ACF71
:10C1BC00B2C0640911E6823A8E233635FB3F6EFE1F
:10C1CC00E7201BC93AE3D6C64FC0BBF9A1D87432DD
:10C1DC008F15423C713E050E412DBFD2FBF18FC134
:10C1EC00BEC371EA8CCD5F274506B13F2A39C61C08
:10C1FC00E53619DF920105C0CACA72DC7EC5EF199B
:10C20C009CF64E3F7630CD293E3D6CED111152C25D
:10C21C0006D595D0F2C0F10A83E7203BDA245334DB
:10C22C00EC3FDDFC8B1F51C8D5E18FC72DC04BFBFC
:10C23C00E1D967330817B63BC53E7C0C212CA6D13F
:10C24C0074F0ECC13BC3EDEB87CE9928D507843F46
:10C25C00DA395D1B1236C3DD000000C0EEC9C3DD48
:10C26C0026C65D1B2BF8843F79319928C53CEDEB34
:10C27C008C0FECC1DFD3A6D13BC17C0CF8E8B63BEC
:10C28C001F266733D33F4BFB2B1E8FC775E051C85E
:10C29C0014C0DDFC26DB53347D18203B0E3FF10A25
:10C2AC00FA2A95D0EFEE52C2C2C26CED8ACFCD29DC
:10C2BC0064094E3F823AEF19363572DC6EFE05C0CA
:10C2CC001BC919DFD6C6C61CBBF9B13F74325F2738
:10C2DC00423C71EA050E8FC1BFD2BFD28FC1050E91
:10C2EC0071EA423C5F277432B13FBBF9C61CD6C61B
:10C2FC0019DF1BC905C06EFE72DC3635EF19823AA8
:10C30C004E3F6409CD298ACF6CEDC2C252C2EFEE0A
:10C31C0095D0FA2AF10A0E3F203B7D18533426DBC8
:10C32C00DDFC14C051C875E08FC72B1E4BFBD33FEF
:10C33C0067331F26B63BF8E87C0C3BC1A6D1DFD394
:10C34C00ECC18C0FEDEBC53C99287931843F2BF86F
:10C35C005D1B26C6C3DDEEC900C00000C3DD12366E
:10C36C005D1BDA39843FD507992887CEEDEB3BC3AB
:10C37C00ECC174F0A6D1212C7C0CC53EB63B081741
:10C38C006733E1D94BFB2DC08FC7D5E151C88B1F4B
:10C39C00DDFCEC3F5334DA24203B83E7F10AF2C096
:10C3AC0095D006D552C211116CED3E3DCD2976309B
:10C3BC004E3F9CF6EF197EC572DCCACA05C09201CD
:10C3CC0019DFE536C61C2A39B13F45065F278CCDEF
:10C3DC0071EABEC38FC1FBF1BFD2412D050E713E78
:10C3EC00423C8F157432A1D8BBF94FC0D6C63AE384
:10C3FC001BC9E7206EFEFB3F36358E23823A11E6D1
:10C40C006409B2C08ACF33D6C2C29412EFEEAE3DED
:10C41C00FA2A6B2F0E3F0FF57D18E0C426DBADCB4F
:10C42C0014C0230375E0AF372B1E7138D33FB5040E
:10C43C001F2699CCF8E84AC43BC184F3DFD35A2EAB
:10C44C008C0F143EC53C1314793167D72BF87CC084
:10C45C0026C6A3E4EEC93D220000004012363D2260
:10C46C00DA39A3E4D5077CC087CE67D73BC3131456
:10C47C0074F0143E212C5A2EC53E84F308174AC47E
:10C48C00E1D999CC2DC0B504D5E171388B1FAF37EC
:10C49C00EC3F2303DA24ADCB83E7E0C4F2C00FF505
:10C4AC0006D56B2F1111AE3D3E3D9412763033D62E
:10C4BC009CF6B2C07EC511E6CACA8E239201FB3F20
:10C4CC00E536E7202A393AE345064FC08CCDA1D892
:10C4DC00BEC38F15FBF1713E412D412D713EFBF119
:10C4EC008F15BEC3A1D88CCD4FC045063AE32A396F
:10C4FC00E720E536FB3F92018E23CACA11E67EC5C2
:10C50C00B2C09CF633D6763094123E3DAE3D11113E
:10C51C006B2F06D50FF5F2C0E0C483E7ADCBDA2460
:10C52C002303EC3FAF378B1F7138D5E1B5042DC019
:10C53C0099CCE1D94AC4081784F3C53E5A2E212C54
:10C54C00143E74F013143BC367D787CE7CC0D50759
:10C55C00A3E4DA393D221236004000003D22EEC938
:10C56C00A3E426C67CC02BF867D779311314C53CDD
:10C57C00143E8C0F5A2EDFD384F33BC14AC4F8E827
:10C58C0099CC1F26B504D33F71382B1EAF3775E0FD
:10C59C00230314C0ADCB26DBE0C47D180FF50E3F92
:10C5AC006B2FFA2AAE3DEFEE9412C2C233D68ACF6D
:10C5BC00B2C0640911E6823A8E233635FB3F6EFE1B
:10C5CC00E7201BC93AE3D6C64FC0BBF9A1D87432D9
:10C5DC008F15423C713E050E412DBFD2FBF18FC130
:10C5EC00BEC371EA8CCD5F274506B13F2A39C61C04
:10C5FC00E53619DF920105C0CACA72DC7EC5EF1997
:10C60C009CF64E3F7630CD293E3D6CED111152C259
:10C61C0006D595D0F2C0F10A83E7203BDA245334D7
:10C62C00EC3FDDFC8B1F51C8D5E18FC72DC04BFBF8
:10C63C00E1D967330817B63BC53E7C0C212CA6D13B
:10C64C0074F0ECC13BC3EDEB87CE9928D507843F42
:10C65C00DA395D1B1236C3DD000000C0EEC9C3DD44
:10C66C0026C65D1B2BF8843F79319928C53CEDEB30
:10C67C008C0FECC1DFD3A6D13BC17C0CF8E8B63BE8
:10C68C001F266733D33F4BFB2B1E8FC775E051C85A
:10C69C0014C0DDFC26DB53347D18203B0E3FF10A21
:10C6AC00FA2A95D0EFEE52C2C2C26CED8ACFCD29D8
:10C6BC0064094E3F823AEF19363572DC6EFE05C0C6
:10C6CC001BC919DFD6C6C61CBBF9B13F74325F2734
:10C6DC00423C71EA050E8FC1BFD2BFD28FC1050E8D
:10C6EC0071EA423C5F277432B13FBBF9C61CD6C617
:10C6FC0019DF1BC905C06EFE72DC3635EF19823AA4
:10C70C004E3F6409CD298ACF6CEDC2C252C2EFEE06
:10C71C0095D0FA2AF10A0E3F203B7D18533426DBC4
:10C72C00DDFC14C051C875E08FC72B1E4BFBD33FEB
:10C73C0067331F26B63BF8E87C0C3BC1A6D1DFD390
:10C74C00ECC18C0FEDEBC53C99287931843F2BF86B
:10C75C005D1B26C6C3DDEEC900C00000C3DD12366A
:10C76C005D1BDA39843FD507992887CEEDEB3BC3A7
:10C77C00ECC174F0A6D1212C7C0CC53EB63B08173D
:10C78C006733E1D94BFB2DC08FC7D5E151C88B1F47
:10C79C00DDFCEC3F5334DA24203B83E7F10AF2C092
:10C7AC0095D006D552C211116CED3E3DCD29763097
:10C7BC004E3F9CF6EF197EC572DCCACA05C09201C9
:10C7CC0019DFE536C61C2A39B13F45065F278CCDEB
:10C7DC0071EABEC38FC1FBF1BFD2412D050E713E74
:10C7EC00423C8F157432A1D8BBF94FC0D6C63AE380
:10C7FC001BC9E7206EFEFB3F36358E23823A11E6CD
:10C80C006409B2C08ACF33D6C2C29412EFEEAE3DE9
:10C81C00FA2A6B2F0E3F0FF57D18E0C426DBADCB4B
:10C82C0014C0230375E0AF372B1E7138D33FB5040A
:10C83C001F2699CCF8E84AC43BC184F3DFD35A2EA7
:10C84C008C0F143EC53C1314793167D72BF87CC080
:10C85C0026C6A3E4EEC93D220000004000400000C3
:10C86C00000000C000C000000000004000400000BC
:10C87C00000000C000C000000000004000400000AC
:10C88C00000000C000C0000000000040004000009C
:10C89C00000000C000C0000000000040004000008C
:10C8AC00000000C000C0000000000040004000007C
:10C8BC00000000C000C0000000000040004000006C
:10C8CC00000000C000C0000000000040004000005C
:10C8DC00000000C000C0000000000040004000004C
:10C8EC00000000C000C0000000000040004000003C
:10C8FC00000000C000C0000000000040004000002C
:10C90C00000000C000C0000000000040004000001B
:10C91C00000000C000C0000000000040004000000B
:10C92C00000000C000C000000000004000400000FB
:10C93C00000000C000C000000000004000400000EB
:10C94C00000000C000C000000000004000400000DB
:10C95C00000000C000C000000000004000400000CB
:10C96C00000000C000C000000000004000400000BB
:10C97C00000000C000C000000000004000400000AB
:10C98C00000000C000C0000000000040004000009B
:10C99C00000000C000C0000000000040004000008B
:10C9AC00000000C000C0000000000040004000007B
:10C9BC00000000C000C0000000000040004000006B
:10C9CC00000000C000C0000000000040004000005B
:10C9DC00000000C000C0000000000040004000004B
:10C9EC00000000C000C0000000000040004000003B
:10C9FC00000000C000C0000000000040004000002B
:10CA0C00000000C000C0000000000040004000001A
:10CA1C00000000C000C0000000000040004000000A
:10CA2C00000000C000C000000000004000400000FA
:10CA3C00000000C000C000000000004000400000EA
:10CA4C00000000C000C000000000004000400000DA
:10CA5C00000000C000C000000000004000400000CA
:10CA6C00000000C000C000000000004000400000BA
:10CA7C00000000C000C000000000004000400000AA
:10CA8C00000000C000C0000000000040004000009A
:10CA9C00000000C000C0000000000040004000008A
:10CAAC00000000C000C0000000000040004000007A
:10CABC00000000C000C0000000000040004000006A
:10CACC00000000C000C0000000000040004000005A
:10CADC00000000C000C0000000000040004000004A
:10CAEC00000000C000C0000000000040004000003A
:10CAFC00000000C000C0000000000040004000002A
:10CB0C00000000C000C00000000000400040000019
:10CB1C00000000C000C00000000000400040000009
:10CB2C00000000C000C000000000004000400000F9
:10CB3C00000000C000C000000000004000400000E9
:10CB4C00000000C000C000000000004000400000D9
:10CB5C00000000C000C000000000004000400000C9
:10CB6C00000000C000C000000000004000400000B9
:10CB7C00000000C000C000000000004000400000A9
:10CB8C00000000C000C00000000000400040000099
:10CB9C00000000C000C00000000000400040000089
:10CBAC00000000C000C00000000000400040000079
:10CBBC00000000C000C00000000000400040000069
:10CBCC00000000C000C00000000000400040000059
:10CBDC00000000C000C00000000000400040000049
:10CBEC00000000C000C00000000000400040000039
:10CBFC00000000C000C00000000000400040000029
:10CC0C00000000C000C00000000000400040000018
:10CC1C00000000C000C00000000000400040000008
:10CC2C00000000C000C000000000004000400000F8
:10CC3C00000000C000C000000000004000400000E8
:10CC4C00000000C000C000000000004000400000D8
:10CC5C00000000C000C000000000004000400000C8
:10CC6C00000000C000C000000000004000400000B8
:10CC7C00000000C000C000000000004000400000A8
:10CC8C00000000C000C00000000000400040000098
:10CC9C00000000C000C00000000000400040000088
:10CCAC00000000C000C00000000000400040000078
:10CCBC00000000C000C00000000000400040000068
:10CCCC00000000C000C00000000000400040000058
:10CCDC00000000C000C00000000000400040000048
:10CCEC00000000C000C00000000000400040000038
:10CCFC00000000C000C00000000000400040000028
:10CD0C00000000C000C00000000000400040000017
:10CD1C00000000C000C00000000000400040000007
:10CD2C00000000C000C000000000004000400000F7
:10CD3C00000000C000C000000000004000400000E7
:10CD4C00000000C000C000000000004000400000D7
:10CD5C00000000C000C000000000004000400000C7
:10CD6C00000000C000C000000000004000400000B7
:10CD7C00000000C000C000000000004000400000A7
:10CD8C00000000C000C00000000000400040000097
:10CD9C00000000C000C00000000000400040000087
:10CDAC00000000C000C00000000000400040000077
:10CDBC00000000C000C00000000000400040000067
:10CDCC00000000C000C00000000000400040000057
:10CDDC00000000C000C00000000000400040000047
:10CDEC00000000C000C00000000000400040000037
:10CDFC00000000C000C00000000000400040000027
:10CE0C00000000C000C00000000000400040000016
:10CE1C00000000C000C00000000000400040000006
:10CE2C00000000C000C000000000004000400000F6
:10CE3C00000000C000C000000000004000400000E6
:10CE4C00000000C000C000000000004000400000D6
:10CE5C00000000C000C000000000004000400000C6
:10CE6C00000000C000C000000000004000400000B6
:10CE7C00000000C000C000000000004000400000A6
:10CE8C00000000C000C00000000000400040000096
:10CE9C00000000C000C00000000000400040000086
:10CEAC00000000C000C00000000000400040000076
:10CEBC00000000C000C00000000000400040000066
:10CECC00000000C000C00000000000400040000056
:10CEDC00000000C000C00000000000400040000046
:10CEEC00000000C000C00000000000400040000036
:10CEFC00000000C000C00000000000400040000026
:10CF0C00000000C000C00000000000400040000015
:10CF1C00000000C000C00000000000400040000005
:10CF2C00000000C000C000000000004000400000F5
:10CF3C00000000C000C000000000004000400000E5
:10CF4C00000000C000C000000000004000400000D5
:10CF5C00000000C000C000000000004000400000C5
:10CF6C00000000C000C000000000004000400000B5
:10CF7C00000000C000C000000000004000400000A5
:10CF8C00000000C000C00000000000400040000095
:10CF9C00000000C000C00000000000400040000085
:10CFAC00000000C000C00000000000400040000075
:10CFBC00000000C000C00000000000400040000065
:10CFCC00000000C000C00000000000400040000055
:10CFDC00000000C000C00000000000400040000045
:10CFEC00000000C000C00000000000400040000035
:10CFFC00000000C000C00000000000400040000025
:10D00C00000000C000C00000000000400040000014
:10D01C00000000C000C00000000000400040000004
:10D02C00000000C000C000000000004000400000F4
:10D03C00000000C000C000000000004000400000E4
:10D04C00000000C000C000000000004000400000D4
:10D05C00000000C000C0000000000040C53C1314DC
:10D06C001F2699CC26DBADCBC2C294126EFEFB3FC1
:10D07C00423C8F155F278CCD72DCCACA52C211118B
:10D08C00DDFCEC3FB63B0817992887CEC3DDEEC913
:10D09C00ECC18C0F4BFBD33F203B7D18CD298ACFA5
:10D0AC0019DF1BC98FC1050EBBF9B13F823AEF19CD
:10D0BC00FA2A95D075E051C83BC17C0C2BF8843F03
:10D0CC00DA395D1B212CA6D1D5E18FC7F2C0F10A4C
:10D0DC009CF64E3F2A39C61C412DBFD23AE3D6C628
:10D0EC00B2C064090FF50E3F71382B1E5A2EDFD3D8
:10D0FC00A3E426C67CC0D50784F3C53EAF378B1F8F
:10D10C006B2F06D511E67EC54FC04506FBF1713E6F
:10D11C00E536E720763033D683E7E0C42DC0B5047E
:10D12C0074F0143E12363D22793167D7F8E84AC4C0
:10D13C0014C02303EFEEAE3D36358E237432A1D8E6
:10D14C0071EABEC305C092016CED3E3D5334DA2446
:10D15C006733E1D9EDEB3BC300C00000EDEBC53C00
:10D16C0067331F26533426DB6CEDC2C205C06EFE3E
:10D17C0071EA423C74325F27363572DCEFEE52C2F4
:10D18C0014C0DDFCF8E8B63B793199281236C3DDC2
:10D19C0074F0ECC12DC04BFB83E7203B7630CD29DE
:10D1AC00E53619DFFBF18FC14FC0BBF911E6823AAE
:10D1BC006B2FFA2AAF3775E084F33BC17CC02BF898
:10D1CC00A3E4DA395A2E212C7138D5E10FF5F2C0CF
:10D1DC00B2C09CF63AE32A39412D412D2A393AE363
:10D1EC009CF6B2C0F2C00FF5D5E17138212C5A2E45
:10D1FC00DA39A3E42BF87CC03BC184F375E0AF377C
:10D20C00FA2A6B2F823A11E6BBF94FC08FC1FBF1A2
:10D21C0019DFE536CD297630203B83E74BFB2DC05B
:10D22C00ECC174F0C3DD123699287931B63BF8E8BD
:10D23C00DDFC14C052C2EFEE72DC36355F2774325F
:10D24C00423C71EA6EFE05C0C2C26CED26DB533463
:10D25C001F266733C53CEDEB000000C03BC3EDEB74
:10D26C00E1D96733DA2453343E3D6CED920105C0AD
:10D27C00BEC371EAA1D874328E233635AE3DEFEEC3
:10D28C00230314C04AC4F8E867D779313D2212361B
:10D29C00143E74F0B5042DC0E0C483E733D6763069
:10D2AC00E720E536713EFBF145064FC07EC511E621
:10D2BC0006D56B2F8B1FAF37C53E84F3D5077CC0CB
:10D2CC0026C6A3E4DFD35A2E2B1E71380E3F0FF562
:10D2DC006409B2C0D6C63AE3BFD2412DC61C2A3966
:10D2EC004E3F9CF6F10AF2C08FC7D5E1A6D1212C96
:10D2FC005D1BDA39843F2BF87C0C3BC151C875E0BF
:10D30C0095D0FA2AEF19823AB13FBBF9050E8FC1BD
:10D31C001BC919DF8ACFCD297D18203BD33F4BFB8E
:10D32C008C0FECC1EEC9C3DD87CE99280817B63B2C
:10D33C00EC3FDDFC111152C2CACA72DC8CCD5F27E6
:10D34C008F15423CFB3F6EFE9412C2C2ADCB26DB66
:10D35C0099CC1F261314C53C0040000013143BC38A
:10D36C0099CCE1D9ADCBDA2494123E3DFB3F92012E
:10D37C008F15BEC38CCDA1D8CACA8E231111AE3D58
:10D38C00EC3F230308174AC487CE67D7EEC93D226A
:10D39C008C0F143ED33FB5047D18E0C48ACF33D62E
:10D3AC001BC9E720050E713EB13F4506EF197EC53E
:10D3BC0095D006D551C88B1F7C0CC53E843FD50734
:10D3CC005D1B26C6A6D1DFD38FC72B1EF10A0E3FDD
:10D3DC004E3F6409C61CD6C6BFD2BFD2D6C6C61C29
:10D3EC0064094E3F0E3FF10A2B1E8FC7DFD3A6D127
:10D3FC0026C65D1BD507843FC53E7C0C8B1F51C8D0
:10D40C0006D595D07EC5EF194506B13F713E050E88
:10D41C00E7201BC933D68ACFE0C47D18B504D33FAF
:10D42C00143E8C0F3D22EEC967D787CE4AC408172D
:10D43C002303EC3FAE3D11118E23CACAA1D88CCD6B
:10D44C00BEC38F159201FB3F3E3D9412DA24ADCB47
:10D45C00E1D999CC3BC3131400000040C53C131414
:10D46C001F2699CC26DBADCBC2C294126EFEFB3FBD
:10D47C00423C8F155F278CCD72DCCACA52C2111187
:10D48C00DDFCEC3FB63B0817992887CEC3DDEEC90F
:10D49C00ECC18C0F4BFBD33F203B7D18CD298ACFA1
:10D4AC0019DF1BC98FC1050EBBF9B13F823AEF19C9
:10D4BC00FA2A95D075E051C83BC17C0C2BF8843FFF
:10D4CC00DA395D1B212CA6D1D5E18FC7F2C0F10A48
:10D4DC009CF64E3F2A39C61C412DBFD23AE3D6C624
:10D4EC00B2C064090FF50E3F71382B1E5A2EDFD3D4
:10D4FC00A3E426C67CC0D50784F3C53EAF378B1F8B
:10D50C006B2F06D511E67EC54FC04506FBF1713E6B
:10D51C00E536E720763033D683E7E0C42DC0B5047A
:10D52C0074F0143E12363D22793167D7F8E84AC4BC
:10D53C0014C02303EFEEAE3D36358E237432A1D8E2
:10D54C0071EABEC305C092016CED3E3D5334DA2442
:10D55C006733E1D9EDEB3BC300C00000EDEBC53CFC
:10D56C0067331F26533426DB6CEDC2C205C06EFE3A
:10D57C0071EA423C74325F27363572DCEFEE52C2F0
:10D58C0014C0DDFCF8E8B63B793199281236C3DDBE
:10D59C0074F0ECC12DC04BFB83E7203B7630CD29DA
:10D5AC00E53619DFFBF18FC14FC0BBF911E6823AAA
:10D5BC006B2FFA2AAF3775E084F33BC17CC02BF894
:10D5CC00A3E4DA395A2E212C7138D5E10FF5F2C0CB
:10D5DC00B2C09CF63AE32A39412D412D2A393AE35F
:10D5EC009CF6B2C0F2C00FF5D5E17138212C5A2E41
:10D5FC00DA39A3E42BF87CC03BC184F375E0AF3778
:10D60C00FA2A6B2F823A11E6BBF94FC08FC1FBF19E
:10D61C0019DFE536CD297630203B83E74BFB2DC057
:10D62C00ECC174F0C3DD123699287931B63BF8E8B9
:10D63C00DDFC14C052C2EFEE72DC36355F2774325B
:10D64C00423C71EA6EFE05C0C2C26CED26DB53345F
:10D65C001F266733C53CEDEB000000C03BC3EDEB70
:10D66C00E1D96733DA2453343E3D6CED920105C0A9
:10D67C00BEC371EAA1D874328E233635AE3DEFEEBF
:10D68C00230314C04AC4F8E867D779313D22123617
:10D69C00143E74F0B5042DC0E0C483E733D6763065
:10D6AC00E720E536713EFBF145064FC07EC511E61D
:10D6BC0006D56B2F8B1FAF37C53E84F3D5077CC0C7
:10D6CC0026C6A3E4DFD35A2E2B1E71380E3F0FF55E
:10D6DC006409B2C0D6C63AE3BFD2412DC61C2A3962
:10D6EC004E3F9CF6F10AF2C08FC7D5E1A6D1212C92
:10D6FC005D1BDA39843F2BF87C0C3BC151C875E0BB
:10D70C0095D0FA2AEF19823AB13FBBF9050E8FC1B9
:10D71C001BC919DF8ACFCD297D18203BD33F4BFB8A
:10D72C008C0FECC1EEC9C3DD87CE99280817B63B28
:10D73C00EC3FDDFC111152C2CACA72DC8CCD5F27E2
:10D74C008F15423CFB3F6EFE9412C2C2ADCB26DB62
:10D75C0099CC1F261314C53C0040000013143BC386
:10D76C0099CCE1D9ADCBDA2494123E3DFB3F92012A
:10D77C008F15BEC38CCDA1D8CACA8E231111AE3D54
:10D78C00EC3F230308174AC487CE67D7EEC93D2266
:10D79C008C0F143ED33FB5047D18E0C48ACF33D62A
:10D7AC001BC9E720050E713EB13F4506EF197EC53A
:10D7BC0095D006D551C88B1F7C0CC53E843FD50730
:10D7CC005D1B26C6A6D1DFD38FC72B1EF10A0E3FD9
:10D7DC004E3F6409C61CD6C6BFD2BFD2D6C6C61C25
:10D7EC0064094E3F0E3FF10A2B1E8FC7DFD3A6D123
:10D7FC0026C65D1BD507843FC53E7C0C8B1F51C8CC
:10D80C0006D595D07EC5EF194506B13F713E050E84
:10D81C00E7201BC933D68ACFE0C47D18B504D33FAB
:10D82C00143E8C0F3D22EEC967D787CE4AC4081729
:10D83C002303EC3FAE3D11118E23CACAA1D88CCD67
:10D84C00BEC38F159201FB3F3E3D9412DA24ADCB43
:10D85C00E1D999CC3BC3131400000040D33FB5046D
:10D86C006409B2C08FC1FBF16CED3E3DB63B0817AD
:10D87C005D1B26C651C875E072DC363574325F27E5
:10D88C00FA2A95D0DFD3A6D187CE9928DA2453343F
:10D89C00E53619DF3AE3D6C6E0C47D181314C53C4F
:10D8AC00143E74F00FF5F2C04FC045069201FB3FD9
:10D8BC00EC3F2303D5077CC03BC184F3EFEEAE3DB8
:10D8CC00423C8F15EF197EC58FC7D5E1C3DD1236EB
:10D8DC0067331F26CD298ACFBFD2BFD28ACFCD299D
:10D8EC001F2667331236C3DDD5E18FC77EC5EF190E
:10D8FC008F15423CAE3DEFEE84F33BC17CC0D507A7
:10D90C002303EC3FFB3F920145064FC0F2C00FF5DD
:10D91C0074F0143EC53C13147D18E0C4D6C63AE32B
:10D92C0019DFE5365334DA24992887CEA6D1DFD314
:10D93C0095D0FA2A5F277432363572DC75E051C8FF
:10D94C0026C65D1B0817B63B3E3D6CEDFBF18FC147
:10D95C00B2C06409B504D33F00400000B5042DC02B
:10D96C00B2C09CF6FBF1713E3E3D941208174AC4BE
:10D97C0026C6A3E475E0AF3736358E235F278CCDF2
:10D98C0095D006D5A6D1212C99287931533426DB94
:10D99C0019DF1BC9D6C6C61C7D18203BC53CEDEB58
:10D9AC0074F0ECC1F2C0F10A4506B13FFB3F6EFECC
:10D9BC00230314C07CC02BF884F3C53EAE3D11117B
:10D9CC008F15BEC37EC511E6D5E1713812363D22E6
:10D9DC001F2699CC8ACF33D6BFD2412DCD29763094
:10D9EC006733E1D9C3DDEEC98FC72B1EEF19823A1D
:10D9FC00423C71EAEFEE52C23BC17C0CD507843F2E
:10DA0C00EC3FDDFC920105C04FC0BBF90FF50E3F9A
:10DA1C00143E8C0F13143BC3E0C483E73AE32A395A
:10DA2C00E536E720DA24ADCB87CE67D7DFD35A2E85
:10DA3C00FA2A6B2F7432A1D872DCCACA51C88B1F58
:10DA4C005D1BDA39B63BF8E86CEDC2C28FC1050E2E
:10DA5C0064094E3FD33F4BFB000000C02DC04BFB75
:10DA6C009CF64E3F713E050E9412C2C24AC4F8E8B1
:10DA7C00A3E4DA39AF378B1F8E23CACA8CCDA1D859
:10DA8C0006D56B2F212C5A2E793167D726DBADCBDF
:10DA9C001BC9E720C61C2A39203B83E7EDEB3BC3AF
:10DAAC00ECC18C0FF10A0E3FB13FBBF96EFE05C005
:10DABC0014C0DDFC2BF8843FC53E7C0C111152C206
:10DACC00BEC371EA11E6823A71382B1E3D22EEC9B3
:10DADC0099CCE1D933D67630412D412D763033D6E1
:10DAEC00E1D999CCEEC93D222B1E7138823A11E650
:10DAFC0071EABEC352C211117C0CC53E843F2BF897
:10DB0C00DDFC14C005C06EFEBBF9B13F0E3FF10A3F
:10DB1C008C0FECC13BC3EDEB83E7203B2A39C61CD1
:10DB2C00E7201BC9ADCB26DB67D779315A2E212CC8
:10DB3C006B2F06D5A1D88CCDCACA8E238B1FAF37BD
:10DB4C00DA39A3E4F8E84AC4C2C29412050E713E55
:10DB5C004E3F9CF64BFB2DC000C000004BFBD33F4F
:10DB6C004E3F6409050E8FC1C2C26CEDF8E8B63B9E
:10DB7C00DA395D1B8B1F51C8CACA72DCA1D874324A
:10DB8C006B2FFA2A5A2EDFD367D787CEADCBDA2488
:10DB9C00E720E5362A393AE383E7E0C43BC31314A4
:10DBAC008C0F143E0E3F0FF5BBF94FC005C0920110
:10DBBC00DDFCEC3F843FD5077C0C3BC152C2EFEE41
:10DBCC0071EA423C823AEF192B1E8FC7EEC9C3DDB6
:10DBDC00E1D967337630CD29412DBFD233D68ACFE8
:10DBEC0099CC1F263D2212367138D5E111E67EC53F
:10DBFC00BEC38F151111AE3DC53E84F32BF87CC00E
:10DC0C0014C023036EFEFB3FB13F4506F10AF2C080
:10DC1C00ECC174F0EDEBC53C203B7D18C61CD6C6A0
:10DC2C001BC919DF26DB533479319928212CA6D155
:10DC3C0006D595D08CCD5F278E233635AF3775E062
:10DC4C00A3E426C64AC4081794123E3D713EFBF16C
:10DC5C009CF6B2C02DC0B50400000040D33FB50403
:10DC6C006409B2C08FC1FBF16CED3E3DB63B0817A9
:10DC7C005D1B26C651C875E072DC363574325F27E1
:10DC8C00FA2A95D0DFD3A6D187CE9928DA2453343B
:10DC9C00E53619DF3AE3D6C6E0C47D181314C53C4B
:10DCAC00143E74F00FF5F2C04FC045069201FB3FD5
:10DCBC00EC3F2303D5077CC03BC184F3EFEEAE3DB4
:10DCCC00423C8F15EF197EC58FC7D5E1C3DD1236E7
:10DCDC0067331F26CD298ACFBFD2BFD28ACFCD2999
:10DCEC001F2667331236C3DDD5E18FC77EC5EF190A
:10DCFC008F15423CAE3DEFEE84F33BC17CC0D507A3
:10DD0C002303EC3FFB3F920145064FC0F2C00FF5D9
:10DD1C0074F0143EC53C13147D18E0C4D6C63AE327
:10DD2C0019DFE5365334DA24992887CEA6D1DFD310
:10DD3C0095D0FA2A5F277432363572DC75E051C8FB
:10DD4C0026C65D1B0817B63B3E3D6CEDFBF18FC143
:10DD5C00B2C06409B504D33F00400000B5042DC027
:10DD6C00B2C09CF6FBF1713E3E3D941208174AC4BA
:10DD7C0026C6A3E475E0AF3736358E235F278CCDEE
:10DD8C0095D006D5A6D1212C99287931533426DB90
:10DD9C0019DF1BC9D6C6C61C7D18203BC53CEDEB54
:10DDAC0074F0ECC1F2C0F10A4506B13FFB3F6EFEC8
:10DDBC00230314C07CC02BF884F3C53EAE3D111177
:10DDCC008F15BEC37EC511E6D5E1713812363D22E2
:10DDDC001F2699CC8ACF33D6BFD2412DCD29763090
:10DDEC006733E1D9C3DDEEC98FC72B1EEF19823A19
:10DDFC00423C71EAEFEE52C23BC17C0CD507843F2A
:10DE0C00EC3FDDFC920105C04FC0BBF90FF50E3F96
:10DE1C00143E8C0F13143BC3E0C483E73AE32A3956
:10DE2C00E536E720DA24ADCB87CE67D7DFD35A2E81
:10DE3C00FA2A6B2F7432A1D872DCCACA51C88B1F54
:10DE4C005D1BDA39B63BF8E86CEDC2C28FC1050E2A
:10DE5C0064094E3FD33F4BFB000000C02DC04BFB71
:10DE6C009CF64E3F713E050E9412C2C24AC4F8E8AD
:10DE7C00A3E4DA39AF378B1F8E23CACA8CCDA1D855
:10DE8C0006D56B2F212C5A2E793167D726DBADCBDB
:10DE9C001BC9E720C61C2A39203B83E7EDEB3BC3AB
:10DEAC00ECC18C0FF10A0E3FB13FBBF96EFE05C001
:10DEBC0014C0DDFC2BF8843FC53E7C0C111152C202
:10DECC00BEC371EA11E6823A71382B1E3D22EEC9AF
:10DEDC0099CCE1D933D67630412D412D763033D6DD
:10DEEC00E1D999CCEEC93D222B1E7138823A11E64C
:10DEFC0071EABEC352C211117C0CC53E843F2BF893
:10DF0C00DDFC14C005C06EFEBBF9B13F0E3FF10A3B
:10DF1C008C0FECC13BC3EDEB83E7203B2A39C61CCD
:10DF2C00E7201BC9ADCB26DB67D779315A2E212CC4
:10DF3C006B2F06D5A1D88CCDCACA8E238B1FAF37B9
:10DF4C00DA39A3E4F8E84AC4C2C29412050E713E51
:10DF5C004E3F9CF64BFB2DC000C000004BFBD33F4B
:10DF6C004E3F6409050E8FC1C2C26CEDF8E8B63B9A
:10DF7C00DA395D1B8B1F51C8CACA72DCA1D8743246
:10DF8C006B2FFA2A5A2EDFD367D787CEADCBDA2484
:10DF9C00E720E5362A393AE383E7E0C43BC31314A0
:10DFAC008C0F143E0E3F0FF5BBF94FC005C092010C
:10DFBC00DDFCEC3F843FD5077C0C3BC152C2EFEE3D
:10DFCC0071EA423C823AEF192B1E8FC7EEC9C3DDB2
:10DFDC00E1D967337630CD29412DBFD233D68ACFE4
:10DFEC0099CC1F263D2212367138D5E111E67EC53B
:10DFFC00BEC38F151111AE3DC53E84F32BF87CC00A
:10E00C0014C023036EFEFB3FB13F4506F10AF2C07C
:10E01C00ECC174F0EDEBC53C203B7D18C61CD6C69C
:10E02C001BC919DF26DB533479319928212CA6D151
:10E03C0006D595D08CCD5F278E233635AF3775E05E
:10E04C00A3E426C64AC4081794123E3D713EFBF168
:10E05C009CF6B2C02DC0B50400000040C53E7C0C3F
:10E06C007D18E0C4CACA72DCBFD2412D8E2336356E
:10E07C00203B83E784F33BC100C0000084F3C53E22
:10E08C00203B7D188E23CACABFD2BFD2CACA8E23E8
:10E09C007D18203BC53E84F3000000C03BC184F3D7
:10E0AC0083E7203B36358E23412DBFD272DCCACAA2
:10E0BC00E0C47D187C0CC53E004000007C0C3BC1CC
:10E0CC00E0C483E772DC3635412D412D363572DCE8
:10E0DC0083E7E0C43BC17C0C00000040C53E7C0CD7
:10E0EC007D18E0C4CACA72DCBFD2412D8E233635EE
:10E0FC00203B83E784F33BC100C0000084F3C53EA2
:10E10C00203B7D188E23CACABFD2BFD2CACA8E2367
:10E11C007D18203BC53E84F3000000C03BC184F356
:10E12C0083E7203B36358E23412DBFD272DCCACA21
:10E13C00E0C47D187C0CC53E004000007C0C3BC14B
:10E14C00E0C483E772DC3635412D412D363572DC67
:10E15C0083E7E0C43BC17C0C00000040C53E7C0C56
:10E16C007D18E0C4CACA72DCBFD2412D8E2336356D
:10E17C00203B83E784F33BC100C0000084F3C53E21
:10E18C00203B7D188E23CACABFD2BFD2CACA8E23E7
:10E19C007D18203BC53E84F3000000C03BC184F3D6
:10E1AC0083E7203B36358E23412DBFD272DCCACAA1
:10E1BC00E0C47D187C0CC53E004000007C0C3BC1CB
:10E1CC00E0C483E772DC3635412D412D363572DCE7
:10E1DC0083E7E0C43BC17C0C00000040C53E7C0CD6
:10E1EC007D18E0C4CACA72DCBFD2412D8E233635ED
:10E1FC00203B83E784F33BC100C0000084F3C53EA1
:10E20C00203B7D188E23CACABFD2BFD2CACA8E2366
:10E21C007D18203BC53E84F3000000C03BC184F355
:10E22C0083E7203B36358E23412DBFD272DCCACA20
:10E23C00E0C47D187C0CC53E004000007C0C3BC14A
:10E24C00E0C483E772DC3635412D412D363572DC66
:10E25C0083E7E0C43BC17C0C00000040C53E7C0C55
:10E26C007D18E0C4CACA72DCBFD2412D8E2336356C
:10E27C00203B83E784F33BC100C0000084F3C53E20
:10E28C00203B7D188E23CACABFD2BFD2CACA8E23E6
:10E29C007D18203BC53E84F3000000C03BC184F3D5
:10E2AC0083E7203B36358E23412DBFD272DCCACAA0
:10E2BC00E0C47D187C0CC53E004000007C0C3BC1CA
:10E2CC00E0C483E772DC3635412D412D363572DCE6
:10E2DC0083E7E0C43BC17C0C00000040C53E7C0CD5
:10E2EC007D18E0C4CACA72DCBFD2412D8E233635EC
:10E2FC00203B83E784F33BC100C0000084F3C53EA0
:10E30C00203B7D188E23CACABFD2BFD2CACA8E2365
:10E31C007D18203BC53E84F3000000C03BC184F354
:10E32C0083E7203B36358E23412DBFD272DCCACA1F
:10E33C00E0C47D187C0CC53E004000007C0C3BC149
:10E34C00E0C483E772DC3635412D412D363572DC65
:10E35C0083E7E0C43BC17C0C00000040C53E7C0C54
:10E36C007D18E0C4CACA72DCBFD2412D8E2336356B
:10E37C00203B83E784F33BC100C0000084F3C53E1F
:10E38C00203B7D188E23CACABFD2BFD2CACA8E23E5
:10E39C007D18203BC53E84F3000000C03BC184F3D4
:10E3AC0083E7203B36358E23412DBFD272DCCACA9F
:10E3BC00E0C47D187C0CC53E004000007C0C3BC1C9
:10E3CC00E0C483E772DC3635412D412D363572DCE5
:10E3DC0083E7E0C43BC17C0C00000040C53E7C0CD4
:10E3EC007D18E0C4CACA72DCBFD2412D8E233635EB
:10E3FC00203B83E784F33BC100C0000084F3C53E9F
:10E40C00203B7D188E23CACABFD2BFD2CACA8E2364
:10E41C007D18203BC53E84F3000000C03BC184F353
:10E42C0083E7203B36358E23412DBFD272DCCACA1E
:10E43C00E0C47D187C0CC53E004000007C0C3BC148
:10E44C00E0C483E772DC3635412D412D363572DC64
:10E45C0083E7E0C43BC17C0C00000040C53E7C0C53
:10E46C007D18E0C4CACA72DCBFD2412D8E2336356A
:10E47C00203B83E784F33BC100C0000084F3C53E1E
:10E48C00203B7D188E23CACABFD2BFD2CACA8E23E4
:10E49C007D18203BC53E84F3000000C03BC184F3D3
:10E4AC0083E7203B36358E23412DBFD272DCCACA9E
:10E4BC00E0C47D187C0CC53E004000007C0C3BC1C8
:10E4CC00E0C483E772DC3635412D412D363572DCE4
:10E4DC0083E7E0C43BC17C0C00000040C53E7C0CD3
:10E4EC007D18E0C4CACA72DCBFD2412D8E233635EA
:10E4FC00203B83E784F33BC100C0000084F3C53E9E
:10E50C00203B7D188E23CACABFD2BFD2CACA8E2363
:10E51C007D18203BC53E84F3000000C03BC184F352
:10E52C0083E7203B36358E23412DBFD272DCCACA1D
:10E53C00E0C47D187C0CC53E004000007C0C3BC147
:10E54C00E0C483E772DC3635412D412D363572DC63
:10E55C0083E7E0C43BC17C0C00000040C53E7C0C52
:10E56C007D18E0C4CACA72DCBFD2412D8E23363569
:10E57C00203B83E784F33BC100C0000084F3C53E1D
:10E58C00203B7D188E23CACABFD2BFD2CACA8E23E3
:10E59C007D18203BC53E84F3000000C03BC184F3D2
:10E5AC0083E7203B36358E23412DBFD272DCCACA9D
:10E5BC00E0C47D187C0CC53E004000007C0C3BC1C7
:10E5CC00E0C483E772DC3635412D412D363572DCE3
:10E5DC0083E7E0C43BC17C0C00000040C53E7C0CD2
:10E5EC007D18E0C4CACA72DCBFD2412D8E233635E9
:10E5FC00203B83E784F33BC100C0000084F3C53E9D
:10E60C00203B7D188E23CACABFD2BFD2CACA8E2362
:10E61C007D18203BC53E84F3000000C03BC184F351
:10E62C0083E7203B36358E23412DBFD272DCCACA1C
:10E63C00E0C47D187C0CC53E004000007C0C3BC146
:10E64C00E0C483E772DC3635412D412D363572DC62
:10E65C0083E7E0C43BC17C0C00000040C53E7C0C51
:10E66C007D18E0C4CACA72DCBFD2412D8E23363568
:10E67C00203B83E784F33BC100C0000084F3C53E1C
:10E68C00203B7D188E23CACABFD2BFD2CACA8E23E2
:10E69C007D18203BC53E84F3000000C03BC184F3D1
:10E6AC0083E7203B36358E23412DBFD272DCCACA9C
:10E6BC00E0C47D187C0CC53E004000007C0C3BC1C6
:10E6CC00E0C483E772DC3635412D412D363572DCE2
:10E6DC0083E7E0C43BC17C0C00000040C53E7C0CD1
:10E6EC007D18E0C4CACA72DCBFD2412D8E233635E8
:10E6FC00203B83E784F33BC100C0000084F3C53E9C
:10E70C00203B7D188E23CACABFD2BFD2CACA8E2361
:10E71C007D18203BC53E84F3000000C03BC184F350
:10E72C0083E7203B36358E23412DBFD272DCCACA1B
:10E73C00E0C47D187C0CC53E004000007C0C3BC145
:10E74C00E0C483E772DC3635412D412D363572DC61
:10E75C0083E7E0C43BC17C0C00000040C53E7C0C50
:10E76C007D18E0C4CACA72DCBFD2412D8E23363567
:10E77C00203B83E784F33BC100C0000084F3C53E1B
:10E78C00203B7D188E23CACABFD2BFD2CACA8E23E1
:10E79C007D18203BC53E84F3000000C03BC184F3D0
:10E7AC0083E7203B36358E23412DBFD272DCCACA9B
:10E7BC00E0C47D187C0CC53E004000007C0C3BC1C5
:10E7CC00E0C483E772DC3635412D412D363572DCE1
:10E7DC0083E7E0C43BC17C0C00000040C53E7C0CD0
:10E7EC007D18E0C4CACA72DCBFD2412D8E233635E7
:10E7FC00203B83E784F33BC100C0000084F3C53E9B
:10E80C00203B7D188E23CACABFD2BFD2CACA8E2360
:10E81C007D18203BC53E84F3000000C03BC184F34F
:10E82C0083E7203B36358E23412DBFD272DCCACA1A
:10E83C00E0C47D187C0CC53E004000007C0C3BC144
:10E84C00E0C483E772DC3635412D412D363572DC60
:10E85C0083E7E0C43BC17C0C6C090108700901081A
:10E86C008439020864A8000884310208842902084B
:10E87C0064B800085401010854F900088421020806
:10E88C008419020864C00008841102088409020873
:10E89C008401020884F9010864B0000884F10108BD
:10E8AC0084E9010884E1010884D9010864D00008D6
:10E8BC0084D1010884C9010884C1010884B9010804
:10E8CC0064E0000884B1010884A9010884A101084E
:10E8DC008499010864D8000884910108848901088E
:10E8EC0064C80008848101088479010884710108D6
:10E8FC008469010884610108845901088451010864
:10E90C0084490108844101088439010884310108D3
:10E91C008429010884210108841901088411010843
:10E92C008409010800000040000000C00000004005
:10E93C00000000C000000040000000C000000040CB
:10E94C00000000C000000040000000C000000040BB
:10E95C00000000C000000040000000C000000040AB
:10E96C00000000C000000040000000C0000000409B
:10E97C00000000C000000040000000C0000000408B
:10E98C00000000C000000040000000C0000000407B
:10E99C00000000C000000040000000C0000000406B
:10E9AC00000000C000000040000000C0000000405B
:10E9BC00000000C000000040000000C0000000404B
:10E9CC00000000C000000040000000C0000000403B
:10E9DC00000000C000000040000000C0000000402B
:10E9EC00000000C000000040000000C0000000401B
:10E9FC00000000C000000040000000C0000000400B
:10EA0C00000000C000000040000000C000000040FA
:10EA1C00000000C000000040000000C000000040EA
:10EA2C00000000C000000040000000C000000040DA
:10EA3C00000000C000000040000000C000000040CA
:10EA4C00000000C000000040000000C000000040BA
:10EA5C00000000C000000040000000C000000040AA
:10EA6C00000000C000000040000000C0000000409A
:10EA7C00000000C000000040000000C0000000408A
:10EA8C00000000C000000040000000C0000000407A
:10EA9C00000000C000000040000000C0000000406A
:10EAAC00000000C000000040000000C0000000405A
:10EABC00000000C000000040000000C0000000404A
:10EACC00000000C000000040000000C0000000403A
:10EADC00000000C000000040000000C0000000402A
:10EAEC00000000C000000040000000C0000000401A
:10EAFC00000000C000000040000000C0000000400A
:10EB0C00000000C000000040000000C000000040F9
:10EB1C00000000C000000040000000C000000040E9
:10EB2C00000000C000000040000000C000000040D9
:10EB3C00000000C000000040000000C000000040C9
:10EB4C00000000C000000040000000C000000040B9
:10EB5C00000000C000000040000000C000000040A9
:10EB6C00000000C000000040000000C00000004099
:10EB7C00000000C000000040000000C00000004089
:10EB8C00000000C000000040000000C00000004079
:10EB9C00000000C000000040000000C00000004069
:10EBAC00000000C000000040000000C00000004059
:10EBBC00000000C000000040000000C00000004049
:10EBCC00000000C000000040000000C00000004039
:10EBDC00000000C000000040000000C00000004029
:10EBEC00000000C000000040000000C00000004019
:10EBFC00000000C000000040000000C00000004009
:10EC0C00000000C000000040000000C000000040F8
:10EC1C00000000C000000040000000C000000040E8
:10EC2C00000000C000000040000000C000000040D8
:10EC3C00000000C000000040000000C000000040C8
:10EC4C00000000C000000040000000C000000040B8
:10EC5C00000000C000000040000000C000000040A8
:10EC6C00000000C000000040000000C00000004098
:10EC7C00000000C000000040000000C00000004088
:10EC8C00000000C000000040000000C00000004078
:10EC9C00000000C000000040000000C00000004068
:10ECAC00000000C000000040000000C00000004058
:10ECBC00000000C000000040000000C00000004048
:10ECCC00000000C000000040000000C00000004038
:10ECDC00000000C000000040000000C00000004028
:10ECEC00000000C000000040000000C00000004018
:10ECFC00000000C000000040000000C00000004008
:10ED0C00000000C000000040000000C000000040F7
:10ED1C00000000C000000040000000C000000040E7
:10ED2C00000000C000005A2EEC3FCD29BBF98CCD61
:10ED3C00B2C026DB7C0C1236143E8B1F6CEDD6C693
:10ED4C00BEC311E67D18B63BDA391314D5E152C2B5
:10ED5C001BC9FBF18E230E3F6733D50767D72DC038
:10ED6C0095D06EFE412DFB3FFA2A4BFB87CE7CC023
:10ED7C00E1D9F10A3635713EE720EFEE8FC73BC380
:10ED8C00A3E40817203B823A8F153AE3C2C251C85C
:10ED9C0074F03D22C53E53346409A1D84FC08ACFCC
:10EDAC00DDFC212C0040212CDDFC8ACF4FC0A1D8EA
:10EDBC0064095334C53E3D2274F051C8C2C23AE3D3
:10EDCC008F15823A203B0817A3E43BC38FC7EFEEA5
:10EDDC00E720713E3635F10AE1D97CC087CE4BFB7A
:10EDEC00FA2AFB3F412D6EFE95D02DC067D7D50773
:10EDFC0067330E3F8E23FBF11BC952C2D5E11314AE
:10EE0C00DA39B63B7D1811E6BEC3D6C66CED8B1F46
:10EE1C00143E12367C0C26DBB2C08CCDBBF9CD294E
:10EE2C00EC3F5A2E0000A6D114C033D645067432DE
:10EE3C004E3FDA2484F3EEC9ECC175E094122A3902
:10EE4C00423CEF1983E74AC426C6EDEB2B1EAE3DC0
:10EE5C00E536050E72DCF2C099CC2BF89928D33F1D
:10EE6C006B2F9201BFD205C006D5B5047931843F12
:10EE7C001F260FF5CACA8FC119DF11117138C53C95
:10EE8C005D1BF8E8E0C47EC571EAC61C3E3DAF3799
:10EE9C008C0FC3DD3BC1ADCB9CF65F27B13F763009
:10EEAC002303DFD300C0DFD323037630B13F5F27CA
:10EEBC009CF6ADCB3BC1C3DD8C0FAF373E3DC61CC2
:10EECC0071EA7EC5E0C4F8E85D1BC53C71381111D0
:10EEDC0019DF8FC1CACA0FF51F26843F7931B504DB
:10EEEC0006D505C0BFD292016B2FD33F99282BF8C2
:10EEFC0099CCF2C072DC050EE536AE3D2B1EEDEB67
:10EF0C0026C64AC483E7EF19423C2A39941275E0AD
:10EF1C00ECC1EEC984F3DA244E3F7432450633D685
:10EF2C0014C0A6D100005A2EEC3FCD29BBF98CCDD4
:10EF3C00B2C026DB7C0C1236143E8B1F6CEDD6C691
:10EF4C00BEC311E67D18B63BDA391314D5E152C2B3
:10EF5C001BC9FBF18E230E3F6733D50767D72DC036
:10EF6C0095D06EFE412DFB3FFA2A4BFB87CE7CC021
:10EF7C00E1D9F10A3635713EE720EFEE8FC73BC37E
:10EF8C00A3E40817203B823A8F153AE3C2C251C85A
:10EF9C0074F03D22C53E53346409A1D84FC08ACFCA
:10EFAC00DDFC212C0040212CDDFC8ACF4FC0A1D8E8
:10EFBC0064095334C53E3D2274F051C8C2C23AE3D1
:10EFCC008F15823A203B0817A3E43BC38FC7EFEEA3
:10EFDC00E720713E3635F10AE1D97CC087CE4BFB78
:10EFEC00FA2AFB3F412D6EFE95D02DC067D7D50771
:10EFFC0067330E3F8E23FBF11BC952C2D5E11314AC
:10F00C00DA39B63B7D1811E6BEC3D6C66CED8B1F44
:10F01C00143E12367C0C26DBB2C08CCDBBF9CD294C
:10F02C00EC3F5A2E0000A6D114C033D645067432DC
:10F03C004E3FDA2484F3EEC9ECC175E094122A3900
:10F04C00423CEF1983E74AC426C6EDEB2B1EAE3DBE
:10F05C00E536050E72DCF2C099CC2BF89928D33F1B
:10F06C006B2F9201BFD205C006D5B5047931843F10
:10F07C001F260FF5CACA8FC119DF11117138C53C93
:10F08C005D1BF8E8E0C47EC571EAC61C3E3DAF3797
:10F09C008C0FC3DD3BC1ADCB9CF65F27B13F763007
:10F0AC002303DFD300C0DFD323037630B13F5F27C8
:10F0BC009CF6ADCB3BC1C3DD8C0FAF373E3DC61CC0
:10F0CC0071EA7EC5E0C4F8E85D1BC53C71381111CE
:10F0DC0019DF8FC1CACA0FF51F26843F7931B504D9
:10F0EC0006D505C0BFD292016B2FD33F99282BF8C0
:10F0FC0099CCF2C072DC050EE536AE3D2B1EEDEB65
:10F10C0026C64AC483E7EF19423C2A39941275E0AB
:10F11C00ECC1EEC984F3DA244E3F7432450633D683
:10F12C0014C0A6D10000DA39793174F03BC1E1D9B1
:10F13C002B1EEC3F7D1806D5C2C29CF63635E53643
:10F14C00BBF9BEC3BFD28F15B13FE72072DCB2C092
:10F15C006CED6B2F203B23038FC799CC7C0C143E9A
:10F16C009928A3E400C0A3E49928143E7C0C99CC04
:10F17C008FC72303203B6B2F6CEDB2C072DCE720F2
:10F18C00B13F8F15BFD2BEC3BBF9E53636359CF601
:10F19C00C2C206D57D18EC3F2B1EE1D93BC174F0E1
:10F1AC007931DA39000026C687CE8C0FC53E1F2672
:10F1BC00D5E114C083E7FA2A3E3D6409CACA1BC9CB
:10F1CC004506423C412D71EA4FC019DF8E234E3F5C
:10F1DC00941295D0E0C4DDFC7138673384F3ECC134
:10F1EC0067D75D1B00405D1B67D7ECC184F36733A9
:10F1FC007138DDFCE0C495D094124E3F8E2319DF9C
:10F20C004FC071EA412D423C45061BC9CACA64096C
:10F21C003E3DFA2A83E714C0D5E11F26C53E8C0F6C
:10F22C0087CE26C60000DA39793174F03BC1E1D9BA
:10F23C002B1EEC3F7D1806D5C2C29CF63635E53642
:10F24C00BBF9BEC3BFD28F15B13FE72072DCB2C091
:10F25C006CED6B2F203B23038FC799CC7C0C143E99
:10F26C009928A3E400C0A3E49928143E7C0C99CC03
:10F27C008FC72303203B6B2F6CEDB2C072DCE720F1
:10F28C00B13F8F15BFD2BEC3BBF9E53636359CF600
:10F29C00C2C206D57D18EC3F2B1EE1D93BC174F0E0
:10F2AC007931DA39000026C687CE8C0FC53E1F2671
:10F2BC00D5E114C083E7FA2A3E3D6409CACA1BC9CA
:10F2CC004506423C412D71EA4FC019DF8E234E3F5B
:10F2DC00941295D0E0C4DDFC7138673384F3ECC133
:10F2EC0067D75D1B00405D1B67D7ECC184F36733A8
:10F2FC007138DDFCE0C495D094124E3F8E2319DF9B
:10F30C004FC071EA412D423C45061BC9CACA64096B
:10F31C003E3DFA2A83E714C0D5E11F26C53E8C0F6B
:10F32C0087CE26C60000DA39793174F03BC1E1D9B9
:10F33C002B1EEC3F7D1806D5C2C29CF63635E53641
:10F34C00BBF9BEC3BFD28F15B13FE72072DCB2C090
:10F35C006CED6B2F203B23038FC799CC7C0C143E98
:10F36C009928A3E400C0A3E49928143E7C0C99CC02
:10F37C008FC72303203B6B2F6CEDB2C072DCE720F0
:10F38C00B13F8F15BFD2BEC3BBF9E53636359CF6FF
:10F39C00C2C206D57D18EC3F2B1EE1D93BC174F0DF
:10F3AC007931DA39000026C687CE8C0FC53E1F2670
:10F3BC00D5E114C083E7FA2A3E3D6409CACA1BC9C9
:10F3CC004506423C412D71EA4FC019DF8E234E3F5A
:10F3DC00941295D0E0C4DDFC7138673384F3ECC132
:10F3EC0067D75D1B00405D1B67D7ECC184F36733A7
:10F3FC007138DDFCE0C495D094124E3F8E2319DF9A
:10F40C004FC071EA412D423C45061BC9CACA64096A
:10F41C003E3DFA2A83E714C0D5E11F26C53E8C0F6A
:10F42C0087CE26C60000DA39793174F03BC1E1D9B8
:10F43C002B1EEC3F7D1806D5C2C29CF63635E53640
:10F44C00BBF9BEC3BFD28F15B13FE72072DCB2C08F
:10F45C006CED6B2F203B23038FC799CC7C0C143E97
:10F46C009928A3E400C0A3E49928143E7C0C99CC01
:10F47C008FC72303203B6B2F6CEDB2C072DCE720EF
:10F48C00B13F8F15BFD2BEC3BBF9E53636359CF6FE
:10F49C00C2C206D57D18EC3F2B1EE1D93BC174F0DE
:10F4AC007931DA39000026C687CE8C0FC53E1F266F
:10F4BC00D5E114C083E7FA2A3E3D6409CACA1BC9C8
:10F4CC004506423C412D71EA4FC019DF8E234E3F59
:10F4DC00941295D0E0C4DDFC7138673384F3ECC131
:10F4EC0067D75D1B00405D1B67D7ECC184F36733A6
:10F4FC007138DDFCE0C495D094124E3F8E2319DF99
:10F50C004FC071EA412D423C45061BC9CACA640969
:10F51C003E3DFA2A83E714C0D5E11F26C53E8C0F69
:10F52C0087CE26C60000C53C1F2626DBC2C26EFE57
:10F53C00423C5F2772DC52C2DDFCB63B9928C3DD2E
:10F54C00ECC14BFB203BCD2919DF8FC1BBF9823AB3
:10F55C00FA2A75E03BC12BF8DA39212CD5E1F2C03F
:10F56C009CF62A39412D3AE3B2C00FF571385A2E68
:10F57C00A3E47CC084F3AF376B2F11E64FC0FBF1D3
:10F58C00E536763083E72DC074F012367931F8E821
:10F59C0014C0EFEE3635743271EA05C06CED53349D
:10F5AC006733EDEB00C0EDEB673353346CED05C006
:10F5BC0071EA74323635EFEE14C0F8E87931123650
:10F5CC0074F02DC083E77630E536FBF14FC011E6C1
:10F5DC006B2FAF3784F37CC0A3E45A2E71380FF530
:10F5EC00B2C03AE3412D2A399CF6F2C0D5E1212C68
:10F5FC00DA392BF83BC175E0FA2A823ABBF98FC194
:10F60C0019DFCD29203B4BFBECC1C3DD9928B63B60
:10F61C00DDFC52C272DC5F27423C6EFEC2C226DBAE
:10F62C001F26C53C00003BC3E1D9DA243E3D9201C4
:10F63C00BEC3A1D88E23AE3D23034AC467D73D2257
:10F64C00143EB504E0C433D6E720713E45067EC5B2
:10F65C0006D58B1FC53ED50726C6DFD32B1E0E3F06
:10F66C006409D6C6BFD2C61C4E3FF10A8FC7A6D1BD
:10F67C005D1B843F7C0C51C895D0EF19B13F050E32
:10F68C001BC98ACF7D18D33F8C0FEEC987CE0817C4
:10F69C00EC3F1111CACA8CCD8F15FB3F9412ADCB28
:10F6AC0099CC13140040131499CCADCB9412FB3F9E
:10F6BC008F158CCDCACA1111EC3F081787CEEEC935
:10F6CC008C0FD33F7D188ACF1BC9050EB13FEF19A4
:10F6DC0095D051C87C0C843F5D1BA6D18FC7F10A15
:10F6EC004E3FC61CBFD2D6C664090E3F2B1EDFD3BD
:10F6FC0026C6D507C53E8B1F06D57EC54506713E71
:10F70C00E72033D6E0C4B504143E3D2267D74AC483
:10F71C002303AE3D8E23A1D8BEC392013E3DDA2415
:10F72C00E1D93BC30000C53C1F2626DBC2C26EFEDE
:10F73C00423C5F2772DC52C2DDFCB63B9928C3DD2C
:10F74C00ECC14BFB203BCD2919DF8FC1BBF9823AB1
:10F75C00FA2A75E03BC12BF8DA39212CD5E1F2C03D
:10F76C009CF62A39412D3AE3B2C00FF571385A2E66
:10F77C00A3E47CC084F3AF376B2F11E64FC0FBF1D1
:10F78C00E536763083E72DC074F012367931F8E81F
:10F79C0014C0EFEE3635743271EA05C06CED53349B
:10F7AC006733EDEB00C0EDEB673353346CED05C004
:10F7BC0071EA74323635EFEE14C0F8E8793112364E
:10F7CC0074F02DC083E77630E536FBF14FC011E6BF
:10F7DC006B2FAF3784F37CC0A3E45A2E71380FF52E
:10F7EC00B2C03AE3412D2A399CF6F2C0D5E1212C66
:10F7FC00DA392BF83BC175E0FA2A823ABBF98FC192
:10F80C0019DFCD29203B4BFBECC1C3DD9928B63B5E
:10F81C00DDFC52C272DC5F27423C6EFEC2C226DBAC
:10F82C001F26C53C00003BC3E1D9DA243E3D9201C2
:10F83C00BEC3A1D88E23AE3D23034AC467D73D2255
:10F84C00143EB504E0C433D6E720713E45067EC5B0
:10F85C0006D58B1FC53ED50726C6DFD32B1E0E3F04
:10F86C006409D6C6BFD2C61C4E3FF10A8FC7A6D1BB
:10F87C005D1B843F7C0C51C895D0EF19B13F050E30
:10F88C001BC98ACF7D18D33F8C0FEEC987CE0817C2
:10F89C00EC3F1111CACA8CCD8F15FB3F9412ADCB26
:10F8AC0099CC13140040131499CCADCB9412FB3F9C
:10F8BC008F158CCDCACA1111EC3F081787CEEEC933
:10F8CC008C0FD33F7D188ACF1BC9050EB13FEF19A2
:10F8DC0095D051C87C0C843F5D1BA6D18FC7F10A13
:10F8EC004E3FC61CBFD2D6C664090E3F2B1EDFD3BB
:10F8FC0026C6D507C53E8B1F06D57EC54506713E6F
:10F90C00E72033D6E0C4B504143E3D2267D74AC481
:10F91C002303AE3D8E23A1D8BEC392013E3DDA2413
:10F92C00E1D93BC301000001540901086009010839
:10F93C0000030102010301000203020001000201A5
:10F94C0000020100020100020000004067331F2684
:10F95C003E3D6CED8F15BEC372DCCACA14C0DDFC13
:10F96C0067D779318C0F143E203B7D18E53619DFB3
:10F97C0045064FC095D006D53BC17C0CA3E4DA39C3
:10F98C002B1E71384E3F6409412DBFD29CF6B2C07C
:10F99C008FC7D5E126C65D1B84F3C53EFA2A6B2FB3
:10F9AC00B13FBBF9E7201BC983E7E0C4ECC174F09D
:10F9BC0087CE99282303EC3F36358E23423C71EADF
:10F9CC009412C2C2E1D999CC00C00000E1D96733CE
:10F9DC0094123E3D423C8F15363572DC230314C025
:10F9EC0087CE67D7ECC18C0F83E7203BE720E53649
:10F9FC00B13F4506FA2A95D084F33BC126C6A3E451
:10FA0C008FC72B1E9CF64E3F412D412D4E3F9CF631
:10FA1C002B1E8FC7A3E426C63BC184F395D0FA2ACC
:10FA2C004506B13FE536E720203B83E78C0FECC160
:10FA3C0067D787CE14C0230372DC36358F15423C52
:10FA4C003E3D94126733E1D9000000C099CCE1D956
:10FA5C00C2C2941271EA423C8E233635EC3F23032A
:10FA6C00992887CE74F0ECC1E0C483E71BC9E7206A
:10FA7C00BBF9B13F6B2FFA2AC53E84F35D1B26C63A
:10FA8C00D5E18FC7B2C09CF6BFD2412D64094E3F61
:10FA9C0071382B1EDA39A3E47C0C3BC106D595D00A
:10FAAC004FC0450619DFE5367D18203B143E8C0F00
:10FABC00793167D7DDFC14C0CACA72DCBEC38F159E
:10FACC006CED3E3D1F266733004000001F2699CC8D
:10FADC006CEDC2C2BEC371EACACA8E23DDFCEC3F18
:10FAEC0079319928143E74F07D18E0C419DF1BC9D4
:10FAFC004FC0BBF906D56B2F7C0CC53EDA395D1BAC
:10FB0C007138D5E16409B2C0BFD2BFD2B2C06409AA
:10FB1C00D5E171385D1BDA39C53E7C0C6B2F06D5EF
:10FB2C00BBF94FC01BC919DFE0C47D1874F0143E3B
:10FB3C0099287931EC3FDDFC8E23CACA71EABEC329
:10FB4C00C2C26CED99CC1F260000004067331F2603
:10FB5C003E3D6CED8F15BEC372DCCACA14C0DDFC11
:10FB6C0067D779318C0F143E203B7D18E53619DFB1
:10FB7C0045064FC095D006D53BC17C0CA3E4DA39C1
:10FB8C002B1E71384E3F6409412DBFD29CF6B2C07A
:10FB9C008FC7D5E126C65D1B84F3C53EFA2A6B2FB1
:10FBAC00B13FBBF9E7201BC983E7E0C4ECC174F09B
:10FBBC0087CE99282303EC3F36358E23423C71EADD
:10FBCC009412C2C2E1D999CC00C00000E1D96733CC
:10FBDC0094123E3D423C8F15363572DC230314C023
:10FBEC0087CE67D7ECC18C0F83E7203BE720E53647
:10FBFC00B13F4506FA2A95D084F33BC126C6A3E44F
:10FC0C008FC72B1E9CF64E3F412D412D4E3F9CF62F
:10FC1C002B1E8FC7A3E426C63BC184F395D0FA2ACA
:10FC2C004506B13FE536E720203B83E78C0FECC15E
:10FC3C0067D787CE14C0230372DC36358F15423C50
:10FC4C003E3D94126733E1D9000000C099CCE1D954
:10FC5C00C2C2941271EA423C8E233635EC3F230328
:10FC6C00992887CE74F0ECC1E0C483E71BC9E72068
:10FC7C00BBF9B13F6B2FFA2AC53E84F35D1B26C638
:10FC8C00D5E18FC7B2C09CF6BFD2412D64094E3F5F
:10FC9C0071382B1EDA39A3E47C0C3BC106D595D008
:10FCAC004FC0450619DFE5367D18203B143E8C0FFE
:10FCBC00793167D7DDFC14C0CACA72DCBEC38F159C
:10FCCC006CED3E3D1F266733004000001F2699CC8B
:10FCDC006CEDC2C2BEC371EACACA8E23DDFCEC3F16
:10FCEC0079319928143E74F07D18E0C419DF1BC9D2
:10FCFC004FC0BBF906D56B2F7C0CC53EDA395D1BAA
:10FD0C007138D5E16409B2C0BFD2BFD2B2C06409A8
:10FD1C00D5E171385D1BDA39C53E7C0C6B2F06D5ED
:10FD2C00BBF94FC01BC919DFE0C47D1874F0143E39
:10FD3C0099287931EC3FDDFC8E23CACA71EABEC327
:10FD4C00C2C26CED99CC1F260000004067331F2601
:10FD5C003E3D6CED8F15BEC372DCCACA14C0DDFC0F
:10FD6C0067D779318C0F143E203B7D18E53619DFAF
:10FD7C0045064FC095D006D53BC17C0CA3E4DA39BF
:10FD8C002B1E71384E3F6409412DBFD29CF6B2C078
:10FD9C008FC7D5E126C65D1B84F3C53EFA2A6B2FAF
:10FDAC00B13FBBF9E7201BC983E7E0C4ECC174F099
:10FDBC0087CE99282303EC3F36358E23423C71EADB
:10FDCC009412C2C2E1D999CC00C00000E1D96733CA
:10FDDC0094123E3D423C8F15363572DC230314C021
:10FDEC0087CE67D7ECC18C0F83E7203BE720E53645
:10FDFC00B13F4506FA2A95D084F33BC126C6A3E44D
:10FE0C008FC72B1E9CF64E3F412D412D4E3F9CF62D
:10FE1C002B1E8FC7A3E426C63BC184F395D0FA2AC8
:10FE2C004506B13FE536E720203B83E78C0FECC15C
:10FE3C0067D787CE14C0230372DC36358F15423C4E
:10FE4C003E3D94126733E1D9000000C099CCE1D952
:10FE5C00C2C2941271EA423C8E233635EC3F230326
:10FE6C00992887CE74F0ECC1E0C483E71BC9E72066
:10FE7C00BBF9B13F6B2FFA2AC53E84F35D1B26C636
:10FE8C00D5E18FC7B2C09CF6BFD2412D64094E3F5D
:10FE9C0071382B1EDA39A3E47C0C3BC106D595D006
:10FEAC004FC0450619DFE5367D18203B143E8C0FFC
:10FEBC00793167D7DDFC14C0CACA72DCBEC38F159A
:10FECC006CED3E3D1F266733004000001F2699CC89
:10FEDC006CEDC2C2BEC371EACACA8E23DDFCEC3F14
:10FEEC0079319928143E74F07D18E0C419DF1BC9D0
:10FEFC004FC0BBF906D56B2F7C0CC53EDA395D1BA8
:10FF0C007138D5E16409B2C0BFD2BFD2B2C06409A6
:10FF1C00D5E171385D1BDA39C53E7C0C6B2F06D5EB
:10FF2C00BBF94FC01BC919DFE0C47D1874F0143E37
:10FF3C0099287931EC3FDDFC8E23CACA71EABEC325
:10FF4C00C2C26CED99CC1F260000004067331F26FF
:10FF5C003E3D6CED8F15BEC372DCCACA14C0DDFC0D
:10FF6C0067D779318C0F143E203B7D18E53619DFAD
:10FF7C0045064FC095D006D53BC17C0CA3E4DA39BD
:10FF8C002B1E71384E3F6409412DBFD29CF6B2C076
:10FF9C008FC7D5E126C65D1B84F3C53EFA2A6B2FAD
:10FFAC00B13FBBF9E7201BC983E7E0C4ECC174F097
:10FFBC0087CE99282303EC3F36358E23423C71EAD9
:10FFCC009412C2C2E1D999CC00C00000E1D96733C8
:10FFDC0094123E3D423C8F15363572DC230314C01F
:10FFEC0087CE67D7ECC18C0F83E7203BE720E53643
:04FFFC00B13F4506C6
:020000040801F1
:10000000FA2A95D084F33BC126C6A3E48FC72B1EE2
:100010009CF64E3F412D412D4E3F9CF62B1E8FC727
:10002000A3E426C63BC184F395D0FA2A4506B13F26
:10003000E536E720203B83E78C0FECC167D787CEFE
:1000400014C0230372DC36358F15423C3E3D9412BA
:100050006733E1D9000000C099CCE1D9C2C2941243
:1000600071EA423C8E233635EC3F2303992887CE34
:1000700074F0ECC1E0C483E71BC9E720BBF9B13FD2
:100080006B2FFA2AC53E84F35D1B26C6D5E18FC7C8
:10009000B2C09CF6BFD2412D64094E3F71382B1E71
:1000A000DA39A3E47C0C3BC106D595D04FC0450698
:1000B00019DFE5367D18203B143E8C0F793167D768
:1000C000DDFC14C0CACA72DCBEC38F156CED3E3DA8
:1000D0001F266733004000001F2699CC6CEDC2C27A
:1000E000BEC371EACACA8E23DDFCEC3F7931992880
:1000F000143E74F07D18E0C419DF1BC94FC0BBF972
:1001000006D56B2F7C0CC53EDA395D1B7138D5E105
:100110006409B2C0BFD2BFD2B2C06409D5E17138A0
:100120005D1BDA39C53E7C0C6B2F06D5BBF94FC081
:100130001BC919DFE0C47D1874F0143E9928793189
:10014000EC3FDDFC8E23CACA71EABEC3C2C26CEDAD
:1001500099CC1F260000004074325F27143E74F0D3
:10016000EF197EC5D5E18FC7F2C00FF595D0FA2AF9
:10017000B504D33F36358E23C53CEDEB8F15BEC39A
:10018000C3DDEEC94FC0BBF9DFD35A2E64094E3F21
:10019000AF378B1F203B83E7111152C2E1D999CCB5
:1001A00005C06EFE67D77931050E713EDA395D1BE9
:1001B0002A393AE37C0C3BC133D68ACF14C02303DF
:1001C00026DB533494123E3DB63B0817E53619DF63
:1001D000D5077CC0BFD2BFD27CC0D50719DFE536BA
:1001E0000817B63B3E3D9412533426DB230314C05C
:1001F0008ACF33D63BC17C0C3AE32A395D1BDA390E
:10020000713E050E793167D76EFE05C099CCE1D9F4
:1002100052C2111183E7203B8B1FAF374E3F640959
:100220005A2EDFD3BBF94FC0EEC9C3DDBEC38F1555
:10023000EDEBC53C8E233635D33FB504FA2A95D075
:100240000FF5F2C08FC7D5E17EC5EF1974F0143EEB
:100250005F277432004000005F278CCD74F0ECC142
:100260007EC511E68FC72B1E0FF50E3FFA2A6B2FA6
:10027000D33F4BFB8E23CACAEDEB3BC3BEC371EA2F
:10028000EEC93D22BBF9B13F5A2E212C4E3F9CF6C0
:100290008B1F51C883E7E0C452C2EFEE99CC1F26F2
:1002A0006EFEFB3F79319928713EFBF15D1B26C63E
:1002B0003AE3D6C63BC184F38ACFCD292303EC3F72
:1002C0005334DA243E3D6CED08174AC419DF1BC9CC
:1002D0007CC02BF8BFD2412DD507843FE536E720FF
:1002E000B63BF8E89412C2C226DBADCB14C0DDFCED
:1002F00033D676307C0CC53E2A39C61CDA39A3E4E5
:10030000050E8FC167D787CE05C09201E1D967334B
:100310001111AE3D203B7D18AF3775E06409B2C0C6
:10032000DFD3A6D14FC04506C3DD12368F15423C40
:10033000C53C1314363572DCB5042DC095D006D5F6
:10034000F2C0F10AD5E17138EF19823A143E8C0FF0
:100350007432A1D8000000C08CCDA1D8ECC18C0FA4
:1003600011E6823A2B1E71380E3FF10A6B2F06D52B
:100370004BFB2DC0CACA72DC3BC3131471EA423C6A
:100380003D221236B13F4506212CA6D19CF6B2C0C3
:1003900051C875E0E0C47D18EFEEAE3D1F2667330F
:1003A000FB3F9201992887CEFBF18FC126C6A3E4BB
:1003B000D6C6C61C84F3C53ECD297630EC3FDDFCA5
:1003C000DA24ADCB6CEDC2C24AC4F8E81BC9E72001
:1003D0002BF8843F412D412D843F2BF8E7201BC98A
:1003E000F8E84AC4C2C26CEDADCBDA24DDFCEC3FC8
:1003F0007630CD29C53E84F3C61CD6C6A3E426C6F6
:100400008FC1FBF187CE99289201FB3F67331F26EE
:10041000AE3DEFEE7D18E0C475E051C8B2C09CF669
:10042000A6D1212C4506B13F12363D22423C71EA4D
:1004300013143BC372DCCACA2DC04BFB06D56B2F0D
:10044000F10A0E3F71382B1E823A11E68C0FECC177
:10045000A1D88CCD00C00000A1D874328C0F143EFE
:10046000823AEF197138D5E1F10AF2C006D595D07C
:100470002DC0B50472DC36351314C53C423C8F15D3
:100480001236C3DD45064FC0A6D1DFD3B2C0640922
:1004900075E0AF377D18203BAE3D11116733E1D9D0
:1004A000920105C087CE67D78FC1050EA3E4DA3964
:1004B000C61C2A39C53E7C0C763033D6DDFC14C010
:1004C000ADCB26DBC2C29412F8E8B63BE720E53696
:1004D000843FD507412DBFD22BF87CC01BC919DF43
:1004E0004AC408176CED3E3DDA245334EC3F230335
:1004F000CD298ACF84F33BC1D6C63AE326C65D1B1D
:10050000FBF1713E99287931FB3F6EFE1F2699CC95
:10051000EFEE52C2E0C483E751C88B1F9CF64E3FFA
:10052000212C5A2EB13FBBF93D22EEC971EABEC360
:100530003BC3EDEBCACA8E234BFBD33F6B2FFA2A8A
:100540000E3F0FF52B1E8FC711E67EC5ECC174F070
:100550008CCD5F270000004074325F27143E74F09A
:10056000EF197EC5D5E18FC7F2C00FF595D0FA2AF5
:10057000B504D33F36358E23C53CEDEB8F15BEC396
:10058000C3DDEEC94FC0BBF9DFD35A2E64094E3F1D
:10059000AF378B1F203B83E7111152C2E1D999CCB1
:1005A00005C06EFE67D77931050E713EDA395D1BE5
:1005B0002A393AE37C0C3BC133D68ACF14C02303DB
:1005C00026DB533494123E3DB63B0817E53619DF5F
:1005D000D5077CC0BFD2BFD27CC0D50719DFE536B6
:1005E0000817B63B3E3D9412533426DB230314C058
:1005F0008ACF33D63BC17C0C3AE32A395D1BDA390A
:10060000713E050E793167D76EFE05C099CCE1D9F0
:1006100052C2111183E7203B8B1FAF374E3F640955
:100620005A2EDFD3BBF94FC0EEC9C3DDBEC38F1551
:10063000EDEBC53C8E233635D33FB504FA2A95D071
:100640000FF5F2C08FC7D5E17EC5EF1974F0143EE7
:100650005F277432004000005F278CCD74F0ECC13E
:100660007EC511E68FC72B1E0FF50E3FFA2A6B2FA2
:10067000D33F4BFB8E23CACAEDEB3BC3BEC371EA2B
:10068000EEC93D22BBF9B13F5A2E212C4E3F9CF6BC
:100690008B1F51C883E7E0C452C2EFEE99CC1F26EE
:1006A0006EFEFB3F79319928713EFBF15D1B26C63A
:1006B0003AE3D6C63BC184F38ACFCD292303EC3F6E
:1006C0005334DA243E3D6CED08174AC419DF1BC9C8
:1006D0007CC02BF8BFD2412DD507843FE536E720FB
:1006E000B63BF8E89412C2C226DBADCB14C0DDFCE9
:1006F00033D676307C0CC53E2A39C61CDA39A3E4E1
:10070000050E8FC167D787CE05C09201E1D9673347
:100710001111AE3D203B7D18AF3775E06409B2C0C2
:10072000DFD3A6D14FC04506C3DD12368F15423C3C
:10073000C53C1314363572DCB5042DC095D006D5F2
:10074000F2C0F10AD5E17138EF19823A143E8C0FEC
:100750007432A1D8000000C08CCDA1D8ECC18C0FA0
:1007600011E6823A2B1E71380E3FF10A6B2F06D527
:100770004BFB2DC0CACA72DC3BC3131471EA423C66
:100780003D221236B13F4506212CA6D19CF6B2C0BF
:1007900051C875E0E0C47D18EFEEAE3D1F2667330B
:1007A000FB3F9201992887CEFBF18FC126C6A3E4B7
:1007B000D6C6C61C84F3C53ECD297630EC3FDDFCA1
:1007C000DA24ADCB6CEDC2C24AC4F8E81BC9E720FD
:1007D0002BF8843F412D412D843F2BF8E7201BC986
:1007E000F8E84AC4C2C26CEDADCBDA24DDFCEC3FC4
:1007F0007630CD29C53E84F3C61CD6C6A3E426C6F2
:100800008FC1FBF187CE99289201FB3F67331F26EA
:10081000AE3DEFEE7D18E0C475E051C8B2C09CF665
:10082000A6D1212C4506B13F12363D22423C71EA49
:1008300013143BC372DCCACA2DC04BFB06D56B2F09
:10084000F10A0E3F71382B1E823A11E68C0FECC173
:10085000A1D88CCD00C00000A1D874328C0F143EFA
:10086000823AEF197138D5E1F10AF2C006D595D078
:100870002DC0B50472DC36351314C53C423C8F15CF
:100880001236C3DD45064FC0A6D1DFD3B2C064091E
:1008900075E0AF377D18203BAE3D11116733E1D9CC
:1008A000920105C087CE67D78FC1050EA3E4DA3960
:1008B000C61C2A39C53E7C0C763033D6DDFC14C00C
:1008C000ADCB26DBC2C29412F8E8B63BE720E53692
:1008D000843FD507412DBFD22BF87CC01BC919DF3F
:1008E0004AC408176CED3E3DDA245334EC3F230331
:1008F000CD298ACF84F33BC1D6C63AE326C65D1B19
:10090000FBF1713E99287931FB3F6EFE1F2699CC91
:10091000EFEE52C2E0C483E751C88B1F9CF64E3FF6
:10092000212C5A2EB13FBBF93D22EEC971EABEC35C
:100930003BC3EDEBCACA8E234BFBD33F6B2FFA2A86
:100940000E3F0FF52B1E8FC711E67EC5ECC174F06C
:100950008CCD5F270205070A0C0F111416191B1EF8
:100960000306080B0D101215171A1C1F0104201D79
:100970000E0913180000000000000000010203042B
:100980000607080900000040203B83E7BFD2BFD222
:1009900083E7203B0040000083E7E0C4BFD2412D45
:1009A000203B7D18000000C0E0C47D18412D412D82
:1009B0007D18E0C400C000007D18203B412DBFD24F
:1009C000E0C483E700000040203B83E7BFD2BFD2F2
:1009D00083E7203B0040000083E7E0C4BFD2412D05
:1009E000203B7D18000000C0E0C47D18412D412D42
:1009F0007D18E0C400C000007D18203B412DBFD20F
:100A0000E0C483E700000040203B83E7BFD2BFD2B1
:100A100083E7203B0040000083E7E0C4BFD2412DC4
:100A2000203B7D18000000C0E0C47D18412D412D01
:100A30007D18E0C400C000007D18203B412DBFD2CE
:100A4000E0C483E700000040203B83E7BFD2BFD271
:100A500083E7203B0040000083E7E0C4BFD2412D84
:100A6000203B7D18000000C0E0C47D18412D412DC1
:100A70007D18E0C400C000007D18203B412DBFD28E
:100A8000E0C483E700000040203B83E7BFD2BFD231
:100A900083E7203B0040000083E7E0C4BFD2412D44
:100AA000203B7D18000000C0E0C47D18412D412D81
:100AB0007D18E0C400C000007D18203B412DBFD24E
:100AC000E0C483E700000040203B83E7BFD2BFD2F1
:100AD00083E7203B0040000083E7E0C4BFD2412D04
:100AE000203B7D18000000C0E0C47D18412D412D41
:100AF0007D18E0C400C000007D18203B412DBFD20E
:100B0000E0C483E700000040203B83E7BFD2BFD2B0
:100B100083E7203B0040000083E7E0C4BFD2412DC3
:100B2000203B7D18000000C0E0C47D18412D412D00
:100B30007D18E0C400C000007D18203B412DBFD2CD
:100B4000E0C483E700000040203B83E7BFD2BFD270
:100B500083E7203B0040000083E7E0C4BFD2412D83
:100B6000203B7D18000000C0E0C47D18412D412DC0
:100B70007D18E0C400C000007D18203B412DBFD28D
:100B8000E0C483E700000040203B83E7BFD2BFD230
:100B900083E7203B0040000083E7E0C4BFD2412D43
:100BA000203B7D18000000C0E0C47D18412D412D80
:100BB0007D18E0C400C000007D18203B412DBFD24D
:100BC000E0C483E700000040203B83E7BFD2BFD2F0
:100BD00083E7203B0040000083E7E0C4BFD2412D03
:100BE000203B7D18000000C0E0C47D18412D412D40
:100BF0007D18E0C400C000007D18203B412DBFD20D
:100C0000E0C483E700000040203B83E7BFD2BFD2AF
:100C100083E7203B0040000083E7E0C4BFD2412DC2
:100C2000203B7D18000000C0E0C47D18412D412DFF
:100C30007D18E0C400C000007D18203B412DBFD2CC
:100C4000E0C483E700000040203B83E7BFD2BFD26F
:100C500083E7203B0040000083E7E0C4BFD2412D82
:100C6000203B7D18000000C0E0C47D18412D412DBF
:100C70007D18E0C400C000007D18203B412DBFD28C
:100C8000E0C483E700000040203B83E7BFD2BFD22F
:100C900083E7203B0040000083E7E0C4BFD2412D42
:100CA000203B7D18000000C0E0C47D18412D412D7F
:100CB0007D18E0C400C000007D18203B412DBFD24C
:100CC000E0C483E700000040203B83E7BFD2BFD2EF
:100CD00083E7203B0040000083E7E0C4BFD2412D02
:100CE000203B7D18000000C0E0C47D18412D412D3F
:100CF0007D18E0C400C000007D18203B412DBFD20C
:100D0000E0C483E700000040203B83E7BFD2BFD2AE
:100D100083E7203B0040000083E7E0C4BFD2412DC1
:100D2000203B7D18000000C0E0C47D18412D412DFE
:100D30007D18E0C400C000007D18203B412DBFD2CB
:100D4000E0C483E700000040203B83E7BFD2BFD26E
:100D500083E7203B0040000083E7E0C4BFD2412D81
:100D6000203B7D18000000C0E0C47D18412D412DBE
:100D70007D18E0C400C000007D18203B412DBFD28B
:100D8000E0C483E700000040203B83E7BFD2BFD22E
:100D900083E7203B0040000083E7E0C4BFD2412D41
:100DA000203B7D18000000C0E0C47D18412D412D7E
:100DB0007D18E0C400C000007D18203B412DBFD24B
:100DC000E0C483E700000040203B83E7BFD2BFD2EE
:100DD00083E7203B0040000083E7E0C4BFD2412D01
:100DE000203B7D18000000C0E0C47D18412D412D3E
:100DF0007D18E0C400C000007D18203B412DBFD20B
:100E0000E0C483E700000040203B83E7BFD2BFD2AD
:100E100083E7203B0040000083E7E0C4BFD2412DC0
:100E2000203B7D18000000C0E0C47D18412D412DFD
:100E30007D18E0C400C000007D18203B412DBFD2CA
:100E4000E0C483E700000040203B83E7BFD2BFD26D
:100E500083E7203B0040000083E7E0C4BFD2412D80
:100E6000203B7D18000000C0E0C47D18412D412DBD
:100E70007D18E0C400C000007D18203B412DBFD28A
:100E8000E0C483E700000040203B83E7BFD2BFD22D
:100E900083E7203B0040000083E7E0C4BFD2412D40
:100EA000203B7D18000000C0E0C47D18412D412D7D
:100EB0007D18E0C400C000007D18203B412DBFD24A
:100EC000E0C483E700000040203B83E7BFD2BFD2ED
:100ED00083E7203B0040000083E7E0C4BFD2412D00
:100EE000203B7D18000000C0E0C47D18412D412D3D
:100EF0007D18E0C400C000007D18203B412DBFD20A
:100F0000E0C483E700000040203B83E7BFD2BFD2AC
:100F100083E7203B0040000083E7E0C4BFD2412DBF
:100F2000203B7D18000000C0E0C47D18412D412DFC
:100F30007D18E0C400C000007D18203B412DBFD2C9
:100F4000E0C483E700000040203B83E7BFD2BFD26C
:100F500083E7203B0040000083E7E0C4BFD2412D7F
:100F6000203B7D18000000C0E0C47D18412D412DBC
:100F70007D18E0C400C000007D18203B412DBFD289
:100F8000E0C483E700000040203B83E7BFD2BFD22C
:100F900083E7203B0040000083E7E0C4BFD2412D3F
:100FA000203B7D18000000C0E0C47D18412D412D7C
:100FB0007D18E0C400C000007D18203B412DBFD249
:100FC000E0C483E700000040203B83E7BFD2BFD2EC
:100FD00083E7203B0040000083E7E0C4BFD2412DFF
:100FE000203B7D18000000C0E0C47D18412D412D3C
:100FF0007D18E0C400C000007D18203B412DBFD209
:10100000E0C483E700000040203B83E7BFD2BFD2AB
:1010100083E7203B0040000083E7E0C4BFD2412DBE
:10102000203B7D18000000C0E0C47D18412D412DFB
:101030007D18E0C400C000007D18203B412DBFD2C8
:10104000E0C483E700000040203B83E7BFD2BFD26B
:1010500083E7203B0040000083E7E0C4BFD2412D7E
:10106000203B7D18000000C0E0C47D18412D412DBB
:101070007D18E0C400C000007D18203B412DBFD288
:10108000E0C483E700000040203B83E7BFD2BFD22B
:1010900083E7203B0040000083E7E0C4BFD2412D3E
:1010A000203B7D18000000C0E0C47D18412D412D7B
:1010B0007D18E0C400C000007D18203B412DBFD248
:1010C000E0C483E700000040203B83E7BFD2BFD2EB
:1010D00083E7203B0040000083E7E0C4BFD2412DFE
:1010E000203B7D18000000C0E0C47D18412D412D3B
:1010F0007D18E0C400C000007D18203B412DBFD208
:10110000E0C483E700000040203B83E7BFD2BFD2AA
:1011100083E7203B0040000083E7E0C4BFD2412DBD
:10112000203B7D18000000C0E0C47D18412D412DFA
:101130007D18E0C400C000007D18203B412DBFD2C7
:10114000E0C483E700000040203B83E7BFD2BFD26A
:1011500083E7203B0040000083E7E0C4BFD2412D7D
:10116000203B7D18000000C0E0C47D18412D412DBA
:101170007D18E0C400C000007D18203B412DBFD287
:10118000E0C483E700000040B63BF8E806D595D000
:101190003AE32A39B13F4506EFEE52C299CC1F26F9
:1011A00012363D227C0C3BC1F2C0F10AE720E53645
:1011B0005F278CCDC2C26CEDB504D33FDA39A3E40E
:1011C000A6D1DFD383E7203BFB3F920171EABEC388
:1011D0008ACFCD2971382B1ED5077CC0ECC18C0F6E
:1011E000DA2453348E23CACA8FC1FBF164094E3FFF
:1011F000AF3775E087CE67D7EDEBC53CEC3FDDFC44
:1012000011E67EC5BFD2412D823AEF19230314C0E7
:101210003BC31314992879318B1F51C8B2C09CF677
:10122000050E713E363572DCADCB26DB74F0143E14
:10123000843F2BF8D5E18FC733D67630423C8F15EB
:101240006EFE05C0E0C47D18212C5A2E5D1B26C6FB
:101250002DC04BFB94123E3D7432A1D81BC919DF3F
:101260000FF50E3FC53E84F3C3DDEEC9E1D9673308
:10127000AE3D1111BBF94FC0D6C6C61C6B2FFA2A62
:1012800008174AC400C000000817B63B6B2F06D5EC
:10129000D6C63AE3BBF9B13FAE3DEFEEE1D999CC0A
:1012A000C3DD1236C53E7C0C0FF5F2C01BC9E7202A
:1012B00074325F279412C2C22DC0B5045D1BDA39A7
:1012C000212CA6D1E0C483E76EFEFB3F423C71EACD
:1012D00033D68ACFD5E17138843FD50774F0ECC19D
:1012E000ADCBDA2436358E23050E8FC1B2C064092A
:1012F0008B1FAF37992887CE3BC3EDEB2303EC3F21
:10130000823A11E6BFD2BFD211E6823AEC3F230304
:10131000EDEB3BC387CE9928AF378B1F6409B2C072
:101320008FC1050E8E233635DA24ADCBECC174F0B7
:10133000D507843F7138D5E18ACF33D671EA423C74
:10134000FB3F6EFE83E7E0C4A6D1212CDA395D1B9A
:10135000B5042DC0C2C294125F277432E7201BC9A6
:10136000F2C00FF57C0CC53E1236C3DD99CCE1D935
:10137000EFEEAE3DB13FBBF93AE3D6C606D56B2FD3
:10138000B63B0817000000C04AC40817FA2A6B2FA2
:10139000C61CD6C64FC0BBF91111AE3D6733E1D9AB
:1013A000EEC9C3DD84F3C53E0E3F0FF519DF1BC93F
:1013B000A1D874323E3D94124BFB2DC026C65D1B56
:1013C0005A2E212C7D18E0C405C06EFE8F15423CBC
:1013D000763033D68FC7D5E12BF8843F143E74F0B6
:1013E00026DBADCB72DC3635713E050E9CF6B2C005
:1013F00051C88B1F7931992813143BC314C02303A0
:10140000EF19823A412DBFD27EC511E6DDFCEC3FDB
:10141000C53CEDEB67D787CE75E0AF374E3F64092B
:10142000FBF18FC1CACA8E235334DA248C0FECC16E
:101430007CC0D5072B1E7138CD298ACFBEC371EA77
:101440009201FB3F203B83E7DFD3A6D1A3E4DA3947
:10145000D33FB5046CEDC2C28CCD5F27E536E720E3
:10146000F10AF2C03BC17C0C3D2212361F2699CCFA
:1014700052C2EFEE4506B13F2A393AE395D006D580
:10148000F8E8B63B00400000F8E84AC495D0FA2AD4
:101490002A39C61C45064FC052C211111F26673398
:1014A0003D22EEC93BC184F3F10A0E3FE53619DF58
:1014B0008CCDA1D86CED3E3DD33F4BFBA3E426C6BB
:1014C000DFD35A2E203B7D18920105C0BEC38F1575
:1014D000CD2976302B1E8FC77CC02BF88C0F143E85
:1014E000533426DBCACA72DCFBF1713E4E3F9CF6D8
:1014F00075E051C867D77931C53C1314DDFC14C0C1
:101500007EC5EF19412D412DEF197EC514C0DDFCBC
:101510001314C53C793167D751C875E09CF64E3F2E
:10152000713EFBF172DCCACA26DB5334143E8C0FC9
:101530002BF87CC08FC72B1E7630CD298F15BEC3EC
:1015400005C092017D18203B5A2EDFD326C6A3E4A6
:101550004BFBD33F3E3D6CEDA1D88CCD19DFE5367A
:101560000E3FF10A84F33BC1EEC93D2267331F26CB
:10157000111152C24FC04506C61C2A39FA2A95D00D
:101580004AC4F8E800000040B63BF8E806D595D01C
:101590003AE32A39B13F4506EFEE52C299CC1F26F5
:1015A00012363D227C0C3BC1F2C0F10AE720E53641
:1015B0005F278CCDC2C26CEDB504D33FDA39A3E40A
:1015C000A6D1DFD383E7203BFB3F920171EABEC384
:1015D0008ACFCD2971382B1ED5077CC0ECC18C0F6A
:1015E000DA2453348E23CACA8FC1FBF164094E3FFB
:1015F000AF3775E087CE67D7EDEBC53CEC3FDDFC40
:1016000011E67EC5BFD2412D823AEF19230314C0E3
:101610003BC31314992879318B1F51C8B2C09CF673
:10162000050E713E363572DCADCB26DB74F0143E10
:10163000843F2BF8D5E18FC733D67630423C8F15E7
:101640006EFE05C0E0C47D18212C5A2E5D1B26C6F7
:101650002DC04BFB94123E3D7432A1D81BC919DF3B
:101660000FF50E3FC53E84F3C3DDEEC9E1D9673304
:10167000AE3D1111BBF94FC0D6C6C61C6B2FFA2A5E
:1016800008174AC400C000000817B63B6B2F06D5E8
:10169000D6C63AE3BBF9B13FAE3DEFEEE1D999CC06
:1016A000C3DD1236C53E7C0C0FF5F2C01BC9E72026
:1016B00074325F279412C2C22DC0B5045D1BDA39A3
:1016C000212CA6D1E0C483E76EFEFB3F423C71EAC9
:1016D00033D68ACFD5E17138843FD50774F0ECC199
:1016E000ADCBDA2436358E23050E8FC1B2C0640926
:1016F0008B1FAF37992887CE3BC3EDEB2303EC3F1D
:10170000823A11E6BFD2BFD211E6823AEC3F230300
:10171000EDEB3BC387CE9928AF378B1F6409B2C06E
:101720008FC1050E8E233635DA24ADCBECC174F0B3
:10173000D507843F7138D5E18ACF33D671EA423C70
:10174000FB3F6EFE83E7E0C4A6D1212CDA395D1B96
:10175000B5042DC0C2C294125F277432E7201BC9A2
:10176000F2C00FF57C0CC53E1236C3DD99CCE1D931
:10177000EFEEAE3DB13FBBF93AE3D6C606D56B2FCF
:10178000B63B0817000000C04AC40817FA2A6B2F9E
:10179000C61CD6C64FC0BBF91111AE3D6733E1D9A7
:1017A000EEC9C3DD84F3C53E0E3F0FF519DF1BC93B
:1017B000A1D874323E3D94124BFB2DC026C65D1B52
:1017C0005A2E212C7D18E0C405C06EFE8F15423CB8
:1017D000763033D68FC7D5E12BF8843F143E74F0B2
:1017E00026DBADCB72DC3635713E050E9CF6B2C001
:1017F00051C88B1F7931992813143BC314C023039C
:10180000EF19823A412DBFD27EC511E6DDFCEC3FD7
:10181000C53CEDEB67D787CE75E0AF374E3F640927
:10182000FBF18FC1CACA8E235334DA248C0FECC16A
:101830007CC0D5072B1E7138CD298ACFBEC371EA73
:101840009201FB3F203B83E7DFD3A6D1A3E4DA3943
:10185000D33FB5046CEDC2C28CCD5F27E536E720DF
:10186000F10AF2C03BC17C0C3D2212361F2699CCF6
:1018700052C2EFEE4506B13F2A393AE395D006D57C
:10188000F8E8B63B00400000F8E84AC495D0FA2AD0
:101890002A39C61C45064FC052C211111F26673394
:1018A0003D22EEC93BC184F3F10A0E3FE53619DF54
:1018B0008CCDA1D86CED3E3DD33F4BFBA3E426C6B7
:1018C000DFD35A2E203B7D18920105C0BEC38F1571
:1018D000CD2976302B1E8FC77CC02BF88C0F143E81
:1018E000533426DBCACA72DCFBF1713E4E3F9CF6D4
:1018F00075E051C867D77931C53C1314DDFC14C0BD
:101900007EC5EF19412D412DEF197EC514C0DDFCB8
:101910001314C53C793167D751C875E09CF64E3F2A
:10192000713EFBF172DCCACA26DB5334143E8C0FC5
:101930002BF87CC08FC72B1E7630CD298F15BEC3E8
:1019400005C092017D18203B5A2EDFD326C6A3E4A2
:101950004BFBD33F3E3D6CEDA1D88CCD19DFE53676
:101960000E3FF10A84F33BC1EEC93D2267331F26C7
:10197000111152C24FC04506C61C2A39FA2A95D009
:101980004AC4F8E800000040423C71EA67D787CEBD
:1019900019DFE536C53E7C0C9CF6B2C08FC72B1E06
:1019A0006B2FFA2A7D18E0C414C0DDFC94123E3D72
:1019B0006733E1D9CACA72DC74F0143EB13FBBF997
:1019C000A3E426C6BFD2412DDA395D1B45064FC0C0
:1019D000ECC18C0F8E2336351F2699CCC2C26CED1C
:1019E0002303EC3F203B83E706D595D0D5E1713842
:1019F0004E3F640984F33BC11BC9E7207931992824
:101A00008F15BEC300C000008F15423C793167D7E7
:101A10001BC919DF84F3C53E4E3F9CF6D5E18FC745
:101A200006D56B2F203B7D18230314C0C2C294122D
:101A30001F2667338E23CACAECC174F04506B13F36
:101A4000DA39A3E4BFD2BFD2A3E4DA39B13F450605
:101A500074F0ECC1CACA8E2367331F269412C2C227
:101A600014C023037D18203B6B2F06D58FC7D5E10B
:101A70009CF64E3FC53E84F319DF1BC967D7793109
:101A8000423C8F15000000C0BEC38F1599287931E4
:101A9000E7201BC93BC184F364094E3F7138D5E18F
:101AA00095D006D583E7203BEC3F23036CEDC2C203
:101AB00099CC1F2636358E238C0FECC14FC04506BE
:101AC0005D1BDA39412DBFD226C6A3E4BBF9B13F75
:101AD000143E74F072DCCACAE1D967333E3D9412F9
:101AE000DDFC14C0E0C47D18FA2A6B2F2B1E8FC7B3
:101AF000B2C09CF67C0CC53EE53619DF87CE67D7B1
:101B000071EA423C0040000071EABEC387CE9928CA
:101B1000E536E7207C0C3BC1B2C064092B1E71384E
:101B2000FA2A95D0E0C483E7DDFCEC3F3E3D6CED46
:101B3000E1D999CC72DC3635143E8C0FBBF94FC01D
:101B400026C65D1B412D412D5D1B26C64FC0BBF92E
:101B50008C0F143E363572DC99CCE1D96CED3E3DEC
:101B6000EC3FDDFC83E7E0C495D0FA2A71382B1EE8
:101B70006409B2C03BC17C0CE720E536992887CECA
:101B8000BEC371EA00000040423C71EA67D787CECD
:101B900019DFE536C53E7C0C9CF6B2C08FC72B1E04
:101BA0006B2FFA2A7D18E0C414C0DDFC94123E3D70
:101BB0006733E1D9CACA72DC74F0143EB13FBBF995
:101BC000A3E426C6BFD2412DDA395D1B45064FC0BE
:101BD000ECC18C0F8E2336351F2699CCC2C26CED1A
:101BE0002303EC3F203B83E706D595D0D5E1713840
:101BF0004E3F640984F33BC11BC9E7207931992822
:101C00008F15BEC300C000008F15423C793167D7E5
:101C10001BC919DF84F3C53E4E3F9CF6D5E18FC743
:101C200006D56B2F203B7D18230314C0C2C294122B
:101C30001F2667338E23CACAECC174F04506B13F34
